:1000000000400020B5690000F5690000F7690000B4
:1000100000000000000000000000000000000000E0
:10002000000000000000000000000000F96900006E
:100030000000000000000000FB690000FD690000F6
:10004000FF690000454D0000316E0000FF690000AF
:10005000FF69000000000000FF690000FF69000068
:10006000FF69000001710000C52C0000FF6900005D
:10007000FF690000FF690000FF690000FF690000E0
:10008000FF69000099720000FF690000FF6900002D
:10009000FF690000FF690000FF690000FF690000C0
:1000A000FF690000FF690000000000000000000080
:1000B0000000000000000000000000000000000040
:1000C00010B5064C2378002B07D1054B002B02D02E
:1000D000044800E000BF0123237010BD600200202F
:1000E0000000000060DB0000044B10B5002B03D0C3
:1000F0000349044800E000BF10BDC04600000000F6
:100100006402002060DB0000164B002B00D1144B72
:100110009D46402292029A1A924600218B460F4633
:100120001348144A121A0AF05FFE0F4B002B00D03E
:1001300098470E4B002B00D0984700200021040068
:100140000D000D48002802D00C4800E000BF0AF066
:100150000BFE2000290006F089FE0AF0DFFDC046F4
:100160000000080000400020000000000000000027
:1001700060020020982F0020000000000000000016
:100180000123034010D104280CD90268120909D0B8
:10019000531E9B001A1DC1180979002902D0013392
:1001A0009342F8D1180070470023FBE70378002B37
:1001B00003D05AB2002A01DB013070473F2293433B
:1001C000C03B59424B41C01803789343802BF4D174
:1001D0000130F9E710B500240378002B01D120008D
:1001E00010BDFFF7E3FF0134F6E770B5002204000D
:1001F0000D00411C092003F075F8002806D00123EA
:100200006200134343600023A34200DB70BD9A00E9
:10021000A958821891600133F6E770B5012803DC14
:100220001C2000F0A1FE70BD01230D6811201D42AD
:10023000F7D04868184206D1042804D90F23026871
:100240001340042B01D00E20EBE702F0B5FE6D1039
:100250000400002D03DDFFF7BDFFA84206DA1220DF
:10026000DFE72000FFF7A2FF0400013D012DF8D1D8
:1002700020787F2809DDDF280BDCF8233F22DB0014
:10028000800118406378134018430123400018434D
:10029000C9E7EF280BDCFC22637812019B011340B5
:1002A0003F220007000C0343A0781040ECE7F7283A
:1002B00012DCFC22637892021B031340E0228004CC
:1002C000520310403F221843E3781340FC220343BB
:1002D000A07812018001E8E701204042D5E7F0B59F
:1002E000070085B00D001C20012F06DD4C6801239E
:1002F00022001A40019203D10D2000F035FE54E097
:10030000022F02D08A681A42F6D001232E681E42BC
:1003100000D07EE0042E00D87BE01C41002C00DCE5
:100320001C000F2332681340092B29D173685B101E
:100330000193022F05D0AB68019A5B109A4200DD51
:100340000193019B01221F1B0137FB43DB171F4059
:10035000791C092002F0C6FF061E09D001237F0088
:100360001F4303002A68083347600199A14202DA5B
:10037000300005B0F0BD0134A100515802C3F4E7CC
:10038000042B46D1300002F017FEFFF723FF029046
:10039000022F04D0AB685B10984200DD0293029BF1
:1003A0009C4204DD002003F009F80600E0E730007D
:1003B00002F002FE0700019B9C4222DC3000019704
:1003C00002F0FAFD03903800FFF7F0FE029B0134C3
:1003D0000700A342F7DA019BC71A380002F0EEFFCC
:1003E000061EC5D002F0E8FD0400286802F0E4FD16
:1003F000039A019B991A41183A0020000AF0D8FC90
:10040000B6E73800FFF7D2FE019B070001330193E6
:10041000D1E7212071E7F8B54D680F00EB0706D44E
:10042000042D04D90F232E683340092B03D00B2051
:1004300000F09AFDF8BD6B6836095C10731EA3428C
:100440000FD80321200008F08BFB6421642803DC13
:100450000100032800DA03212800891902F072FF45
:1004600005002B6800201B09013B9C42E2D23A6840
:10047000A31C9B005A510123013464001C436C608F
:10048000D8E7F0B585B0012803DC1C2000F06CFD36
:100490002AE001244D682200022806D08B682342FE
:1004A00003D05C10002C00DC140001231D4200D09E
:1004B00073E0042D00D870E00F272B680E683B40D6
:1004C000042B27D1033B1E4205D1042E03D93368E8
:1004D0001F40042F01D00E20D8E72800FFF750FE60
:1004E000A04203DA0120404205B0F0BD280002F02E
:1004F00063FD0700300002F05FFD013C0100381988
:100500000BF028F80028EDD00123C01B013040007B
:100510001843E9E7092B40D16B685B1000939C42BC
:10052000E0DC01231E4230D1042E2ED933683B403B
:10053000042B2AD1300002F03FFD012302900193E9
:100540000397671CBB00E858864203D101986400FA
:100550002043C9E7019B18420ED104280CD9036837
:10056000039A1340042B07D102F026FD01000298E4
:100570000AF0BAFF0028E9D0009B3C009F42E0DD72
:10058000B0E71C00009B9C42ACDC631C9A00AA589C
:10059000B242F6D164000120DAE7212076E710B5F7
:1005A00002F0EEFC43000120184310BD10B57F2976
:1005B00002DC0170013010BD1A4B99420CDC402363
:1005C0008A115B42134303703F230B408021494251
:1005D000194341700230EEE7134B994210DC20239F
:1005E0000A135B4213433F24802203708B11524253
:1005F0002340214013430A43437082700330DAE7FB
:100600000A4B9942D7DCF0230370603B4370113BE7
:100610008A11FF3B1A4382703F2211401943C17077
:100620000430C8E7FF070000FFFF0000FF0F0100D4
:10063000F0B50D0085B0002803DC1C2000F094FC10
:100640000DE009680122080010400AD002AC1141F7
:100650002000FFF7ABFF011B200002F0BBFE0400EF
:100660001AE004293FD90F230C682340092B3AD103
:100670004B685B10019303239C46019B9A420EDD5D
:1006800002F09CFE041E07D02E68012502F094FCA7
:100690002F00019B9D421DDD200005B0F0BD013201
:1006A0009300CC580123234001D10D20C6E76410EC
:1006B0007F2C0DDD0D4E0223B44209DD0C4E634646
:1006C000B44205DD00270B4EE30FA6427B419B00A1
:1006D000C018D2E70135AB00F1583942E5D04910D6
:1006E000FFF764FFD5E72120A8E7C046FF07000019
:1006F000FFFF0000FF0F010010B5040001200840BB
:1007000010D104290DD90F230A681340042B08D1F6
:10071000080002F051FC010020000AF0E5FE43420F
:10072000584110BD0020FCE7F7B50F00012803DC9D
:100730001C2000F019FCFEBD01264D682E4006D19C
:10074000042D04D90F222B681A40092A01D00B204E
:10075000EFE76A681B095410A34200D85C1E396891
:100760001E48FFF7C9FF01230190002813D1396803
:100770001B48FFF7C1FF002811D0002C0DD001232A
:10078000621C013C9C409200535123436B6004E087
:100790000136B200AB50B442FADA0020CBE73B6836
:1007A0000D20DA07C5D55B10002B11DD9C420FDB55
:1007B0009B00A200291DEB1889180433994209D126
:1007C0000123013C9C40AA181C4353606C60E4E781
:1007D0001220AEE758681860EFE7C04673C4000007
:1007E00077C40000002310B50C000B70C30705D5BB
:1007F0000D49421020000AF03BFE08E00B4900289A
:1008000002D0042804D10A4920000AF051FE10BD8C
:100810000428FCD90F2302681340042BF7D102F0FF
:10082000CBFB04490200E5E774CD00007CC4000066
:1008300082C4000087C40000F0B593B003900300A9
:1008400002911C20012B1DDD029B01251B681C0051
:100850002C4000D0A8E0042B00D8A5E01A680F2394
:100860001A40092A48D10194019A029992008A58A3
:1008700016002E4005D1042A03D910681840092813
:1008800004D0222000F070FB07002CE052685210C8
:10089000A418019A013201920199039A8A42E3D184
:1008A000611C012202F01EFD071E01D100271AE083
:1008B00064002543456005000835029AB300D1580D
:1008C0004B680A685B1012099A4200D8531E002236
:1008D00093420BDCDA43D21713409B00ED18019BC7
:1008E00001369E42E9DB380013B0F0BD90000C18D1
:1008F000A46801322C50EBE7042A55D12F002600C2
:100900001D00029AB300D058384237D1042835D997
:1009100003682B40042BB4D1FFF732FC039B013654
:100920002418B342EDD1200002F048FD071EBDD0CF
:10093000039B029D9B00EB18041D029301232E686C
:100940001E4222D1042E20D90F2233681340042BDB
:100950000DD13000FFF714FC0190300002F02CFBA9
:10096000019A010020000AF023FA019BE418029B7F
:100970000435AB42E2D100232370B4E705A9FFF7A9
:1009800031FF05A80AF0BAFDC8E705A93000FFF756
:1009900029FF05A80AF0B2FD0600020005A9200003
:1009A0000AF006FAA419E2E7212000F0DDFA7DE75B
:1009B000F0B50D0095B0002806DC1C2000F0D4FA3C
:1009C0000400200015B0F0BD0C68012123000B408D
:1009D000009306D1042C04D922680F331A40092A47
:1009E00001D00B20EAE7626852100392002A03DC70
:1009F000009802F0E3FCE3E73F4A019201280BD0A4
:100A00006868084208D1042806D902681340042BFC
:100A100002D102F0D1FA019001980AF06FFD0600B0
:100A20000F27039B0834013B04935E43039B029012
:100A30009B001B19059301232068184251D10428FB
:100A40004FD903683B40042B52D1FFF799FB059B1C
:100A500004343618A342EED1300002F0AFFC041E7D
:100A6000AFD02B680593029B002B03D0686802F07F
:100A7000A3FA0190200002F09FFA0500009B059A5E
:100A80009B00D3189F68380002F096FA01230600F5
:100A90001F4201D1042F04D807A93800FFF7A2FE96
:100AA00007AE30000AF02AFD0700020031002800DE
:100AB0000AF07EF9029BED19002B0AD0049B009AE4
:100AC000934206DD2800029A01990AF071F9029B0F
:100AD000ED18009B01330093009A039B9342CDD104
:100AE0006FE707A9FFF77EFE07A80AF007FDAEE74C
:100AF00002F062FAF9E7C046D6C7000010B500243C
:100B0000A04207DD0B6801341C4003D05C10E343B6
:100B1000DB171C40611C0122092002F0E3FB0028C6
:100B200003D0012364001C43446010BD0B6870B502
:100B300018000125284032D1042B30D90F241A681F
:100B400049681440092C16D15C6812092C41A24254
:100B500000D8541E844205DC02200132904206DB9C
:100B600000200FE085005D19A9600130F2E78400E4
:100B700019510130F2E7032C11D1294203D113207E
:100B800000F0F2F970BD4910FF29F8D812090433BA
:100B900092009A189A42E3D919700133FAE70B20B0
:100BA00000F0E2F9DCE700000123F7B500264D680C
:100BB0000F002B400093B3420DD11E00042D0AD923
:100BC0000F222B681A40092A0FD16A681B09561098
:100BD000B34200D85E1E3968CB0713D54C10002CE9
:100BE00001DDA64219DA12202EE0042A04D12800E1
:100BF000FFF7C6FA0600EEE7009E032AEBD11E09B6
:100C0000B600E8E72E48FFF777FD002814D00AF079
:100C1000CBFB310008F08AF84C1C009B002B4CD118
:100C2000042D4AD92A680F331340092B10D10134FF
:100C3000A40064592000FEBD39682248FFF75CFD1E
:100C400034000028E9D1113000F08EF90400F1E7FA
:100C5000042B2AD1280002F0AFF90600FFF7BAFAF8
:100C6000A042C0DB012C1ADC280002F0A5F900909C
:100C70003000FFF79BFA851B280002F09FFB041E43
:100C8000D8D002F099F90190786802F095F9009BAC
:100C90002A00F11A411801980AF08AF8CAE73000D0
:100CA000FFF784FA013C0600DCE7032B05D12C1981
:100CB000E478023B64001C43BCE70B20C4E7C04659
:100CC0006CC4000077C40000F7B54C680F00012029
:100CD000210001402AD1042C28D90F222368BE68A4
:100CE0001A40092A13D162681B0955100191AB42C1
:100CF00000D85D1E39682848FFF7FEFC002829D07F
:100D00000F2322681340092B19D1012313E0032A72
:100D10000CD1064203D1132000F026F9FEBD72105B
:100D20000192FF2AF7D81D09AD00E3E70B20F3E796
:100D300001339A00A6509D42FADA0020EEE7032B19
:100D4000FBD1230001331A1BAA42F6DC6A46127952
:100D5000DA70F7E73968CB0706D54910002901DDBD
:100D60008D4209DA1220D7E70C48FFF7C5FC2900AD
:100D7000002801D11130CFE70F2322681340092B3F
:100D800003D1013189000E51D7E7032BD5D16B4632
:100D90001B796418E370D0E773C4000077C40000C7
:100DA00010B501240868204216D1042814D90F2256
:100DB00003681A40092A01D1406810BD032A03D1F3
:100DC0001809C0002043F8E7042A05D102F0F4F81E
:100DD000FFF700FA4000F5E70B2000F0C5F8ECE75C
:100DE00010B5034A0A21034804F0B6F810BDC04606
:100DF0001CC4000014C40000F0B585B0039301903A
:100E000002912C4E2C4B002A02D002223270013A61
:100E100000251A601B68F554019B9D4201DB05B05B
:100E2000F0BD029AAB00D058234B1C68C8239B002E
:100E300037191C1B0123184206D0204A43102100F9
:100E400038000AF0E3FA09E01D4A002802D004281D
:100E50001BD11C4A210038000AF0D8FA30000AF0F1
:100E60004DFB154A039B1060002B0CD0019B013BEE
:100E7000AB4208DD144B984205D8431C1360202276
:100E800032540022F2540135C6E704280FD90F234B
:100E900002681340042B04D102F08EF80B4A0300C1
:100EA000CDE7092B04D14368094A5B10C7E701234A
:100EB000084AC4E7A1020020C405002074CD000048
:100EC0007CC4000082C400001F03000093D3000014
:100ED000ECC60000FBC6000010B50124044002D09F
:100EE0004410200010BD04280CD90F2302681340C1
:100EF000042B07D102F060F821000A220AF0C6FB99
:100F00000400EEE70D22014B1A70EAE7A002002070
:100F10000123020010B51A4015D1042801D9026836
:100F200012090B4011D1042901D90B681B090024B7
:100F3000934206D104309B000431C318984206D373
:100F40000124200010BD0022EBE70023EFE7047826
:100F50000A78002C01D1002AF2D0013001319442EC
:100F6000ECD00024EDE70000014B18700020704722
:100F7000A002002070B501F093FD094C0100251D71
:100F80001F2228000AF0D2FA28000AF0B7FA042338
:100F900004308008000118432060200070BDC04666
:100FA0007C020020C368F0B59D00836889B05D199C
:100FB0000300183306930369069A9F00069B02906C
:100FC000DF19436901939B00D3180393CD4B1B7822
:100FD000002B26D17F222B68CB491C1213409B008B
:100FE0005B58043501929F46029B587804F090FBB1
:100FF0000023029A137027E0C24B1B78002B10D1FC
:101000002B68019A1C121340BF4A9B009B58043561
:10101000E9E7069B3A1DD11ABA4BD82928DD1A22D6
:101020001A70029BB74C9B6821780193EA1A029BC5
:1010300092109B7812021A43029B587804F070FBBE
:101040000023029A23701370029B069A9B680193F7
:10105000ED1A029BAD10DD60069BFE1A029BB610D6
:101060001E61039B9B1A029A9B10536109B0F0BD4D
:101070001B783C60002B01D01700D2E72B68019948
:101080001C120B40A0499B005B5817000435AAE7CF
:10109000069B3A1DD11A9B4BD82902DD1A221A70E1
:1010A000BFE728681B78291D3860002B02D0170085
:1010B0000D00B6E76B6801991C120B4092499B002A
:1010C0005B58170008358EE7069B3A1DD11A8D4BE9
:1010D000D82902DD1A221A70A3E7A4001B782C1964
:1010E0003C60002B01D017009BE72B6801991C1274
:1010F0000B4085499B005B581700043573E7069B3E
:101100003A1DD11A7F4BD82902DD1A221A7088E7BE
:101110007E49A40061581B783960002B01D017006C
:101120007FE72B6801991C120B4077499B005B58A5
:101130001700043557E7043F744B3A68A400E250A7
:10114000704B1B78002B00D06BE72B68019A1C12A8
:1011500013406D4A9B009B58043544E76B4BA40039
:10116000E058FFF7B9FE043F06003868FFF7B4FE09
:1011700036180120654B76000643E650614B1B781C
:10118000002B00D04DE72B68019A1C1213405E4AD9
:101190009B009B58043526E7069B3A1DD11A594BF4
:1011A000D82902DD1A221A703BE70698039C012118
:1011B000A04202D221000C3909681B783960002B4B
:1011C00001D017002DE72B6801991C120B404E49E6
:1011D0009B005B581700043505E7069B3A1DD11AA2
:1011E000484BD82902DD1A221A701AE7069903988B
:1011F00081420FD203000C3B1B6845495B10641809
:10120000E41AA40023583B603E4B1B78002B05D00A
:10121000170006E7182119700023F4E72B680199DD
:101220001C120B4038499B005B5817000435DAE666
:10123000069B039A934219D213000C3B1B68344A55
:10124000043FA4185B10E31A039A39689B00995075
:101250002C4B1B78002B00D0E3E62B68019A1C1264
:101260001340294A9B009B580435BCE61822254BA5
:101270001A70EDE7069B039A93422DD2244B3E1F32
:10128000E31814000C3C04932368049A5B10D31AEF
:10129000039A9B009858FFF71FFE07903068FFF7EE
:1012A0001BFE2468049B64101C1B079BA4001F18D2
:1012B00001207F00039B0743E7503700114B1B7849
:1012C000002B00D0ADE62B68019A1C1213400E4A89
:1012D0009B009B58043586E618220A4B1A70EDE7EE
:1012E000069B3A1DD11A074BD82902DD1A221A7023
:1012F00097E60399A40061581B783960002B09D048
:1013000017008EE6A0020020ECC400007C2D002017
:10131000FDFFFF3F2B6801991C120B40D7499B0032
:101320005B58170004355EE6043F039B3A68A4004F
:10133000E250D34B1B78002B00D072E62B68019A49
:101340001C121340CD4A9B009B5804354BE6039B6F
:10135000A4001C192368043F38685E10FFF7BCFD29
:1013600036180120C64B76001B7806432660002BFA
:1013700000D056E62B68019A1C121340BF4A9B000E
:101380009B5804352FE6069BA4003F1BBC4CBB4278
:101390000CD82378002B00D043E62B68019A1C124E
:1013A0001340B64A9B009B5804351CE6B54801F033
:1013B000F3FD2378002B00D033E62B68019A1C1232
:1013C0001340AE4A9B009B5804350CE6A300ED1871
:1013D000002C00DA38E6AA4B1B78002B00D020E660
:1013E0002B68019A1C121340A44A9B009B58043599
:1013F000F9E5043F3B68042B04D1A300ED18002C51
:1014000000DA21E69E4B1B78002B00D009E62B6802
:10141000019A1C121340994A9B009B580435E2E53F
:10142000043F3B68042B06D0A200AD18002C02DA62
:10143000002B00D108E6924B1B78002B00D0F0E582
:101440002B68019A1C1213408C4A9B009B58043550
:10145000C9E53A1F13685B10013B002B06DD012133
:101460005B00A4000B432D191360EDE5844B1700BE
:101470001B78002B00D0D4E52B68019A1C12134076
:101480007E4A9B009B580435ADE53A00069B0C3222
:10149000D31AD82B03DD1A22794B1A70C1E5FF232A
:1014A00061005B001940FE3BFF3B19433960029924
:1014B00006988968241204916D1A0299AD108978F2
:1014C0002D020D4303999D40091A891099401D432F
:1014D0000B43BB60029B7D609C70E4B26A4BE400EE
:1014E0000392E358029A9360654A1278002A03D067
:1014F00008331D00039F94E51D00019A9B680C357D
:101500001C1213405D4A9B009B58039F6BE53B1FD9
:101510001C68039A069B93422DD10A20E3070CD442
:10152000042C13D90F2322681340042B11D120005F
:1015300001F042FD09F0E2FF0630643003F09CFD4B
:1015400000280FD1043D069B03937DE50720042C62
:10155000F3D02000431E9841FA234042FF33184045
:101560000730EAE7029B2100587804F0EBF80023EB
:10157000029A1370E7E7039B039A0C3B1B680299DE
:101580005B109B00D31A0C3B1C601F1D1300083B13
:101590001B685A108A70D2B23B49D2005B00555882
:1015A0009B0A029A9B009560ED18039B069A043BE8
:1015B0001B685B109B00D3180393314B1B78002BE7
:1015C00000D02EE52B68019A1C1213402B4A9B0079
:1015D0009B58043507E53B1F1868FFF77DFCA40006
:1015E00006003F1B1E2827DC00280DDC244B1B783F
:1015F000002B00D015E52B68019A1C1213401F4ADE
:101600009B009B580435EEE401F038FA033E36188F
:1016100001F034FA1D4B801B9842F9D8184B1B7807
:10162000002B00D0FDE42B68019A1C121340134AD2
:101630009B009B580435D6E40123029A137001F0F5
:101640001DFA029B0A3886195E60FDE43B1F18688C
:10165000FFF742FCA40006003F1B002818DC084BE3
:101660001B78002B00D0DCE42B68019A1C1213407D
:10167000024A9B009B580435B5E4C046ECC4000008
:10168000A00200200DC70000842500203F420F006B
:10169000CA4B984203DD1D22C94B1A70C1E40123D5
:1016A000029A137001F0EAF9FA239B005E43029B51
:1016B0000A3E30185860C7E4A300FF1A0023200038
:1016C0001A003900FFF798FBBE4EBF4C316820006E
:1016D00001F080FEBD4B31681860200003F0E6FE8B
:1016E0003168200004F035F83168200002F06DF810
:1016F000B34B1B78002B00D093E42B68019A1C128B
:101700001340B34A9B009B5804356CE4AC4BA400D7
:101710001B783F1B002B00D083E42B68019A1C121E
:101720001340AB4A9B009B5804355CE4029803F0DD
:1017300007FDA34B1B78002B00D072E42B68019AA5
:101740001C121340A24A9B009B5804354BE43B1FDC
:101750001B68002B3ED13B000C3B1B68DA072CD5E5
:10176000390001225B105800083902430A60002B3F
:1017700044DD012259001143381F01603900083946
:1017800009681141CB1A39000C390968114224D07B
:101790009B189340A4001343039AA350884B1B78D3
:1017A000002B00D03DE42B68019A1C121340884A9C
:1017B0009B009B580435FFF716FC042B06D90F221B
:1017C00019680A40092A01D15B68C9E719227C4BD4
:1017D0001A7026E45B10013BC9E7042909D90F22DE
:1017E00008680240092A04D102339B005B58A40018
:1017F000D2E71922724B1A70FFF713FC0435CDE7BC
:10180000A300069AFB189B1AD82B13DC0122631E37
:10181000002C14DC6A4B1B78002B01D0FFF701FC75
:101820002B68019A1C121340694A9B009B5804358F
:10183000FFF7D9FB1A22624B1A70FFF7F2FB3A60EE
:101840001C000437E3E7069A3B1D9B1A5C4ED82B1D
:1018500003DD1A233370FFF7E4FB069B039AA40011
:1018600093422AD23B1F1868FFF736FB011E21DD89
:10187000039B0C3B1A68521082421BDB9007801AB4
:10188000544B4018C018039B8000C2583B1B1A6081
:101890004B4B3F1B1B780437002B01D0FFF7C1FBDC
:1018A0002B68019A1C121340494A9B009B5804352F
:1018B000FFF799FB20233370EAE71823FBE7434B3C
:1018C000A4001A683B1B1F001A603D4B04371B78AD
:1018D000002B01D0FFF7A5FB2B68019A1C121340C7
:1018E0003B4A9B009B580435FFF77DFBA3009C46B9
:1018F000FE1A002C17DC1C22314B1A7000233360B7
:101900006346FF1A2E4B04371B78002B01D0FFF7DC
:1019100088FB2B68019A1C1213402D4A9B009B5890
:101920000435FFF760FB002033685A108300F1583C
:1019300001230B4003D10D21214A1170DFE749102B
:101940008A4200DD0A0001308442EFDC01235200AC
:101950001343D4E7A3009C46FE1A002C17DC1C227C
:10196000174B1A70002333606346FF1A144B043779
:101970001B78002B01D0FFF754FB2B68019A1C1237
:101980001340134A9B009B580435FFF72CFB0020A3
:1019900033685A108300F15801230B4003D10D2105
:1019A000074A1170DFE749108A4200DA0A00013065
:1019B0008442EFDC012352001343D4E780EE36006B
:1019C000A0020020C4050020A10200200800002081
:1019D000ECC40000FCFFFF3F3B00083B1868FFF72A
:1019E0007BFA3B1F06001868FFF776FA0023864251
:1019F00000DA0433A4003A1B17001360E34B0437EA
:101A00001B78002B01D0FFF70CFB2B68019A1C12EE
:101A10001340DF4A9B009B580435FFF7E4FA3B0074
:101A2000083B1868FFF758FA3B1F06001868FFF7D5
:101A300053FAF30FC217B0425341A4003A1B1700E8
:101A40009B001360D14B04371B78002B01D0FFF7AC
:101A5000E8FA2B68019A1C121340CD4A9B009B5850
:101A60000435FFF7C0FA3B00083B18683B1F1968B4
:101A7000A600BE1B0423814202D0042802D8002302
:101A8000336016E001231842F9D10F2302681A408F
:101A9000042AF4D1033A1142F1D10429EFD90A689A
:101AA0001340042BEBD1FFF733FA431E984180001B
:101AB0003060B64BA4001B783F1B0437002B01D0CD
:101AC000FFF7AFFA2B68019A1C121340B04A9B0033
:101AD0009B580435FFF787FA3B00083B18683B1F0B
:101AE0001968A600BE1B0023814202D0042802D838
:101AF0000423336016E001231842F9D10F23026852
:101B00001A40042AF4D1033A1142F1D10429EFD941
:101B10000A681340042BEBD1FFF7FAF9434258410E
:101B200080003060994BA4001B783F1B0437002BCA
:101B300001D0FFF776FA2B68019A1C121340944AE1
:101B40009B009B580435FFF74EFA3B00083B186892
:101B5000FFF7C2F93B1F06001868FFF7BDF9F3173E
:101B6000C20F86425341A4003A1B17009B0013602A
:101B7000864B04371B78002B01D0FFF752FA2B68F5
:101B8000019A1C121340824A9B009B580435FFF7B0
:101B90002AFA3B00083B1868FFF79EF93B1F060036
:101BA0001868FFF799F90023864200DD0433A4008A
:101BB0003A1B17001360754B04371B78002B01D0BC
:101BC000FFF72FFA2B68019A1C121340704A9B00F2
:101BD0009B580435FFF707FA3B1F1B68A400043B22
:101BE0005A1E93413A1B17009B001360674B043742
:101BF0001B78002B01D0FFF714FA2B68019A1C12F6
:101C00001340634A9B009B580435FFF7ECF93B00F7
:101C1000083B1868FFF760F93B1F06001868FFF7DC
:101C20005BF932180120A4003B1B1F005200024345
:101C30001A60564B04371B78002B01D0FFF7F1F9DF
:101C40002B68019A1C121340514A9B009B58043583
:101C5000FFF7C9F93B00083B1868FFF73DF93B1F48
:101C600006001868FFF738F9321A0120A4003B1B60
:101C70001F00520002431A60444B04371B78002BAC
:101C800001D0FFF7CEF92B68019A1C121340404A8D
:101C90009B009B580435FFF7A6F93B00083B1868EA
:101CA000FFF71AF93B1F06001868FFF715F9020045
:101CB0000120A4003B1B1F007243520002431A6024
:101CC000324B04371B78002B01D0FFF7AAF92B68A1
:101CD000019A1C1213402E4A9B009B580435FFF7B3
:101CE00082F93B1F1868FFF7F7F8061E17D11F226D
:101CF000264B1A70A4003B1B1F001E60234B0437A9
:101D00001B78002B01D0FFF78CF92B68019A1C126D
:101D100013401F4A9B009B580435FFF764F93B00B2
:101D2000083B1868FFF7D8F8310006F019FF0126C4
:101D300040000643DEE73B1F1868FFF7CDF8061E9C
:101D400017D11F22114B1A70A4003B1B1F001E60ED
:101D50000E4B04371B78002B01D0FFF762F92B687C
:101D6000019A1C1213400A4A9B009B580435FFF746
:101D70003AF93B00083B1868FFF7AEF8310006F06F
:101D8000D5FF012649000E43DEE7C046A002002031
:101D9000ECC400003B1F1868FFF79EF8C2178018BC
:101DA00050400122A4003B1B1F004000104318605C
:101DB000F64B04371B78002B01D0FFF732F92B6864
:101DC000019A1C121340F24A9B009B580435FFF7FE
:101DD0000AF9A300FE1A3068012C24D1FFF77CF821
:101DE0000494079009F0E0FA0799002900DC01212A
:101DF00006F09CFF049BA400C91801234900194365
:101E0000E24B3F1B1B7831600437002B01D0FFF7FA
:101E100008F92B68019A1C121340DD4A9B009B585D
:101E20000435FFF7E0F8FFF757F804907068FFF704
:101E300053F8049B0130C31A0793D3E7A300FE1A9B
:101E400031002000049301F047FC049B3060FF1A2E
:101E5000CE4B04371B78002B01D0FFF7E2F82B683C
:101E6000019A1C121340CA4A9B009B580435FFF785
:101E7000BAF83B00083B1868FFF72EF83B1F060036
:101E80001868FFF729F802000120A4003B1B1F007F
:101E90003240520002431A60BC4B04371B78002BBF
:101EA00001D0FFF7BEF82B68019A1C121340B84A04
:101EB0009B009B580435FFF796F83B00083B1868D9
:101EC000FFF70AF806003B1F1868FFF705F8320015
:101ED00002430120A4003B1B1F00520002431A6072
:101EE000AA4B04371B78002B01D0FFF79AF82B6818
:101EF000019A1C121340A64A9B009B580435FFF719
:101F000072F83B00083B1868FEF7E6FF06003B1F2F
:101F10001868FEF7E1FF320042400120A4003B1B9D
:101F20001F00520002431A60984B04371B78002BA5
:101F300001D0FFF776F82B68019A1C121340944ADF
:101F40009B009B580435FFF74EF83B1F1868FEF7BF
:101F5000C3FFC0430122A4003B1B1F0040001043ED
:101F600018608A4B04371B78002B01D0FFF759F813
:101F70002B68019A1C121340854A9B009B5804351C
:101F8000FFF731F83B00083B1868FEF7A5FF060095
:101F90003B1F1868FEF7A0FF32008240510001226B
:101FA000A4003B1B1F000A431A60784B04371B78C0
:101FB000002B01D0FFF735F82B68019A1C12134053
:101FC000734A9B009B580435FFF70DF83B00083B14
:101FD0001868FEF781FF06003B1F1868FEF77CFFBC
:101FE0003200024151000122A4003B1B1F000A43A2
:101FF0001A60664B04371B78002B01D0FFF711F8ED
:102000002B68019A1C121340614A9B009B580435AF
:10201000FEF7E9FF3B000C3B1868FEF75DFF3B0055
:10202000083B06001868FEF757FFF1170200C317B8
:10203000300006F0CDFE3B1F049005911868FEF7B6
:102040004BFF02000498059906F076FE430001203C
:10205000A4003E1B370018434C4B30601B780437FC
:10206000002B01D0FEF7DDFF2B68019A1C121340F4
:10207000474A9B009B580435FEF7B5FFA300FE1AA4
:10208000310020000493FEF739FD049B3060FF1AF5
:102090003E4B04371B78002B01D0FEF7C2FF2B68A4
:1020A000019A1C1213403A4A9B009B580435FEF7D4
:1020B0009AFFA300FF1A39002000FEF737FD334BCB
:1020C0001B78002B01D0FEF7ACFF2B68019A1C1285
:1020D00013402F4A9B009B580435FEF784FFA30052
:1020E000FE1A310020000493FEF75EFD049B306071
:1020F000FF1A264B04371B78002B01D0FEF791FF07
:102100002B68019A1C121340214A9B009B580435EE
:10211000FEF769FFA300FF1A39002000FEF7D4FD87
:102120001A4B1B78002B01D0FEF77BFF2B68019A1E
:102130001C121340164A9B009B580435FEF753FFB0
:10214000A300FE1A310020000493FEF729FE049B31
:102150003060FF1A0D4B04371B78002B01D0FEF7BF
:1021600060FF2B68019A1C121340094A9B009B5880
:102170000435FEF738FF069B3E1DF31A034CD82B9F
:1021800008DD1A232370FEF74CFFC046A002002092
:10219000ECC4000000F07CFC4300012018432378CD
:1021A0003860002B02D03700FEF73BFF2B68019A06
:1021B0001C121340F44A9B009B5837000435FEF76D
:1021C00012FF069B3E1DF31AF04CD82B03DD1A2399
:1021D0002370FEF726FF00F051FCED4B4000184045
:1021E0000123184323783860002B02D03700FEF714
:1021F00018FF2B68019A1C121340E34A9B009B585E
:1022000037000435FEF7EFFE0123A600BE1B2000B9
:102210001A003100FEF7F0FDDE4C2068643002F059
:102220002BFF002802D1043DFEF70EFF029B216820
:102230005A78D94803F09BFA0123029A37001370A9
:1022400000F01CFCD54B22681B680632534318185B
:10225000029B5860FEF7F8FEA600BE1B200001237B
:1022600000223100FEF7C8FDCA4C2068643002F03D
:1022700003FF0028D7D0C84803F070F8DCE7A400BB
:102280003E1BFEF777FE3700C04B30601B780437EB
:10229000002B01D0FEF7C5FE2B68019A1C121340DB
:1022A000B94A9B009B580435FEF79DFEA4003E1BD7
:1022B000300000F01CFC3700B44B30601B78043752
:1022C000002B01D0FEF7ADFE2B68019A1C121340C3
:1022D000AD4A9B009B580435FEF785FEA4003E1BCB
:1022E000300000F006FC3700A84B30601B78043744
:1022F000002B01D0FEF795FE2B68019A1C121340AB
:10230000A14A9B009B580435FEF76DFEA300FE1A00
:1023100031002000049300F0EFFB049B3060FF1AB3
:102320009A4B04371B78002B01D0FEF77AFE2B68FE
:10233000019A1C121340944A9B009B580435FEF7E7
:1023400052FEA4003F1B380000F008FC8F4B1B78A6
:10235000002B01D0FEF765FE2B68019A1C1213407A
:10236000894A9B009B580435FEF73DFEA300FE1AE8
:1023700031002000049300F019FC049B3060FF1A28
:10238000824B04371B78002B01D0FEF74AFE2B68E6
:10239000019A1C1213407C4A9B009B580435FEF79F
:1023A00022FEA4003F1B380000F042FC774B1B7854
:1023B000002B01D0FEF735FE2B68019A1C1213404A
:1023C000714A9B009B580435FEF70DFE0121200049
:1023D00000F016FC6D4B1B78002B01D0FEF721FEA0
:1023E0002B68019A1C121340674A9B009B580435C6
:1023F000FEF7F9FD0021200000F002FC634B1B7882
:10240000002B01D0FEF70DFE2B68019A1C12134021
:102410005D4A9B009B580435FEF7E5FDA4003E1B7A
:10242000300000F027FC3700584B30601B78043731
:10243000002B01D0FEF7F5FD2B68019A1C1213400A
:10244000514A9B009B580435FEF7CDFDA4003E1B6E
:10245000300000F023FC37004C4B30601B78043711
:10246000002B01D0FEF7DDFD2B68019A1C121340F2
:10247000454A9B009B580435FEF7B5FDA4003F1B61
:10248000380000F0E5FB414B1B78002B01D0FEF734
:10249000C8FD2B68019A1C1213403B4A9B009B58B5
:1024A0000435FEF7A0FDA4003F1B380003F040FCFC
:1024B000364B1B78002B01D0FEF7B3FD2B68019A39
:1024C0001C121340304A9B009B580435FEF78BFDCD
:1024D000A4003E1B300003F0D9FC37002B4B3060CA
:1024E0001B780437002B01D0FEF79BFD2B68019A67
:1024F0001C121340244A9B009B580435FEF773FDC1
:10250000A4003F1B380003F0E3FB204B1B78002B9B
:1025100001D0FEF786FD2B68019A1C1213401A4A5F
:102520009B009B580435FEF75EFDA4003E1B300067
:1025300003F0E4FB3700154B30601B780437002BA9
:1025400001D0FEF76EFD2B68019A1C1213400E4A53
:102550009B009B580435FEF746FDA300FF1A390087
:10256000200001F0E1FB094B1B78002B01D0FEF7A6
:1025700058FD2B68019A1C121340034A9B009B587C
:102580000435FEF730FDC046ECC40000A002002078
:10259000FEFFFF7FC4050020A102002004000020F0
:1025A000A300FF1A3900200001F0FAF99F4B1B78B5
:1025B000002B01D0FEF735FD2B68019A1C12134049
:1025C0009B4A9B009B580435FEF70DFDA300FF1AA4
:1025D0003900200001F0E0FA944B1B78002B01D069
:1025E000FEF71FFD2B68019A1C121340904A9B00B6
:1025F0009B580435FEF7F7FCA300FF1A39002000B2
:1026000001F0F2FA894B1B78002B01D0FEF709FD8F
:102610002B68019A1C121340854A9B009B58043575
:10262000FEF7E1FCA300FE1A31002000049303F042
:10263000A8FC049B3060FF1A7C4B04371B78002BEE
:1026400001D0FEF7EEFC2B68019A1C121340784A69
:102650009B009B580435FEF7C6FCA300FE1A310010
:102660002000049303F095FC049B3060FF1A6F4B2D
:1026700004371B78002B01D0FEF7D3FC2B68019A9E
:102680001C1213406A4A9B009B580435FEF7ABFCB2
:10269000A300FE1A31002000049303F082FC049B87
:1026A0003060FF1A614B04371B78002B01D0FEF716
:1026B000B8FC2B68019A1C1213405D4A9B009B5882
:1026C0000435FEF790FCA300FE1A310020000493AD
:1026D00003F06FFC049B3060FF1A544B04371B78E7
:1026E000002B01D0FEF79DFC2B68019A1C121340B1
:1026F0004F4A9B009B580435FEF775FCA300FF1A58
:102700003900200001F084F9484B1B78002B01D0E0
:10271000FEF787FC2B68019A1C121340444A9B0069
:102720009B580435FEF75FFCA300FF1A3900200018
:1027300001F082FA3D4B1B78002B01D0FEF771FCB3
:102740002B68019A1C121340394A9B009B58043590
:10275000FEF749FCA300FE1A31002000049301F0AB
:10276000E9F9049B3060FF1A304B04371B78002BCB
:1027700001D0FEF756FC2B68019A1C1213402C4A1C
:102780009B009B580435FEF72EFCA300FF1A39006E
:10279000200001F09BF9254B1B78002B01D0FEF7A0
:1027A00040FC2B68019A1C121340214A9B009B5845
:1027B0000435FEF718FC069B029AFB1A9B10136166
:1027C000A300FF1A3900200002F0DAFB174B1B7838
:1027D000002B01D0FEF725FC2B68019A1C12134038
:1027E000134A9B009B580435FEF7FDFB069B029A9B
:1027F000FB1A9B101361A300FE1A31002000049302
:1028000002F0BEFB049B3060FF1A084B04371B78B4
:10281000002B01D0FEF705FC2B68019A1C12134017
:10282000034A9B009B580435FEF7DDFBA002002005
:10283000ECC400000023F7B55A1E0192002B07DA02
:1028400001F088FA02F090FE02F0F0FF19230193E4
:1028500000263000194B1968B14212DD184B1A6876
:1028600001328A420FDAF0241A601D68154F6C435A
:10287000E35D002B1FD0E419022B06D12000FEF7E8
:1028800091FB019BD8E70022EDE7012B0DD1002839
:1028900001D100F0F3F8F0226A43BB185B680A49E3
:1028A000C31A8B4201D80223BB54F0235D43054B6E
:1028B000EB5C022BE2D00136CCE7C046C805002015
:1028C00000000020241C00203F420F0001220021B4
:1028D0000A4B0B481A61195004301950A2210420E8
:1028E000C9005850C121C0208900800258501A6088
:1028F000044BFC311960044B1A70704700A0004073
:102900000405000000E100E0EC0500200420704711
:10291000F8B550C9012322001A40101E2DD03340B3
:10292000181E2AD064100020192C26D81D4B7610B2
:1029300035009E4200DD1D001B4F3B5D012B05D085
:102940000121200004F028FC01233B55174B1B7884
:10295000002B01D1FFF7BAFF0023154A9E420DDC80
:10296000FF2514491448D65CB44202D15E0070526F
:10297000D5540133042BF6D10420F8BDD15C8C4230
:1029800003D10C4A5B009D52F6E70133042BF5D1CD
:102990000023D15CFF2901D1D454F2E70133042B89
:1029A000F7D1E9E788130000D0050020EC050020EE
:1029B0001C0000200E000020DC050000F8B530C926
:1029C000012623003340181E1BD02B003340181E55
:1029D00017D034410020192C13D8174F3B5DB34258
:1029E00004D03100200004F0D7FB3E5569100800E8
:1029F000124A1038124B904204D9012252421A60F6
:102A00000420F8BD1C600F4806F0AAF80E4B188091
:102A10000E4B1B78002B02D1FFF758FFF0E7012285
:102A20000B4B9A64A922D2009A588018A82280B22F
:102A3000D2009850E4E7C046D005002090860100FF
:102A40001800002020A107000C000020EC05002049
:102A500000A000400420704701220020054B0649D9
:102A60001A615850043103305850083180185850BA
:102A70001A60704700800040040500000122034BEB
:102A80001A64A822D20098587047C04600800040BF
:102A900010B5FFF7F3FFFA21890005F0D7FF10BD4D
:102AA0000048704760C700001A20704770B5054E97
:102AB0000400335C0D008B4202D004F06DFB3555F1
:102AC00070BDC046D005002070B50024064D635D82
:102AD000012B05D10021200004F05EFB002363558B
:102AE00001341A2CF2D170BDD005002070470D20A2
:102AF0007047352070470000F8B501240B680600C8
:102B00000D00234204D10D20FEF72EFA2000F8BD5F
:102B10005B102000052BFAD80E4A9B009C580E4FE4
:102B20003B5D002B05D00021200004F035FB002385
:102B30003B55012E06DD6B68042B03D102212000DA
:102B400004F02AFB200004F0D5F9012440002043C2
:102B5000DDE7C04648C70000D0050020F8B50126D3
:102B60000568354202D04468344203D10D20FEF797
:102B7000FBF9F8BD6D10192DFBD80A4F7B5D012BB9
:102B800004D03100280004F007FB7E55064964108C
:102B90008C4202DCE143C9172140280004F030FADE
:102BA000E7E7C046D0050020FF03000070B5012410
:102BB0000D68254204D10D20FEF7D6F9200070BD26
:102BC0006D10192D17D80024012804DD4C68043C31
:102BD00063425C416400094E735DA34204D021004E
:102BE000280004F0D9FA7455280004F009FB03000A
:102BF0000420012BE3D00020E1E7C046D0050020EF
:102C000070B504000D0019280ED8084E335C012B56
:102C100004D0012104F0C0FA01233355290020001B
:102C20004D1EA94104F0D6FA70BDC046D005002063
:102C3000036810B5DA0703D40D20FEF795F910BD2F
:102C40004168581004394A425141FFF7D9FFF6E76D
:102C500037B569460A00064B30CB30C20368022004
:102C6000042B02D100F098FF37BD00F0BDFFFBE759
:102C700020C7000010B5084C237D002B05D0002193
:102C8000142004F089FA00232375142004F0B8FA04
:102C900043425841800010BDD005002010B5084CBB
:102CA000A37D002B05D00021162004F075FA002327
:102CB000A375162004F0A4FA43425841800010BDC9
:102CC000D0050020F7B5304D304E6B6C002B15D081
:102CD000A8240023E40037596B642D4B18680028A2
:102CE0000CDB2C4B19784A425141C9B2197004F0DF
:102CF00071FA294B1B88DF19BFB23751AB6C002B1F
:102D000039D00021254B264FF458A9643A780C3469
:102D10000193244D8A4206D02B68032B03D8224A04
:102D2000D05C04F057FA2B68204A0133134004D5D5
:102D30000422013B5242134301331B4900228C46BB
:102D40002B60042B18D06046C05C591CFF2802D1B0
:102D50000B000122F5E7002A00D02B60012104F0CE
:102D600039FA01233B702B68114A5B009B5AE41827
:102D7000019BA4B2F450F7BD01235B422B600023FA
:102D80003B700C4BF3E7C046FCA0004000A00040A5
:102D900018000020EB0500200C0000204405000076
:102DA000EA050020CC0500201C0000200300008064
:102DB0000E00002050460000084B094AFF201A80F0
:102DC0005A809A80DA800023064A07491370074A1E
:102DD000087048708870C870136070470E0000203B
:102DE000DC050000EA0500201C000020CC050020C6
:102DF0000122024B52421A607047C0461800002060
:102E000010B5034A0421034802F0A6F810BDC046DD
:102E100028C70000B4CE0000E12170B54902144873
:102E200003F060FEFFF718FE0A2004F05DF80023AF
:102E3000FF21104A995401331A2BFBD101220020A3
:102E40000D4B01001A6004230C4A0D4D1468002C30
:102E5000FCD02C680002013B20431160002BF5D10F
:102E60000122084B1A6003F0F9FF01F0BFF870BDB2
:102E7000AC1B0020D005002000D0004000D1004055
:102E800008D5004004D00040F8B50B4E07003000D4
:102E90000D0003F06FFE0400A84200DD2C003D0091
:102EA000EB1B9C4205DD300003F06EFE28700135FF
:102EB000F6E72000F8BDC046AC1B002010B50100AD
:102EC000014803F017FE10BDAC1B002010B5054CE7
:102ED000200003F01DFEE1212000490203F002FE64
:102EE00010BDC046AC1B0020C3070CD4064B1B68AA
:102EF000834208D8054B1B68984204D8031F1B68FF
:102F0000002B00D018007047F8050020F4050020C1
:102F10000023012210B50A48990001334250642B66
:102F2000FAD1084C084B00211A602000074A07F02C
:102F30005BFF074B074A6360074B1A6010BDC04632
:102F40007C2D0020FC05002008000020D409000092
:102F50003027000000060020F005002010B5044BCB
:102F6000044A1A60044B054A1A60FFF7D1FF10BDEE
:102F7000F8050020FC050020F4050020D00F0020FB
:102F8000044B1B68186800090238C343DB1718405C
:102F90007047C046F005002000B59BB0020005490F
:102FA00001A808F065FA01A802F0F4F902F03EFC6D
:102FB000FCE7C046C6C700000A4BC20704D4042879
:102FC00004D8094B00D0094B180070470F22036842
:102FD0001A40031D042AF7D0054B092AF4D0054BEB
:102FE000F2E7C046ACC7000082C400007CC4000009
:102FF000BFC70000B6C700000020064A0649131FDD
:10300000186013681B0902339B00D2188A42F6D35A
:103010007047C04600060020D00F0020F7B50F24EF
:103020000126304B304A1968304B314D186813680F
:103030001F002740072F25D813681B0902339B0068
:10304000D218AA42F3D300242A4EA500AD1928684D
:10305000FFF74AFF01342860642CF6D1264C206823
:10306000FFF742FF2060254C2068002802D0FFF7C0
:103070003BFF20600025224B1B680093009B9D4274
:1030800013DBF7BD1B099B00D3189A42D4D01F68ED
:10309000374208D1B94206D2B84204D3043F3F6850
:1030A000002F00D01F60043BEFE7F0236B43154A6D
:1030B0009B181A78002A01D10135DFE71F693C23EC
:1030C00000266B43DB199B0001930136BB1BF3D435
:1030D000019BB4001C1B0B4B1C19A069FFF704FFDC
:1030E000A061F2E7F805002000060020F4050020AA
:1030F000D00F00207C2D002008000020D00F0020E1
:10310000C8050020241C0020F7B50124204244D12A
:10311000224B1B689C4698423FD3214B1B6801936E
:1031200098423AD8031F1B68002B36D1020003686F
:1031300000941B09002B0FD10099131F19609042B6
:103140002BD015682B1F1B68990069180C68013B70
:1031500014600A602A00EDE79D0055192968009C5B
:10316000214218D18C4516D8019C8C4213D30E1FD6
:103170003468002C0FD10F680F343C40072C07D95E
:103180002F60151F2B600B680A601B090A00D1E72E
:1031900000993160CEE7013BCCE7F7BDF805002090
:1031A000F40500200D49F0B50B000F260C4D1868F2
:1031B0001C1F276802090232002F0BD000208B420F
:1031C00000D0080020609000091892009B18AB42C4
:1031D000EDD3F0BDB0431860F7E7C046000600200D
:1031E000D00F0020F8B5114C26000F2233681F09BC
:1031F00013420DD07D1CAD00A64204D02A00310040
:10320000200007F0DEFD00226319043564191A60FE
:103210000237BF00064BF6199E42E6D31B1B9B10DC
:10322000013B1B012360034B1C60F8BD000600201E
:10323000D00F0020F0050020F0B59BB0FFF71EFC7A
:1032400000240700204AA300D0580134FFF75CFF98
:10325000642CF7D11D4B1868FFF756FF1C4B1868FC
:10326000002801D0FFF750FF00261A4B1B689E4232
:1032700016DBFFF797FFFFF7D1FEFFF7B3FFFFF76E
:10328000FDFB154BC21B1B6814491B6801A81B09D9
:10329000023B08F0EDF801A802F07CF81BB0F0BD8D
:1032A000F02575430E4BED182B78002B01D101361C
:1032B000DBE72B695C1E002CF9DBA300EB18986997
:1032C000FFF722FF013CF6E77C2D002008000020DC
:1032D000D00F0020C8050020F00500208CC700009A
:1032E000241C0020F7B5164D4F1C2B6806001B68E8
:1032F0000C0001921B099F420ADBFFF79DFF2B6820
:103300001B681B099F4203DB0A20FDF72DFEFEBD53
:103310002868A71CBA00DB1B81181B010B60296001
:103320000021031F19600F231E40030024012643C0
:1033300040C3083A9A189A42E9D9019902C3FAE7B8
:10334000F0050020F7B503000122134004000D0032
:103350000193002B2AD1164B1B68834226D8154BAC
:103360001B68834222D90F23134F3860006818402E
:10337000FFF7B8FF019B3C68061E3B6016D0236830
:1033800004301B099D4200DD1D00AA00211D251FE0
:1033900007F00EFDFFF730FE2E60FFF73FFE002323
:1033A0002B6022680F339A43226034002000FEBD58
:1033B000F8050020F4050020D00F0020032304307E
:1033C00010B5C11719400918891000220420FFF711
:1033D00089FF10BD70B5050008000C00FFF7EEFF77
:1033E0000023002804D170BDE95CC21811710133BB
:1033F000A342F9DBE343DB171C40002304192371CC
:10340000F1E7F0B50C009BB0022804DC1C20FDF7AE
:10341000ABFD1BB0F0BD01230868184206D104289B
:1034200004D90F2601683140042901D00E20EEE7AF
:1034300061680D001D40F9D10429F7D90A683240AE
:10344000042AF3D1A2681A4201D10D20DFE7FFF769
:10345000B3FD06006068FFF7AFFDA768010001AC8F
:103460007F103000257002F05AFF390064232200DB
:1034700002F0BAFF200008F041F801002000FFF739
:10348000A9FFC6E710B51C4CA544041E02D1FFF7E6
:1034900095FF0BE002F05CFE0138062828D805F005
:1034A000C1FA090911182904240000208023DB0037
:1034B0009D4410BD200002F0C7FE011B2000FFF755
:1034C00089FFF3E7200002F06DFE4300012018435E
:1034D000ECE780226946D200200002F07AFE6846BE
:1034E00008F00CF801006846E9E704210348E6E724
:1034F0000020CCE70420D9E700FCFFFF0CC8000047
:1035000070B50C00022803DC1C20FDF72DFD70BDFA
:1035100001230868184206D1042804D90F25016840
:103520002940042901D00E20EFE761681942FAD141
:103530000429F8D90A682A40042AF4D1A2681A4258
:1035400001D10D20E1E7FFF737FD05006068FFF7C7
:1035500033FDA46801006410280002F0E0FE2100A1
:1035600002F01DFFFFF78EFFD1E770B50D000128B7
:1035700003DC1C20FDF7F8FC70BD01240868204224
:1035800006D1042804D90F2102680A40042A01D078
:103590000E20EFE76A682242FAD1042AF8D91368AC
:1035A0000B40042BF4D1FFF707FD06006868FFF716
:1035B00003FD0100300002F0B2FE02F034FF4000D3
:1035C0002043D9E7F8B507000C001C20012F0BDDC4
:1035D00001250868284206D1042804D90F21026871
:1035E0000A40042A03D00E20FDF7BEFCF8BD626835
:1035F0002A42F8D1042AF6D913680B40042BF2D1E1
:10360000FFF7DAFC06006068FFF7D6FC0100022F26
:1036100014D0A4682C4211D06410300002F07FFE58
:10362000050002F095FD012811D1002C02DD0135C5
:10363000012C06D12800FFF725FFD7E701246442BB
:10364000EBE7280002F00CFE013C0500F0E7022841
:10365000F0D1002CEEDD0135012CEBD0002228004A
:10366000110002F02FFE02F0FBFD013C0500F3E724
:1036700010B501240868044016D04410200005F05D
:1036800003FD134905F0CEFB07F0B4FA03F0FCFE8E
:103690000022104B06F068FC03F09EFE07F03AFA99
:1036A00043000120184310BD04280CD90F230268E1
:1036B0001340042B07D1FFF77FFC21000A2207F0FB
:1036C000E5FF0400DAE70D20FDF74EFCD6E7C04623
:1036D000D30237390000D040086870B501240500D6
:1036E000254006D1042804D90F2302681340042B77
:1036F00003D00E20FDF738FC70BDFFF75DFC0378AA
:103700002900233B5A4253411022C01807F0BEFF44
:1037100080239B05C218044B9A4201D91420E9E783
:1037200040002043E8E7C046FFFFFF3F10B5034AD3
:103730000621034801F010FC10BDC046DCC70000A4
:10374000D7C700000020704710B51E20FDF70CFC05
:1037500010BD10B51E20FDF707FC10BD10B51E20D2
:10376000FDF702FC10BD10B51E20FDF7FDFB10BDDE
:1037700010B51E20FDF7F8FB10BD10B51E20FDF79B
:10378000F3FB10BD10B51E20FDF7EEFB10BD10B50C
:103790001E20FDF7E9FB10BD10B51E20FDF7E4FB70
:1037A00010BD10B51E20FDF7DFFB10BD10B51E20AB
:1037B000FDF7DAFB10BD10B51E20FDF7D5FB10BDDF
:1037C00010B51E20FDF7D0FB10BD704710B5034AA1
:1037D0000E21034801F0C0FB10BDC04648C80000E0
:1037E000B8C800000120034B1860034B1B688340DE
:1037F00018437047F40F0020D40F0020F0B5EFF30A
:1038000010810123194083F31088134C134AA446F6
:103810001268134E013A9340124F134A002B17D0EF
:10382000146803420FD03D682C60C046C046C046B5
:10383000C046C046C046C046C0460C4C1568246809
:1038400025605B08EAE765462C6014683460F8E799
:1038500081F31088F0BDC04608050050200000200C
:103860000C050050E00F0020E80F0020DC0F0020C6
:1038700030B585B001AD0C220649280007F098FA52
:103880000024285D01210134FFF710F90C2CF8D138
:1038900005B030BD77C90000F7B56A46394B01ADB8
:1038A00013800F239370384B2B800A23AB70FFF7E4
:1038B000E5F8364B364CC0182368984201D20023F5
:1038C00023602668002E3DD16B469F5D01213800A4
:1038D000FFF7ECF801360021380003F07BFC032EE3
:1038E000F2D10026AF5D01213800FFF7DFF8013685
:1038F0000121380003F06EFC032EF3D1C8200138FB
:10390000C046C046C046C046C046C046C046C04687
:10391000C046C046C046C046F1D100212878FFF716
:10392000C5F868780021FFF7C1F8A8780021FFF7F3
:10393000BDF8FFF7A3F8FA2300251B01C01820608B
:103940002800FEBDFFF79AF8236800259842F7D3B8
:10395000032003F0CFFA0600042003F0CBFA361858
:103960000A2003F0C7FA0B4B9B1B181A0A4BA842FC
:1039700006DB18600023094A236013600125DFE796
:103980001D60F7E70D0E0000030400001027000083
:10399000EC0F0020E3030000D40F0020F40F002000
:1039A0000022054B10B51A60044B1B68934201D0EE
:1039B00002F06EFB002010BDF00F0020D01A002096
:1039C00010B5041E10DA1A240A4BA400E258012391
:1039D0009340094A09491360094A1160094A0A4992
:1039E00011600A4A136010BDFFF75EF8A042EADDDD
:1039F000EAE7C04624D60000E80F00200805005082
:103A0000E00F0020DC0F00200C05005018050050CE
:103A10002B4BF7B51B680C00002B03D10120404253
:103A2000FFF7CEFF24680126250035401AD0FF227B
:103A30006310120260121040DAB21043FF221B0220
:103A40001204134018431F4B1B68202B06D1B440AF
:103A50001D4BA40EA400E35800021843FFF7CEFE4E
:103A60000020FEBD042CFBD90F2322681340092B34
:103A7000F6D1FF2763683F025B100193019B9D42D3
:103A8000EEDAAB00E3189B68334216D05A10581296
:103A9000D1B238400843FF21120209040A40104302
:103AA000084A1268202A06D15B009B0E06499B003B
:103AB000020258581043FFF7A1FE0135DEE7C04669
:103AC000E80F00202000002060CB00000200086802
:103AD00010B5C3070FD540101823012A03DD4A682B
:103AE000042A00D10833054A1360FEF7FFFFFFF7F1
:103AF00067FF002010BD01204042EDE720000020BC
:103B000010B50124044002D04410200010BD042848
:103B10000CD90F2302681340042B07D1FFF74CFA8E
:103B200021000A2207F0B2FD0400EEE70D20FDF7A8
:103B30001BFAEAE70868F8B5C3071AD5FFF7E0FFF4
:103B40000300203B5E2B23D805200122584300238D
:103B5000104E451DA84217D005211024375C3C4269
:103B600000D09B180139520064100029F7D10130B0
:103B7000F0E704280CD90F2203681A40042A07D161
:103B80001B0905D00079DBE701205B001843F8BD75
:103B90000120FCE783C9000070B508680D00FFF73D
:103BA000AFFF04006868FFF7ABFF621E0100042A44
:103BB00014D8451E042D11D805236B439B180122F0
:103BC00015009D402B00064805682B430360054BFC
:103BD0001B68002B02D0200002F05BFA002070BDB1
:103BE000F00F0020D01A002070B508680D00FFF714
:103BF00087FF04006868FFF783FF621E0100042A44
:103C000013D8451E042D10D805236B439B180122A1
:103C10009A400748036893430360064B1B68002BD8
:103C200003D00022200002F034FA002070BDC0460C
:103C3000F00F0020D01A0020F0B5050089B0086808
:103C40000C00FFF75DFF0690022D36DD6068FFF780
:103C500057FF0190A068FFF753FF04000127231DC1
:103C6000661E0793731C0293079B9E4235D0052363
:103C700073430593019B019D05330493049BAB4261
:103C80001ED0042E16D86B1E042B13D80122059BC0
:103C90002349013B5B199A409446224A0B681068FD
:103CA000069A3A4003920DD062461A430A600122F6
:103CB00000280DD17F000135E0E701240194CDE714
:103CC000029ECFE7624693430B600028F2D0039A2E
:103CD0000299280002F0DDF9ECE7019B1E1D042E7D
:103CE0001AD8012C18D1002505273B0021006B4371
:103CF0009B1999400B000A4A013511689943094BF9
:103D000011601B68002B05D0019B0022581D290063
:103D100002F0BFF9052DE8D1002009B0F0BDC04682
:103D2000F00F0020D01A0020086810B5C30703D593
:103D3000FFF7E6FE054B1860054B1B68002B03D010
:103D4000024B186802F0A6F9002010BDF00F002009
:103D5000D01A00207FB5A04C2368002B0AD19F4ABF
:103D60001268002A06D19E4B1B68002B01D0FFF77A
:103D700093FD7FBD9B4D2A68002A26D1984A126880
:103D8000002A1BD0FFF788FD0028F2D0FFF770FD56
:103D9000924B24681A681C60002A16D0002C14D19B
:103DA00001AD0C229049280007F002F8285D00219F
:103DB0000134FEF77BFE0C2CF8D1DAE7874A126853
:103DC000002AE5D1002BE3D0E0E700210D2003F02D
:103DD00001FA00210E2003F0FDF900210F2003F06D
:103DE000F9F92E68012E5DD0022E00D1A2E0002E3E
:103DF00051D101363100794C04202368994303F0F6
:103E0000E9F904212368052019404B42594103F088
:103E1000E1F910212368062019404B42594103F073
:103E2000D9F980212368090119404B4259410C20DE
:103E300003F0D0F980212368090219404B4259410F
:103E40000B2003F0C7F980212368490219404B4237
:103E500059410A2003F0BEF98021236889021940E4
:103E60004B425941092003F0B5F980212368C9026A
:103E700019404B425941082003F0ACF980232168D6
:103E80001B0319404B425941072003F0A3F93100AD
:103E90000D2003F09FF92B680321581C04F046FF06
:103EA000296066E702214D4C0720236819404B42E8
:103EB000594103F08FF90820216801404B425941D4
:103EC00003F088F980212368C90019404B42594109
:103ED000052003F07FF980212368490119404B42F6
:103EE0005941062003F076F980212368C901194061
:103EF0004B425941042003F06DF980212368890366
:103F000019404B4259410A2003F064F9802321688B
:103F10001B0419404B425941092003F05BF9310061
:103F20000C2003F057F931000B2003F053F9310056
:103F30000E20AEE72021294C0720236819404B4270
:103F4000594103F047F940212368082019404B42AA
:103F5000594103F03FF980212368092019404B4261
:103F6000594103F037F980212368490019404B4239
:103F700059410A2003F02EF9802123688900194055
:103F80004B4259410B2003F025F980212368890118
:103F900019404B4259410C2003F01CF98021236841
:103FA000490319404B425941062003F013F980217F
:103FB0002368C90319404B425941042003F00AF910
:103FC000802321685B0419404B425941052003F0CE
:103FD00001F901210F205CE7F00F0020E40F002021
:103FE000F40F0020D80F002077C90000012010B581
:103FF0004042FFF7E5FC0020FFF700FC10BD000089
:1040000010B5034A0921034800F0A6FF10BDC046C1
:1040100060CC0000A8CC000030B502248025094BFC
:10402000094AED009C505C59002CFCD0A124E4000E
:10403000884202D30021995030BD8025ED001851EF
:104040004019F5E700E001400405000010B5002824
:1040500006D1C020B02140028902FFF7DDFF10BD6C
:10406000B02080218002C902F7E700004342584196
:10407000064B40421840B0239B02C0180368002042
:104080001A0E532A01D11B02180A704700C0FEFF06
:1040900030B501248025054B054AED009C505C5944
:1040A000002CFCD001600021995030BD00E001409F
:1040B0000405000043425841074B40421840B023DA
:1040C0009B02C018A62310B50902DB05090A194393
:1040D000FFF7DEFF10BDC04600C0FEFF70B5012433
:1040E00080250D4B0D4EED009C515C59002CFCD0F1
:1040F000002902DC00229A5170BD557814782D02F7
:1041000025439478013924042543D47804322406C5
:104110002C4310C0ECE7C04600E00140040500005D
:1041200070B505004B680A009C1C2100A400FFF735
:10413000D5FF281970BD0000134B1B68002B0CD055
:104140008022B023D2029B0200280BD11A1D5B688B
:104150001B0E522B00D110007047B022C0239202D8
:104160005B02F1E782420DD903681B0E522B09D185
:10417000436802339B00C018824203D903681B0EB8
:10418000522BE9D00020E7E7F810002070B500209E
:10419000FFF7D2FFFF260500002801D1280070BDDF
:1041A00003681C143440FFF7C7FFDA2CF4D1050074
:1041B000F2E700008022F0B55200A1B0002167486C
:1041C00006F012FE802200215200654806F00CFE27
:1041D000644BFF271B681A00049353425A41100096
:1041E0000592FFF733FF049C0020631E9C415E4B49
:1041F00064421C405D4BE418FFF7C8FF0600002E28
:104200002DD10498FFF732FF411C0598FFF752FFAC
:10421000059A574D534B2C601A60FEF757FE514BD1
:1042200064201B68A0215A4253414F4A5B4213400D
:10423000B0222C6892029B18E41A6043490204F0F1
:104240008FFCA0225202030000924A49220007A8D4
:1042500007F00EF907A801F09DF821B0F0BD326813
:10426000131412123A403B4003921A000A3A092AE8
:1042700049D83A4B039A995C002931D110223E4823
:1042800006F0B2FD35002B6803991A123A409142AC
:1042900009D11A143A400B2A27D0132A2DD00A2A02
:1042A00001D1354B1D602800FFF746FF051EEAD1FE
:1042B000314B196800290FD02000FFF731FF0400AF
:1042C0002D4B5B195968002903D02000FFF728FF08
:1042D000040004350C2DF3D1204B0121039A99548D
:1042E0003000FFF729FF060089E73B40022BDADCAC
:1042F000214A9B00D3185D60D5E7102200211E489B
:1043000006F072FDCFE71A00153A082AE8D8144AD9
:104310000399525C002AE3D13500152B00D015001B
:10432000300003681A143A40152A0FD01D2A00D114
:104330000025FFF701FF0028F3D1002D04D0200055
:104340002900FFF7EDFE0400054BC6E7039A1B1298
:104350003B409A42EDD10500EBE7C046F80F002044
:1043600000110020F810002000C0FEFF04C0020071
:10437000FC10002041CD00000C2F0020F0B50020E3
:10438000B7B00024FFF7D8FE270005002600002D57
:104390002ED1284D2868FFF769FE32003B000190BE
:1043A0000094254904A807F063F804A800F0F2FF80
:1043B000224B64201C682B68A0215A425341204A9A
:1043C0005B421340B02292029B18E41A60434902F8
:1043D00004F0C6FBA02252020300009219492200F9
:1043E00004A807F045F804A800F0D4FF37B0F0BDEA
:1043F000FF226B6829689C460233FF180B120136B6
:1044000013409C4200DA1C00FF200A140240039271
:104410006246014001920091039A0B4904A807F0FB
:1044200027F804A800F0B6FF2800FFF785FE050076
:10443000ADE7C046F8100020B2CD0000FC1000200F
:1044400000C0FEFF5CCD00009ECD000070B50020D6
:10445000FFF70CFE04000120FFF708FE844200DA9B
:1044600004000A4B1D686A42554128001D60FFF791
:10447000EDFDA0226B4252021340054A28009B1812
:10448000044A611C1360FFF715FE70BDF810002090
:1044900004800100FC100020F8B50020FFF7E6FDC5
:1044A00007000120FFF7E2FD3E00204D0643204CAF
:1044B0000DD18021C020C9024002FFF7ADFD0121CE
:1044C0003000FFF7F7FD1B4B2E6023601DE0874295
:1044D00009DD0023B0212B60164B8902236023687D
:1044E0000020012517E0012380212B60124BC90217
:1044F0002360F4E7120E522A08D0002800D023606F
:104500000E4800F047FFFFF7A1FFF8BD28005A68EA
:10451000023292009B188B4205D21A68561CE9D1D0
:104520000028F2D0D1E72160EFE7C046F810002064
:10453000FC1000200480010004C0020077CD0000C0
:10454000F0B585B0039203220333DC17294D1440E4
:10455000E4182B68284F5A42534180225B42D20212
:10456000A4103B409B18A21C0291244E9100009184
:104570000190316800980A18934215D2FFF71AFE8D
:104580002B685A42534180225B421F40D202BF181F
:104590003368009A9B189F4206D2194800F0FAFE31
:1045A0000025280005B0F0BD029B356819066B4652
:1045B0001A7BA423DB051343FF222F00090C1943A8
:1045C000019B12041B04134019432800FFF760FDF0
:1045D0000837281D21003760FFF75AFD002C04D052
:1045E0000A9A21003800FFF779FD009B083BFF186D
:1045F0003760D6E7F810002000C0FEFFFC10002056
:104600001BCD000010B5FFF7D5FD10BD70B59AB0F9
:10461000FFF742FFFF221E4CD2000021200006F0CF
:10462000E3FBFF25FFF7B2FD0026002814D10200AE
:10463000C300E3580130591E8B41D218FF28F7D12F
:10464000144901A806F014FF01A800F0A3FE1248C7
:1046500000F0A0FE1AB070BD03681A142A400A2A9E
:104660000AD11A122A40FF2A03D0D200A1180B71D6
:10467000A050FFF761FDD8E7132AFAD11B122B4097
:10468000FF2BF6D0DB00E2181671E650F1E7C046CA
:1046900084250020E7CD0000FBCD00000021094B60
:1046A000094A59600131516059680029FCD0002144
:1046B0001961012393600222044B8131FF315A506A
:1046C0001A607047FC1000400010004000E100E05C
:1046D0000222064B0121DA670022054B5A61054A86
:1046E00011615A69002AFCD07047C04604E100E01D
:1046F000FC1000400010004010B5044C2378002B43
:1047000001D0FFF7E5FF0020207010BD011200204E
:10471000802301205B055B6E5B001843704700003F
:104720000120024B1B685B00184370478412002075
:104730000120024B1B685B001843704724000020D7
:104740000120024B1B685B00184370478812002051
:1047500070B504000D001600FEF79AF980230121C0
:104760005B055A6E2670002653006170E17062721C
:10477000010A5A0A6071A171A272010C5A0C000E52
:104780005B0EA6702571E1712072E272237370BD19
:1047900010B5044C200006F0B1FE01002000FEF729
:1047A00019FE10BD8D1200200E4B10B51B680E4C6B
:1047B0005A1C0FD00D4C002B0CD00D4C012B09D0E6
:1047C0000C4C022B06D0094C042B03D00A4C052BB1
:1047D00000D1074C200006F091FE01002000FEF7FA
:1047E000F9FD10BD2800002093CE00008CCE000003
:1047F0009ECE0000A3CE000098CE000070B5214CE4
:104800002278002A3DD1204B01215A608022D20516
:1048100011605A68002AFCD0002207201B4B1C495B
:1048200001255A500439585008315A5019481A492C
:1048300058501A491A485A501A495A50A622D200BA
:104840009D50082218495A500431585002201749E7
:1048500058501749174858501748043958501820CD
:1048600016495850C12189005A500539FF39585806
:10487000921802435A501249124A9950FFF70EFFFC
:10488000257070BD01120020FC00004000100040A7
:104890000C050000746962751C0500002405000009
:1048A000200004022C05000014050000340500005F
:1048B0003C050000FFFF000021100100540500002E
:1048C000021200200405000070B50E4B06001B7894
:1048D000002B01D1FFF792FF00200B4D2C78844272
:1048E0000ED00A4B202219780323091B1940084BCC
:1048F0004901C918300006F05BFA0120013C2C7018
:1049000070BDC046011200208C1200200012002051
:1049100002120020002370B588B0984235DD0D6882
:1049200001262C0034409C422FD12300042D2CD989
:104930000F222B681A402300092A26D16A683F2AD1
:1049400023DD6846FFF7C0FF230000281DD06B461B
:1049500019783300A14203DB6B461B5D5B003343D8
:10496000A200AA1801349360202CF2D109216944D5
:104970004A780B7812021A438B781B041A43CB78BF
:104980001B061343024A13600423180008B070BDCD
:104990008812002070B5454B8AB01B78002B01D1DE
:1049A000FFF72CFF02AC2000FFF78EFF002802D19A
:1049B00000200AB070BD23780B2BF9D96378012B46
:1049C000F6D1E378012BF3D100231120384E394D75
:1049D00033602B7068442379374A4178136002783A
:1049E00009021143827812041143C27812060A4365
:1049F00032490A60002B0ED1152169444A780B78A0
:104A000012021A438B781B041A43CB781B061343FC
:104A10003360002318E0012B1AD1152169444A782C
:104A20000B7812021A438B781B041A43CB781A2195
:104A30001B06134333600E23627C6944934200DDFE
:104A4000130000229A422CD100220420EA54B0E73D
:104A5000022B03D1627B10331621EEE7042B0DD11C
:104A6000152108226944684606F0A2F900980199C8
:104A700002F022FC06F04EF83060CAE7052BC8D1E0
:104A8000152108226944684606F092F900980199B8
:104A900002F012FC06F03EF83060627D0A231E210F
:104AA000CBE7885CA8540132CCE7C0460112002055
:104AB000841200208D12002028000020881200207F
:104AC00010B5134B04001B78002B01D1FFF796FEA5
:104AD000FFF7FEFD00200F4A0F49104B545058605D
:104AE0000130106058680028FCD0002018610130A7
:104AF000906018690028FCD0094B0A481B785B01BC
:104B00001B185350FFF7E4FDFFF7C8FD10BDC0466A
:104B1000011200200010004004050000FC100040BD
:104B2000001200200212002010B588B000281DDD00
:104B30000A68012113000B4018D1042A16D90F204E
:104B400014682040092811D150683F280EDD9800D4
:104B5000101880680024084201D04010C4B2684692
:104B6000C4540133202BF2D1FFF7AAFF002008B074
:104B700010BD000010B5002813DD0C68E30710D548
:104B80006410532C0DD8084B1B78002B01D1FFF774
:104B900035FEFFF79DFDA123044ADB00D450FFF74B
:104BA0007DFD002010BDC046011200200010004015
:104BB00010B500280EDD0C68E3070BD56410FF2C40
:104BC00008D8054B1B78002B01D1FFF717FE034ACD
:104BD000034BD450002010BD0112002000100040F3
:104BE0002405000013B5002814DD0C68E30711D577
:104BF000094B64100093094B0193072C0AD8084B0A
:104C00001B78002B01D1FFF7F9FD6B46054A1957B8
:104C1000054BD150002016BDE2ECF0F4F8FC000486
:104C200001120020001000400C05000070B588B093
:104C3000002820DD0124086804401CD104281AD96A
:104C40000F2302681340042B15D1FEF7B5F90600B7
:104C500006F054FC0500122800D912252A00022172
:104C60000D326846FFF774FD6B465D73A54205DCA7
:104C70006846FFF725FF002008B070BD2300325DB5
:104C80006B449A730134F1E7F0B50D008BB0012845
:104C900032DD08680122040014402DD104282BD9EC
:104CA0000F2301680B40042B26D16B68134223D0DD
:104CB000FEF782F96E6807007310019306F01EFC80
:104CC00005000E2800D90E252A000121113202A864
:104CD000FFF73EFD6A46127902AB5A7302AA7312BD
:104CE0009373019B76141B0ED67313745574A542EF
:104CF00005DC02A8FFF7E4FE00200BB0F0BD3A5D32
:104D000002A963189A740134F1E730B589B000281C
:104D100014DD0C68E30711D5102268460021FFF767
:104D200017FD6B466A4665105D73684663122D0E6B
:104D300064149373D4731574FFF7C2FE002009B096
:104D400030BD0000174B184A5968002903D00021D4
:104D5000596001319160196900291FD00020186144
:104D60008023DB00D3581149012B18D1A923DB0084
:104D7000D3585B420B600E490B78032B01D80133EB
:104D80000B7003200B490B78013303400B700A4969
:104D90005B015B1809495350012393607047086019
:104DA000FAE7C046FC10004000100040240000203C
:104DB0008C120020001200200212002004050000C6
:104DC00010B5034A1021034800F0C6F810BDC046D4
:104DD0000CCE000003CE0000044A05491368C854F5
:104DE00001339B059B0D13607047C046BC16002025
:104DF000BC12002070B5114C114A2368834202DCBA
:104E00000023236016E0155C411C2E00FA3E012EA3
:104E100005D899420FDA555C013D1F2D01D90800D4
:104E2000ECE70100151A565C6E5401318B42FADC36
:104E3000181A206070BD1570FAE7C046C81A002025
:104E4000C816002010B5FDF719FE064B1A688242FD
:104E500001D900221A601B68C31A03489842804196
:104E6000404210BDB8120020204E000010B5094C81
:104E7000094A23681268934200D110BD074AD05CEA
:104E8000FEF71CF80028F8D0236801339B059B0D22
:104E90002360ECE7C0160020BC160020BC120020E6
:104EA00010B50400064B074A1B6812689B1ADB43C7
:104EB0009B059B0DA34200DB10BDFFF7D7FFF1E779
:104EC000BC160020C016002070B50020FFF734F992
:104ED000FF260500002801D1280070BD03681C14BE
:104EE0003440FFF729F9DA2CF4D10500F2E7F7B5E1
:104EF000050056680191B000441C06301700FFF70A
:104F0000CFFFFB20FFF768FF1C20FFF765FFE8B22B
:104F1000FFF762FFE0B22412FFF75EFFE0B2FFF797
:104F20005BFF6B461879FFF757FF0025AE4200DCA8
:104F3000F7BDAB00FB189C680135E0B2FFF74CFFF2
:104F40002012C0B2FFF748FF2014C0B2FFF744FFA1
:104F5000200EFFF741FFE9E770B5074E3368092BD4
:104F600008DC0C255D43054C013328516419616050
:104F7000A260336070BDC046C41600201C2F002004
:104F8000F0B587B002900C00012803DC1B20FBF772
:104F9000EBFF45E0244B08680093C30709D40428BD
:104FA00007D90F2302681340042B02D1FEF704F83F
:104FB00000901D4B60680193C30709D4042807D9EA
:104FC0000F2302681340042B02D1FDF7F5FF019077
:104FD0000027164B1B680493049BBB42D6DD0C26AE
:104FE0007E43134B0099F618306806F07DFA051ED3
:104FF00005D17368B6680593059B9D4201DB0137B7
:10500000EAE730680199039606F06EFA0836002840
:1050100008D121000298039B083102385B68984749
:1050200007B0F0BD0135E7E7D6C70000C416002081
:105030001C2F002010B5FBF7D3FEFEF7E1FFFDF7B4
:10504000DFFEFEF773FBFEF7C1FBFFF7B9FE00F0D2
:1050500063FE01F021F810BD962210B51201002167
:10506000034805F0C1FE0022024B1A6010BDC04685
:10507000241C0020C8050020064B074A1B68126844
:105080009B1ADB439B059B0D0122834200DC00221F
:1050900010007047BC160020C0160020F8B50500AF
:1050A0000C0016001F1E0ED10320FFF7E5FF00289D
:1050B00008D0FA20FFF790FEE8B2FFF78DFEE0B2CD
:1050C000FFF78AFEF8BD501DFFF7D6FF0028F9D084
:1050D000FB20FFF781FEE8B2FFF77EFEE0B2FFF7AC
:1050E0007BFEF0B2FFF778FE3012C0B2FFF774FE1D
:1050F0003C00E31B9E42E5DD2078FFF76DFE0134A6
:10510000F7E7000070B50024F0250B4B1B68A342A5
:1051100002DCFFF7A1FF70BD2B006343074A9B1819
:105120001A78002A05D05978002311201A00FFF7B9
:10513000B5FF0134E9E7C046C8050020241C002063
:10514000F8B507000024F0252B0063430C4A013416
:105150009E18B74211D0317800290BD00133D15CB1
:10516000002311201A00FFF799FF2A0000213000C8
:1051700005F03AFE0A2CE7D1F8BD024B1C60F9E7B6
:10518000241C0020C8050020F0B5150001222F00C6
:105190005E4C1740A54401900291002F11D005AB41
:1051A0001A706A105A70120E1A71052269129970DB
:1051B0006D140299DD70FFF771FFCF239B009D44B2
:1051C000F0BD042D1ED90F232A681340042B25D1CE
:1051D000023B04AA28001371FDF7EEFE040006F05E
:1051E0008DF94B4B984200D91800B84204DC421CA0
:1051F00005AB02990198DEE701377B1EE35C05AA47
:10520000D355F2E7042D7CD1032304AA043D137186
:105210006B425D4105AB55710222EAE7092BCCD107
:10522000042205AB1A706A68511000916946521247
:1052300009789A70009A59701F2A01DD2022009285
:105240006A46127806ACDA70009BBB4202DC05AB02
:10525000E21ACEE70126BB00EB189868064006D19B
:10526000042837D90F2302681340022B0CD10123E5
:1052700023704310637042121B0E4014A270E07042
:10528000237105340137DFE7042B21D1023B237062
:10529000FDF792FE039006F031F9A31C0C2809D803
:1052A0006070864201D19C19ECE7039A925D9A5591
:1052B0000136F6E70C226270039A925D9A55013628
:1052C000092EF9D12E23E372237363730E34D9E7C9
:1052D000012B07D1032304382370434258416070E7
:1052E0000234CFE7092B09D1053B23704368E670F0
:1052F0005A105B126270A3700434C3E72670013445
:10530000C0E7002D00D058E77EE7C046C4FCFFFF91
:105310002303000070B502000024F0210D4E0800A8
:10532000604380194578954203D001340A2CF6D1A8
:1053300070BDF022002105F057FD074A1368013BBC
:10534000A34200D11460002329001A001120FFF7A6
:10535000A5FEEDE7241C0020C805002010B5B2B062
:1053600002236A460400137006F0C8F8C72800D963
:10537000C7200023984207DC421C6B46FE21142004
:10538000FFF78CFE32B010BD694601335A1EA25C95
:10539000CA54EFE730B5B3B002236A460500137074
:1053A00006F0ACF80400C72800D9C72400239C42AB
:1053B0000BDC20003230FFF773FD621C6B46FF21CF
:1053C0001420FFF76BFE33B030BD694601335A1E1F
:1053D000AA5CCA54EBE70000F7B5234B06001B6834
:1053E000F02100930023009A9A4211DC0024F0235C
:1053F0001A006243019201991C4A55182F78002F18
:1054000012D001340A2CF3D11948FFF7C3FF29E069
:105410000A005A43154882185078B04202D11278D7
:10542000002A1FD10133DEE7F0223900280005F001
:10543000DBFC02230D4A0199EB6053540D4AF10045
:105440008A58009B6E70AE70AA602F616F61A34294
:1054500002DC054B01341C60002331001A001020CF
:10546000FFF71CFEF7BDC046C8050020241C002025
:10547000A5D300008425002010B5FFF743FEFF24CC
:10548000084AE3005B429B18074AD35C043B012BAC
:1054900003D8E043C0B2FFF79FFF013C002CEFD1DF
:1054A00010BDC046FC07000084250020F7B50F00A2
:1054B000FF247F2501901E4AE300D31A1D4A9A1843
:1054C0001278062A01D0032A20D1FF22D2009B188D
:1054D000186883682B401C2B18D1C3681A002A4017
:1054E000042A13D102692A40192A0FD11B0A013359
:1054F0009B000C30C018FDF75FFD03780600002B01
:1055000010D005F0FBFF0023B84209D0013C002C6D
:10551000D1D1F7BD019AF15CD25C9142F6D1013351
:105520009F42F7DCE043C0B2FFF756FFEEE7C0460C
:1055300084250020FC07000070B50500FF24084A00
:10554000E3005B429B18074AD35CAB4203D1E043C4
:10555000C0B2FFF741FF013C002CF0D170BDC04646
:10556000FC07000084250020F7B5FDF787FA514BB2
:105570001A68824201D900221A601A684E49821ABA
:105580008A4200D883E01860FDF782FA071E00D136
:1055900001370020FDF76EFB01900020FDF77EFB38
:1055A000019B0090454C464D002B14D02368002BE6
:1055B00000D07AE02B682760002B00D171E0414BCE
:1055C00001261B78002B63D10920FFF7B5FF3E4B66
:1055D0001E703C4B1E70009B002B12D02B68002BC2
:1055E0000FD123682F60002B1ED0374B01261B786C
:1055F000002B52D10920FFF79FFF334B1E70314B18
:105600001E702368002B0FD02F4E3278002A0BD14A
:105610009F4200D227602368FB1A312B04D9072050
:10562000FFF78AFF012333702B68002B0FD0254E24
:105630003278002A0BD1BB4200D92F602B68FF1AA9
:10564000312F04D90820FFF777FF01233370236837
:10565000002B0CD0019B002B09D11B4E3378002B63
:1056600002D10720FFF768FF0023236033702B6807
:10567000002B0CD0009B002B09D1124C2378002B5F
:1056800002D10820FFF758FF00232B602370F7BDDD
:105690000720FFF751FF0C4B9CE70820FFF74CFF5A
:1056A000ADE7009B002B9CD1ABE7009A002A95D177
:1056B000AAE7C046B41200200F270000A412002061
:1056C000AC120020B0120020A812002037B5002430
:1056D0000500FFF717FD01A80194FDF7B9FA2100B5
:1056E0002000FEF75DF9FEF735FBFDF765FBFDF7E2
:1056F0007FFBFEF77BFCFDF7E7F9A54204D0FDF741
:1057000007FC0248FFF746FE37BDC04696D30000AF
:10571000002310B501001A001120FFF7BFFC10BDD7
:1057200007B56B46197069465A7013128B701314C3
:10573000120ECB700A716B46010005221320FFF791
:10574000ADFC07BD10B50A0001001220FFF71CFDDB
:1057500010BD70B5050008000C003230FFF7A0FB4B
:105760002B00220000211B20FFF798FC70BD10B514
:105770000C000300110014202200FFF78FFC10BD65
:10578000012370B5FF24084A41185B42884201D3C7
:10579000D84370BD06781D0A234073409B009B5878
:1057A00001306B40F2E7C04678CF0000002313B50C
:1057B00001930B4BC2000400D058002805D0436869
:1057C00008309900FFF7DCFF01900920FFF768FB24
:1057D00001AB042221001720FFF760FC13BDC04677
:1057E00084250020F7B50190FFF76EFB012504002A
:1057F000FF276D42002C01D12800FEBD266833141E
:105800003B40152B0DD121000198083105F06CFEAD
:10581000002801D135123D402000FEF78DFC040028
:10582000E8E71D2BF8D101256D42F5E7F0B580279B
:105830009DB0FFF71BFBA54CA54D2068FF00391A52
:105840004019FDF721FB23680600C3182360002BD5
:105850000ED11DB0F0BD2068391A2818FDF714FBD1
:10586000236806001B182360FDF708F9994B1860A0
:10587000002EF0DC2B78FA2B00D037E12368022BC6
:1058800007DCFFF7DFFA0028E3D00120FFF7B2FAC8
:10589000DFE76878AC78023818282BD803F0CCF80A
:1058A00019002C0030003400370040002A004A0064
:1058B0007C0086008A00A000F10002012A002A0074
:1058C0002A002A002A002A002A002A002A002A0088
:1058D0001001FF2C0ED02000FFF71CFD00227E4B94
:1058E000E100CA505B181A712100009213001320C6
:1058F000FEF726FE0320C9E72000FFF76DFDF9E75C
:105900002000FFF707FDF5E7FFF7B6FDF2E7FFF729
:10591000F9FB0020FFF7DAFE7048FFF73BFDE9E7EF
:10592000632CE7D86E4BA200D25821001520FFF758
:105930002BFCDFE7FFF7C8FAFF270400002CD9D0C3
:1059400025682B143B40152B04D02000FEF7F4FBF8
:105950000400F3E72000083005F0D0FD0600053014
:10596000FFF79EFAFB20FFF737FA2D121D20FFF7F5
:1059700033FAE8B2FFF730FAF0B2FFF72DFA30123F
:10598000C0B2FFF729FA25002B1B9E42DDDD287AE5
:10599000FFF722FA0135F7E700211D2000910B00E7
:1059A0000A00FEF7CDFDFDF7B3FAA3E72000FFF7ED
:1059B000FDFE9FE7FDF774F803AC4A4A64210090AE
:1059C000494B200005F022FD02232000237005F042
:1059D00095FD2300020000211620FFF75FFB89E7F9
:1059E00000243D4AE300D558002D27D06B689E0067
:1059F000701DFFF755FA2B000025320008332100F7
:105A00000120FFF74BFB2F00FFF75EFA2E00002866
:105A100018D1002F04D03A0001212000FFF767FAC7
:105A2000002D04D02A0002212000FFF760FA002E8A
:105A300004D0320000212000FFF759FA0134FF2C76
:105A4000CFD157E7FF2103681A120A40A24209D1B9
:105A50001A140A400B2A08D10B400CD0012B0CD091
:105A6000022B0CD0FEF768FBD1E7132AFAD10025F0
:105A70002F002E00F6E70600F4E70700F2E7050026
:105A8000F0E70024FFF73EFB2200210000942300F2
:105A9000DA20FEF755FDFF222100D2000E4805F066
:105AA000A3F980E7012C02D1FEF768FC22E7022C63
:105AB00002D1FEF7A7FD1DE70120FFF707FE19E75A
:105AC000002321001A001A2087E7C046C81A0020C8
:105AD000C8160020B81200208425002078D30000CA
:105AE0007C2D00208FD300008AD30000FB2B00D038
:105AF000CBE62268042A00DCC3E62E79E878574B0F
:105B0000360206439E4200DDBFE6331D9A4200DCAA
:105B1000B7E6EB5CFE2B00D0B7E66B78AC78771E6F
:105B20001B2B61D019D8072B47D0082B1CD0012B79
:105B300018D1FF2C16D02000FFF7ECFB6D79484AF6
:105B4000B31E009221002A000A20FEF7F9FC454B03
:105B5000E400E0501B191D7104E01D2B56D048D302
:105B60001E2B6AD0701D91E6632CFBD86A79022A3D
:105B700013D0032A1BD0012AF4D1E979AB790902A9
:105B800019432B7AA4001B0419436B7A1B060B43A1
:105B90005B001343344AA350E4E7002FE2DDB11E5B
:105BA0002F48FDF717FC304BA400E050DAE7AB7943
:105BB000A4005A1E93419B00ECE7632FD2DC03AD97
:105BC0003A002A49280005F0F3F800232800EB5595
:105BD000FFF708FE0028C5DB234B8000C2582100D8
:105BE0001520FFF7D1FABDE739002048FFF75EFC2A
:105BF000B8E7FF2CB6D06A79022AB3D818490B202F
:105C000000912100B31EFEF79BFCABE7632F00DD84
:105C10006327002303A99F420ADCFB430022DB1712
:105C20003B40CB181A70152000917B1C2100EAE73D
:105C3000EA185279CA540133EDE7012C92D1002FB2
:105C400090DD6B79002B03D01C00322B00DD322459
:105C500064235C43064B1C6084E7C046F6030000E7
:105C6000CE160020842500207C2D0020CD1600209B
:105C7000040000200120704710B5064C200000F001
:105C800063FC0549200000F087FC0122034B1A60E9
:105C900010BDC046D41A0020801A0600CC1A00207D
:105CA00010B501210D20FCF701FF01210E20FCF7AA
:105CB000FDFE00210F20FCF7F9FE044C200000F04F
:105CC000CFFD1021200000F0E7FD10BD8C1B00204F
:105CD00010B504680D20E30703D56410FF2C03D929
:105CE0001720FBF741F910BDFFF7DAFFE1B20248D8
:105CF00000F0F4FD0020F6E78C1B002010B5FFF744
:105D0000CFFF0021034800F0E9FD430001201843C4
:105D100010BDC0468C1B002010B5034A0821034863
:105D2000FFF71AF910BDC046BCD30000FCD3000039
:105D3000F8B5012306681E4205D045681D4202D011
:105D400084681C4203D10D20FBF70EF9F8BD7610D4
:105D50001520802EF8D86D101620FF2DF4D8641071
:105D6000FF2C01D91720EFE70B4B1B68002B01D14B
:105D7000FFF782FF094FF1B2380000F0A4FCE9B24E
:105D8000380000F0A7FBE1B2380000F0A3FB3800B8
:105D900000F004FD0020D9E7CC1A0020D41A00201E
:105DA000F7B501221400904222DD0D682A421FD06F
:105DB0001D4B15411B684C68002B01D1FFF75CFFA0
:105DC000E9B201272500194E3D40300000F07BFC70
:105DD000002D0FD03C413000E1B200F07BFB3000E1
:105DE00000F0DCFC0024A04202D02320FBF7BCF82A
:105DF0002000FEBD042CF2D90F2322681340092B8A
:105E0000EDD163685B100193019BAB42E7DDAB0012
:105E1000E3189968394204D04910C9B2300000F043
:105E200059FB0135F0E7C046CC1A0020D41A0020F7
:105E3000144B70B51B6805000E00002B01D1FFF755
:105E40001BFF114CEDB22900200000F03CFCF1B228
:105E5000200000F03FFB0021200000F03FFC002864
:105E600001D0404270BD01222900200000F026FC34
:105E7000200000F020FB0028FAD0200000F020FBDA
:105E8000F0E7C046CC1A0020D41A002010B5012437
:105E90000368234202D04168214203D10D20FBF761
:105EA00063F810BD5810802801D91520F7E7491074
:105EB000FF2901D91620F2E7FFF7BAFF400020437F
:105EC000EFE710B50400012814D105211820FFF7D1
:105ED000AFFF7F282BDC03007F3301DA7F204042B5
:105EE00064235B4258437F2102F03AFE052C00D127
:105EF000404210BD032811D101001820FFF798FF80
:105F00007F2814DC03007F3301DA7F2040426423C2
:105F10005B4258437F2102F023FEEAE70020052C74
:105F2000F5D107211830FFF783FF7F2802DD013804
:105F3000FF38D0E703007F3301DA7F20404264233B
:105F40005B4258437F2102F00BFED1E770B5012080
:105F5000FFF7B7FF04000320FFF7B3FF050005209C
:105F6000FFF7AFFF6D43644340436419201804F00A
:105F700007FE01F0D1FA04F0CDFD430001201843E3
:105F800070BD10B50120FFF79CFF430001201843AE
:105F900010BD10B50320FFF794FF43000120184304
:105FA00010BD10B50520FFF78CFF430001201843FA
:105FB00010BD10B508211820FFF73AFF0300C00FED
:105FC000C0180123401015304000184310BD0000D8
:105FD000F8B501231C00984229DD0F683B4226D00A
:105FE0004E6835001D4022D1042E20D90F22316881
:105FF0000A40092A1BD173685C10202C00DD202484
:10600000134B1B68002B01D1FFF736FE7F10F9B24E
:10601000104F2200380000F051FBA54214DA38007E
:1060200000F049FA002804D101246D002C4320001F
:10603000F8BD380000F044FA0122AB004000F3182C
:1060400010439860AD18E8E764000125EEE7C0460C
:10605000CC1A0020D41A002000207047012070477D
:1060600000207047002070470120704700207047D3
:1060700000207047002070470020704700207047C4
:1060800000207047002070470020704700207047B4
:10609000704770477047000010B5034A0E2103484F
:1060A000FEF75AFF10BDC0464CD40000BCD400001F
:1060B0000378013B1F2B00D970470130F8E710B57A
:1060C000FFF7F6FF0378002B0BD00130222B11D104
:1060D0000378002B03D0421C222B03D11000FFF7C2
:1060E000E7FF10BD5C2B03D14378002B00D0821C4E
:1060F0001000EDE73A2BF2D02C2BF0D07B2B0BD1FC
:10610000FFF7D6FF0378002BE9D07D2B01D10130BA
:10611000E5E7FFF7D4FFF5E720225B2B14D1FFF76B
:10612000C7FF0378002BDAD05D2BF0D0FFF7C7FF55
:10613000F7E7202BD3DD2C2BD3D0190091435D2919
:10614000CFD0222BCDD001300378002BF1D1C6E780
:10615000002210B5904216D0FFF7AAFF0378042260
:10616000222B10D0023A7B2B0DD0013A5B2B0AD0A8
:10617000190030390232092905D92D2B05D1417872
:10618000303909290AD8100010BD0522742BFAD025
:106190000132662BF7D001326E2BF4D0581E8341AA
:1061A0005A42F0E770B5FFF783FF037801222D2BE9
:1061B00001D18018023A00230A2502E06B43013026
:1061C000CB1801783039CCB2092CF7D95A431000DA
:1061D00070BDF8B50C001500FFF76AFF0378222B9D
:1061E00002D000232370F8BD0D236A1E210008256C
:1061F0000C260A279C4601300378222B02D100236B
:106200000B70F0E7002BFAD0441C5C2B0BD14378C9
:10621000841C622B0ED0662B0ED06E2B0ED0722BF0
:106220000ED0742B0ED0002AE9DD0B70013A01313B
:106230002000E1E72B00F6E73300F4E73B00F2E74C
:106240006346F0E70923EEE710B50400FFF737FFD8
:10625000A04202D90378202B00D910BD0138F7E7FE
:1062600010B5002815D00378002B13D0FFF720FFBE
:106270002021037802008B4300205D2B09D0100001
:10628000FFF71DFF03782C3B5A425341C018FFF71C
:106290000FFF10BD1800FCE70300002070B50C00D4
:1062A00081420EDD1A785B2A0BD1581CFFF700FFE4
:1062B0000125AC4205D0FFF7D3FF002801D00135FE
:1062C000F7E770BD70B50C001500002901D0002360
:1062D0000B70002820D00378002B1ED0FFF7E8FEBB
:1062E000037806002C2B03D10130FFF7E1FE0600F6
:1062F000337800207D2B0FD0844204D02A00210067
:106300003000FFF766FF3000FFF7D9FE03783A2B25
:1063100002D10130FFF7CCFE70BD1800FCE7F0B5EC
:106320000D0004009DB02E78002E35D02E212800BF
:1063300005F0CCF8071E14D0431B0193303E092E04
:1063400014D82800FFF72EFF01002000FFF7A4FF5C
:106350000400002C20D0002F1ED0019B0133ED182B
:10636000E1E7280005F0CAF80190E7E723787B2BE6
:1063700011D1601C642203A9FFF7A4FF041E0BD0F7
:10638000019A290003A805F0C0F80028E1D02000F8
:10639000FFF795FEEEE7002420001DB0F0BD70B5BC
:1063A000050000200C0081421DDD2800FFF7D0FE13
:1063B0000300681C012B14D00020022B13D10022F3
:1063C000681C1100FFF77EFF012C0CD0FFF748FF7F
:1063D00000221100FFF776FF013CF5E7FFF740FFD1
:1063E000013C012CFAD170BDF8B5050000200C006D
:1063F00016001F0081420DDD2800FFF7A9FE0300F3
:106400000020022B06D1681C3A003100FFF75AFF2A
:10641000012C00D1F8BDFFF723FF3A003100FFF750
:1064200051FF013CF4E710B50024A04218D0FFF75B
:106430003FFE03787B2B0AD1013000221100FFF7C9
:1064400041FF00280CD0FFF73AFE0134F5E75B2B43
:1064500006D10130FFF704FF002801D00134F9E72D
:10646000200010BD10B5FCF7D7FCFCF777FDFEF758
:10647000E1FD0448FEF78EFFFEF7C8F8FEF7FCFFCB
:1064800010BDC04645D5000010B5FCF7D3F910BDCE
:10649000F8B505000E0017000024BC4208D02B6898
:1064A000315D1B6828009847002801D00134F4E7CB
:1064B0002000F8BD704710B51C3000F061FA10BD27
:1064C00010B51C3000F04EFA10BD10B51C3000F0B5
:1064D0005DFA10BD70B5437E0D00002B01D1002088
:1064E00070BD6430040000F05AFA0028F7D1200093
:1064F000290000F028FA0120F2E70000F7B5019327
:10650000FA23002504009B0083600D4B456008338F
:1065100003601C300F00160000F00AFA20006430FF
:1065200000F006FA074A2761B600B35820006375E9
:10653000019B9B009B586576A576A375FEBDC04662
:1065400060D5000024D600000123A022C375837DFE
:106550000E49C133FF33D2059B009950437DC133AF
:10656000FF339B009950CC220169094B5204CA5059
:1065700005220169243BCA50827D01690833CA5053
:106580000269417D034BD1507047C0460C060000A4
:10659000240500000C050000A022002310B50469AA
:1065A000D200A3500A4CA1420FD90A4C8C425B4145
:1065B00009495B420B40CD21C9045B1804690749B6
:1065C000635005210369995010BDCC235B04F5E7A6
:1065D000A086010090D00300000098FD2405000073
:1065E000F7B5040000200D000193824265D016002B
:1065F000402A00D9402627001C37380000F0AEF9A9
:10660000B1232269DB00D550802201232169920049
:106610008B50A27E002A03D1226913622269136083
:106620000025731EAB4207D1019B002B04D08022B2
:106630000221236992009950012223691A62236979
:10664000FC33DA68002A02D19A6A002AF9D09A6AE1
:10665000002A0BD1DA60A3232269DB00D15838006D
:10666000C9B2013500F06FF9B542DAD3019B226956
:10667000002B0FD11300FC339B6A002B0AD101338E
:10668000A376D3612369FC33DA6C002AFCD00022A4
:10669000DA640AE000230121A37651611A0023691C
:1066A000FC3399680029FCD09A602369FC339A6A0C
:1066B000002A01D000229A62E8B2FEBD10B5012383
:1066C000FFF78EFF10BD0300AC3310B50400197046
:1066D000643000F043F90123637610BD002302000B
:1066E00070B5AC3243760D001178B1220400006918
:1066F000D20081508022216992008B50226901339F
:1067000013622269936026006436300000F038F985
:10671000002812D0300000F025F91E4B2269D0501D
:106720002369FC331A6A002A02D19A6A002AF9D036
:106730009A6A002A01D11A62E5E723690122002D35
:106740000DD11900FC31896A002908D1DA61236969
:10675000FC33DA6C002AFCD00022DA6407E05A61CC
:106760002369FC339A68002AFCD000229A6000203A
:106770002369FC339A6A82420BD098622169064AE7
:106780008B588B501800022B03D0181F431E9841C2
:10679000033070BD1C050000C404000010B50121C9
:1067A000FFF79CFF10BD000010B513231222024911
:1067B0000248FFF7A3FE10BD00400040D41A00209D
:1067C00070B5002504AC24780573A94205D10A4BA5
:1067D0000A4A23210A4804F07DFA0160094992001F
:1067E00052589B0002715B58A40083716358856006
:1067F00043710223C37170BD80D50000E5D5000050
:106800008ED5000024D60000037B002B04D14373F7
:106810008373036101330373704700001FB5019157
:10682000A02100240068C900D2B24450012A10D02F
:10683000A24209D0032A0AD0074A8350074B019A83
:10684000C250012343501FBD02221343F4E7042228
:10685000FBE70622F9E7C0465405000024050000C6
:1068600010B50400FFF7D0FFA1222368A179D20060
:1068700099506179064A2000995021790432995043
:10688000044B19685A689B68FFF7C8FF10BDC046E3
:106890000C050000A01B00204BB2002B0FDB802357
:1068A0003F290FD81F290FD80F290FD807290FD834
:1068B00003290FD81B060168074A8B5070478023B5
:1068C0009B04F8E7DB04F6E71B05F4E75B05F2E75A
:1068D0009B05F0E7DB05EEE7240500000368074AA7
:1068E00099501A00FC32D1680029FCD0A321C900BC
:1068F00058580023C0B2D3607047C0461C05000042
:1069000007B58022074BD2051A6000229A60023236
:106910001A7111230E320093034905330348FFF720
:106920004FFF07BDA01B0020003000408C1B002043
:1069300010B540220021040004F056FA0023200084
:106940002364636410BD10B53F24026C531C2340C4
:10695000446C9C4201D08154036410BD0023036445
:1069600043647047436C026C934206D03F21C25C83
:1069700001330B4043641000704701204042FBE7A5
:10698000036C406C181A00D540307047436C026CA1
:10699000934201D0C05C704701204042FBE73F2298
:1069A000036C406C01331340181A43425841C0B283
:1069B0007047000003210A4802680A430260094840
:1069C00002680A4302600849084A094B9B1A03DD22
:1069D000043BC858D050FBDC00F012F8F9F794FBE8
:1069E00024050040540500406CDB0000000000203E
:1069F00060020020FEE7FEE7FEE7FEE7FEE7FEE7B7
:106A00002D4B10B51A68D2B2012A0FD12B4A126849
:106A100012070BD12A4AE0241168F0220800104026
:106A200021422DD12749096811422CD01A68D2B2CF
:106A3000012A12D12149096809070ED1F020204905
:106A400009680140402908D11E490968014204D162
:106A50008020C121C005C90042501B68DBB2012B58
:106A60000DD1164B1B681B0709D1154B1A68F02373
:106A70001A40A02A0FD1134A12681A420ED010BD34
:106A80003028CFD0D2E7104A104911608021104A37
:106A900009021160CAE7D02AF1D1ECE70D4B1A6860
:106AA000012A04D00C4A1A601A68012AFCD1C022BB
:106AB0000A4B1A60E3E7C046E00F00F0E40F00F075
:106AC000E80F00F0EC0F00F004050040DFFF07C006
:106AD000186C004000EC06407593000014EC064072
:106AE0000120704710B503681322DB69984710BD79
:106AF00070470000054B0269D1500369FC331A6AE4
:106B0000002AFCD0002201201A6270471C050000F8
:106B1000030010B55C331A781F231A401E3B19007E
:106B20009140114AD167C222042104699200A15008
:106B3000026953600269D360A02300220169DB006F
:106B4000CA5001230169094A5B428B500169084A16
:106B50008B5001690C3A8B50016908328B5014300C
:106B6000FFF7FCFE10BDC04604E100E00C0500008C
:106B70001405000010B51430FFF702FF10BD10B56A
:106B80001430FFF703FF10BD10B51430FFF7EAFE15
:106B900010BD0000030070B55E331A780469724BB3
:106BA000E25003005D331A780469704BE250030031
:106BB00061331C7802696E4B012C00D09EE0050009
:106BC0005F352E78A225ED0056510200603215780F
:106BD000A1220669D200B5500269D4509623DB0089
:106BE000994200D88CE096231B01994200D88AE094
:106BF00096235B01994200D888E096239B01994235
:106C000000D885E0E1239B01994200D882E09623D9
:106C1000DB01994200D880E0E123DB01994200D8F2
:106C20007DE096231B02994200D87AE0E1231B0203
:106C3000994200D877E096235B02994200D874E02D
:106C4000E1235B02994200D871E0E1239B02994263
:106C500000D86EE0474B994200D86CE0E123DB029C
:106C6000994200D86AE0E122002312038A425B4184
:106C7000414A5B421340802252059B1801693F4AFA
:106C80008B50A02304220169DB00CA500021036954
:106C9000FC33D9600369FC331962012301690B607D
:106CA00001698B60C1210469890062501F215C3039
:106CB00002780A4093406231314AFF31535000213B
:106CC000415600293CDA0F230B40083B2D4C9B0812
:106CD0009B001B1903242140A140FC348C40DD693A
:106CE000A5432C00C0258D4029002143D9611F23D5
:106CF000017819401E3B8B40136070BD00246CE787
:106D00009E23DB02BAE79D231B03B7E71E4BB5E7C3
:106D10001E4BB3E7EC239B03B0E71D4BAEE71D4BC7
:106D2000ACE71D4BAAE71D4BA8E71D4BA6E71D4B83
:106D3000A4E71D4BA2E78023DB049FE71B4B9DE7E5
:106D40008C080F4BA400E41803230B40FF21C0253F
:106D5000DB009940AD0066598E433100C0269E404D
:106D600033000B436351C2E70C050000140500001B
:106D70006C05000090D0030000D0BEFE240500008A
:106D800000E100E000ED00E000B01300005027003B
:106D900000A04E0000F0750000509D0000F0EB00D8
:106DA00000903A0100E0D70100B0AF0300705F0728
:106DB000F7B5009308AB1B7800250193FA23040074
:106DC0009B0083600E4B45600833036014300F0056
:106DD0001600FFF7ADFD23005C3327611E70009B9A
:106DE000084A9B00995823005D331970019B2000CD
:106DF0009B009A5823005E33DD701A70FEBDC046BA
:106E0000A0D6000024D60000036910B51A00FC3299
:106E1000D2680400002A0AD0A322D2009958143064
:106E2000C9B2FFF790FD00222369FC33DA6010BD80
:106E300010B50248FFF7E8FF10BDC046AC1B0020AC
:106E40001D2307B502220093024901330248FFF7D0
:106E5000AFFF07BD00200040AC1B002010B500288C
:106E600001D004F07DFA10BD7047000010B500F0AD
:106E700011F8FFF7F9FF012000F000FAFFF7F2FA2E
:106E8000FFF702FB024B002BFAD000E000BFF7E750
:106E900000000000C420114B80001A581049114016
:106EA000C02212020A431A50C021802249009202D5
:106EB0005A501A608023A3220021DB05D20099508A
:106EC0000122F9309A60074BFF301950C12002317E
:106ED00080001950403019501A60704700E100E0FE
:106EE000FF00FFFF00100140014B18607047C046D3
:106EF00074000020F7B500231E285AD8384B8000B4
:106F0000C258042A5BD007D8022A54D055D804238B
:106F1000012A09D000234CE0062A54D051D31A2A62
:106F200053D002231B2AF5D12E4A116808294ED9C5
:106F300009294FD00A240226A02001252A4AC00090
:106F400015502A482A4D07681C20BF0007402948D1
:106F5000019700685759009027481B0207401F43BC
:106F6000C02300989B020340FF205751575900024D
:106F700007401F43019B1F43009B5801602318409B
:106F800007433E43565101251C4B156058680028A5
:106F9000FCD000205860A1230125DB00D3585560A8
:106FA000A025ED0050511BB2A14202D015D2611AAA
:106FB000CB401800FEBD0823B6E71023B4E720231A
:106FC000B2E74023B0E78023AEE70123ACE7082413
:106FD0000026B1E70C000126AEE7091B8B40E8E76D
:106FE00024D6000070000020007000402C0000201B
:106FF0000405000030000020FF00FFFFFC7000408F
:10700000F0B51E285BD8364B8000C258354B1E6841
:10701000002E30D1C227344BBF00D859334C032542
:107020000440C02000022043D851C02480206400C6
:10703000800018512E4F18602E4B803CD859FF3CD1
:10704000A043D8510437D859A8432043D851083712
:10705000D8590C35A8438446072065462843D851A3
:10706000A820C0001E50C1208026800076021E503D
:107070001C601C4B1C60142500202B001E4C2E0095
:1070800046433659771C1BD14343E250A0230325C6
:10709000C132FF329200DB05D550184B1A68082A1E
:1070A00014D114234343E3189A6812485132FF3233
:1070B000920059601150DA68C1239B00C250F0BDA4
:1070C0009642E1D001300328D9D1F8E7082A02D945
:1070D000083AD140E5E708239A1A9140E1E7C04613
:1070E00024D60000101C002000E100E0FF00FFFF9C
:1070F00004050000009000403400002074000020CF
:107100002149F0B54A6C2148002A14D0A025A126B7
:1071100000230124ED05F600C258571C06D0C718FD
:107120007F68002F02D027009740AF5114333C2BCB
:10713000F2D100234B64A0230121DB0500260F00C0
:107140009C4614234B43C3181A1F1268104C0E4D53
:10715000920014195219526C002A10D01A00143AD5
:107160001268551C09D0103B1B68FF2B05D03B0053
:10717000934065461A00074BEA50FC3466640131BF
:107180000429DED1F0BDC046FC9000403400002050
:10719000009000400C05000000B51E2810D80C4AD5
:1071A0008000835803290BD8A0220800C133FF3385
:1071B000D2059B0001F036FC020905070021D150E1
:1071C00000BD0C21FBE70421F9E70321F7E7C046E6
:1071D00024D600001E280AD8074B8000C25801237D
:1071E0009340A022D205002902D104495350704790
:1071F000A121C900FAE7C04624D600000C05000012
:10720000030000201E2B0AD8A021A222C905D2000B
:107210008858034A9B009B58D84001231840704768
:1072200024D60000F7B506000D000C008B18019362
:10723000019B671B9C4207D0336821781B68300094
:10724000984701340028F3D13800FEBD0849094AA7
:10725000094B10B51B688858FA22190A1B061843F7
:107260009200002301F0B4FD4904C00B084310BD97
:107270000010014004050000141C002070B5041E1D
:1072800009D0FFF7E3FF050000F014F8FFF7DEFF79
:10729000401BA042F8D370BD0022044B9A60044A00
:1072A00013680133DBB213607047C046FC10014025
:1072B000141C002070470000F0B5C64600B5CB0F87
:1072C0009846404A4B005B0D9A1882B00D000400AE
:1072D000132A2FDC002A49DB3B4F17413E000E40AA
:1072E000064323D07F08390029400C430AD0374990
:1072F000BD438C4663445C425C418023DB02134106
:10730000E4071D434146CE0031492B008E1922006F
:10731000346875682000290001F000FF0090019199
:107320000098019922002B0003F090F802B004BCF1
:107330009046F0BD332A08DD8023DB009A42F5D168
:1073400002000B0001F0EAFEF0E7224A9446012217
:1073500063445242DA400242E8D052080242D1D09D
:1073600094438022D2051A411443CBE74B005B08BB
:107370000343DBD00B031B0B1C43634223438024DA
:107380004D0C24031B0B23406D042B431900434673
:10739000DA000F4B9B181C685D6802000B00200090
:1073A000290001F0BBFE0090019100980199220094
:1073B0002B0003F04BF842464B005B08D6073343E3
:1073C0001900B3E701FCFFFFFFFF0F00EEFBFFFF1B
:1073D000D0D60000EDFBFFFFF8B5274A4B005B0D50
:1073E0009A180C000700132A10DC002A36DB234B06
:1073F00013410B423AD08024240314410020641826
:107400009C430600250030002900F8BD332A0EDD1C
:1074100080230600DB000D009A42F4D102000B002D
:107420003800210001F07AFE06000D00EBE7144D54
:107430000600AC46012563446D42DD40AC46634620
:107440000D000342DFD033239A1A323B93401818C1
:10745000874200D94C1C63469843D2E7C90FCC073A
:107460000020531CCDD1074B1C43CAE706000D007A
:107470000028C0D1C7E7C04601FCFFFFFFFF0F0097
:10748000EDFBFFFF0000F03F30B5214A4B0087B015
:107490005B0893421EDD1F4A934205DD02000B008C
:1074A00002F0D4FF07B030BD02AA00F095F8032324
:1074B0001840049A059B012813D002281DD00028EB
:1074C00014D00298039900F06FFB80231B069C46A2
:1074D0006144E7E7002300220093002301F0DEF877
:1074E000E0E70298039900F05FFBDBE701240298D4
:1074F0000399009401F0D2F8D4E70124029803998B
:10750000009401F0CBF880231B069C466144C9E738
:10751000FB21E93FFFFFEF7FF0B54746CE4680B540
:107520008DB004000D0000F067FA294B06001B78AF
:107530000F005BB29846013310D022002B002000D0
:10754000290003F0CBFA8146002807D1002200234E
:107550002000290001F014FC002806D13000390079
:107560000DB00CBC90469946F0BD01230293194B17
:107570000694079503934B460A9343460494059556
:10758000002B15D0002300221900100002F0E2F8B1
:10759000434608900991022B0ED103F0B9FB212339
:1075A00003600A9B0193002B0CD1089E099FD5E72D
:1075B000002300240893099402A801F0C1F90028CF
:1075C000EFD1EAE703F0A4FB0A9B01930360ECE729
:1075D00078000020E0D60000F0B54E464546DE4675
:1075E0005746E0B5E14B4C008FB0904689466408A1
:1075F0009C4200DC87E0DE4B9C4222DCDD4A002915
:1076000000DC92E0DC4B02F021FFDB4B06000F00B8
:107610009C4200D17EE1D94AD94B02F017FF02000B
:107620000B00414630000A604B60390002F00EFF4B
:10763000D34BD24A02F00AFF434601259860D96035
:107640006BE0D04B9C4200DC8FE0CF4B9C4200DDD6
:1076500055E1CE4A231592469A4451460905631ACC
:1076600019001D00040003F055FA03F089FA020026
:107670000B00200029000892099302F0E7FE002287
:10768000C34B02F071FC0F00060003F043FA03F055
:1076900077FA04000D0002000B00300039000A9454
:1076A0000B9502F0D3FE0022B94B02F05DFC0022E4
:1076B00000230C900D9101F05DFB002800D192E1B8
:1076C000002300222000290001F054FB43424341E3
:1076D0000133B04A41460192022208A80092524664
:1076E00000F07CFB4B460500002B16DA8022434657
:1076F0001206944642465B68454263445360D36831
:107700006344D36009E00B00020041460A604B600D
:107710000022002300258A60CB6028000FB03CBC0B
:1077200090469946A246AB46F0BD934B01F0F6FC5D
:10773000914B06000F009C4200D13DE18F4A904BD7
:1077400001F0ECFC02000B00414630000A604B6087
:10775000390002F07BFE894A894B01F0DFFC0125EC
:1077600043466D429860D960D7E701F049F88A4AEC
:107770008A4B06000F0002F0F7FB0022884B01F055
:10778000CDFC03F0C7F9050003F0FAF9794A7A4B0A
:107790000490059102F0E8FB02000B003000390074
:1077A00002F054FE754A06000F0004980599744BC8
:1077B00002F0DAFB029003911F2D00DCC7E0029A71
:1077C000039B3000390002F041FE83468A4653464F
:1077D0005B0024155B0DE31A102B6CDD04980599F2
:1077E000D322674B520502F0BFFB02000B003000B2
:1077F00039000292039302F029FE0A0001001300EF
:107800000691079202003900300002F01FFE029A32
:10781000039B02F01BFE06000F0004980599614AC5
:10782000614B02F0A1FB32003B0002F00FFE069E0E
:10783000079F0B000200390030000292039302F010
:1078400005FE4B005B0D83468A46E41A312C32DD7F
:1078500004980599B822544B920502F085FB030069
:107860000C000200029303940B000698079902F0A3
:10787000EDFD02000B0006000F000698079902F0CC
:10788000E5FD029A039B02F0E1FD484A0290039154
:1078900004980599464B02F067FB029A039B02F09D
:1078A000D5FD02000B00300039000292039302F074
:1078B000CDFD83468A465A465346414630000A600B
:1078C0004B60390002F0C2FD029A039B02F0BEFD3C
:1078D00044460B000200A260E3604B46002B00DB35
:1078E0001BE75B46236080231B06534463608023B1
:1078F0001B069C466144A060E1606D420DE70B00F1
:10790000020002F0A3FD434600259860D96018608C
:10791000596002E7D3221A4B520502F097FD214A23
:10792000214B0D00040002F091FD02000B004146C6
:1079300020000A604B60290002F088FD1A4B194AAA
:1079400002F084FD434601259860D960E5E6020017
:107950000B003000390002F079FD6B1E154A9B00C8
:107960009B5883468A46A342A5D130E7FB21E93FD5
:107970007BD9024000004054FB21F93F3163621A79
:1079800061B4D03DFB213941FFFFEF7FEAFBFFFFF0
:107990000000704168D7000083C8C96D305FE43FC4
:1079A0000000E03F7370032E8A19A33BC1492025D4
:1079B0009A837B39E8D60000D3220C4B520501F0A4
:1079C000ADFB0B4A0B4B04000D0001F0A7FB0200BE
:1079D0000B00414620000A604B60290002F036FD92
:1079E000034A044BB9E6032373E6C04661B4D03DB5
:1079F0007370032E8A19A33BF8B54746CE46674BF2
:107A000080B50A000F00190005003940994200D1E5
:107A10009BE004000100002F69DD3F1500D1B4E0B8
:107A20005F4B12039C468023120B5B0313435B00E6
:107A3000CA0F67449B184A00F80703D5D20F5B00B2
:107A40009B188A0079108C460021802016248946D4
:107A500080030D189D4202DC29185B1B8144D50F61
:107A60005B00013C5B1952004008002CF1D1002062
:107A70008046802020250027000609E08B425CD04C
:107A8000D40F5B00013DE31852004008002D16D0D2
:107A9000C4198B42F2DD27180E00002C49DB5B1A5B
:107AA000A242894149425B1A121BD40F5B00013D7F
:107AB00080443100E31852004008002DE8D1134300
:107AC0004ED143465B0837494A46884649465210DC
:107AD0004244C90702D5802109060B4361460F05C0
:107AE000BD18180029000CBC90469946F8BD7B00D3
:107AF0005B0803433900002BF5D0002F3CD1E30A8B
:107B0000153A6405002BFAD08020400303423FD190
:107B1000002700E00F005B00791C0342FAD025002B
:107B200020208D40401A2900D71B2200C2401A4352
:107B300076E7FE43F60F8E19B1E79442A0D82718D6
:107B4000002CF6DB1E000023AEE702003B002800FD
:107B5000390002F009FA2A003B0001F0DFFAC2E71F
:107B60004346013303D0434601335B08ABE70123AF
:107B700098460023C144A6E73B00020002F066FCE1
:107B800002000B0001F0E6FDADE713000022BBE7A9
:107B90000127210020207F42C6E7C0460000F07F79
:107BA00001FCFFFF0000E03FF0B54746CE4680B540
:107BB00087B000920193754B4F00814688467F083D
:107BC0009F4263DC02F0A6FF002800D1D4E04A46C1
:107BD00043464846414602F0C7F904000D006C4A8E
:107BE0006C4B02F0C1F96C4A6C4B01F097FA220021
:107BF0002B0002F0B9F96A4A6A4B02F027FC220016
:107C00002B0002F0B1F9684A684B01F087FA2200B4
:107C10002B0002F0A9F9664A664B02F017FC22001D
:107C20002B0002F0A1F9644A644B01F077FA2200BC
:107C30002B0002F099F9029003910022604B200082
:107C4000290002F091F9029A039B06000F00200020
:107C5000290002F089F9009A019B04000D004846B2
:107C6000414602F081F902000B002000290002F0D9
:107C7000EDFB02000B003000390002F0E7FB0200D0
:107C80000B0000204F4902F0E1FB70E002000B0006
:107C900002F06AF904000D003D4A3E4B02F064F91F
:107CA0003D4A3E4B01F03AFA22002B0002F05CF90B
:107CB0003B4A3C4B02F0CAFB22002B0002F054F975
:107CC000394A3A4B01F02AFA22002B0002F04CF913
:107CD000374A384B02F0BAFB22002B0002F044F97D
:107CE000354A364B01F01AFA2B00220002F03CF91B
:107CF000354B029003919F429FDD344B00229F42FF
:107D00003DDC334900207B182E4916001F0002F08D
:107D10009DFB049005910022294B2000290002F0D0
:107D200023F932003B0002F091FB029A039B06000C
:107D30000F002000290002F017F9009A019B0400AF
:107D40000D004846414602F00FF902000B002000EA
:107D5000290002F07BFB02000B003000390002F02A
:107D600075FB02000B000498059902F06FFB07B049
:107D70000CBC90469946F0BD00201249F7E7154B20
:107D8000002604920593144FC5E7C046FFFF3F3E0F
:107D9000D43888BEE9FAA8BDC4B1B4BD9EEE213E78
:107DA000AD529C804F7E923E9015CB19A001FA3EB9
:107DB0007751C1166CC1563F4C5555555555A53F89
:107DC0000000E03F0000F03F3233D33F0000E93FC6
:107DD0000000E0FF0000E73F0000D23FF0B5DE46C4
:107DE0004E4645465746E0B5DC4CA5440D9114007F
:107DF0001900A49A0993DA4B9200D6584D1E0390AD
:107E00001821E01E0696029500F0AAFEC343010069
:107E1000DB1719404B1C9A009B1ADB001B190B91B6
:107E200005934C1B771918D4A59BA5009C463F19B8
:107E300022AE6544013707E0286802F0A1FE013454
:107E400003C60435BC4208D0002CF5DA002000211E
:107E5000013403C60435BC42F6D1069B002B01DA7F
:107E600000F0FDFB069B03990133DB009A46099B5A
:107E7000DA00944600920022914672AA0492B94A0E
:107E80006144934688469AAB63449B44029B002B13
:107E900000DABCE15D4600260027039C4D442A68B9
:107EA0006B6803CC02F060F802000B003000390070
:107EB00001F034F9083D06000F004445EFD1049B62
:107EC0004B441E605F6008239C46E144D145DDD1F0
:107ED0000EA804218446494261448C46069A9300C8
:107EE0009C44614684460A910399083B63448C464E
:107EF0000C93009B009263449B46009A0498D10027
:107F000003008C46634408911E685F68002A33DDD5
:107F1000954980468C466244D300984470AB9A469B
:107F20000EAB99460022914B3000390002F01CF84C
:107F300002F0F0FD02F024FE00228D4B04000D0043
:107F400002F012F802000B003000390002F07EFA55
:107F500002F0E0FD4B4601C39946434620001A68F3
:107F60005B68290001F0DAF808235B429C46E04494
:107F700006000F00D045D5D1059B30001A0039000E
:107F8000984600F0DFFCFF2300229B0504000D0053
:107F900001F0EAFF00F038FC0022764B01F0E4FF2C
:107FA00002000B002000290002F050FA0D0004002E
:107FB00002F0B0FD814602F0E3FD02000B0020005C
:107FC000290002F043FA060040460F00002800DCBA
:107FD000EEE0009B18215A1E92000EAB9B58091A26
:107FE0001D000D41A9448D405D1B0EAB9D50172314
:107FF0001B1A1D41002D2DDD01239C46009BE144F1
:10800000002B00DC1CE20E9C0123002C00D0B5E00C
:10801000009A012A09D099000EAA54580133002C65
:1080200000D0ACE0009A9A42F5D1059B002B0EDD02
:10803000012B00D1A8E1022B09D1009B0EA95A1EE9
:1080400092000EAB9B5807939B029B0A8B50022D0C
:1080500000D1C1E0002300223000390000F08AFE88
:10806000009B002800D194E2069A591E8A4210DC37
:10807000414A0A9894460EAA6344944600229B0003
:1080800063441C68043B22438342FAD1002A00D097
:10809000C0E0069B0EAA013B9B00D358002B00D0EA
:1080A000B3E001220C9B043B596801320029FAD04D
:1080B000009B9C466244110007921A0001338B42D8
:1080C00046DC0B9863468046A59C4344A046099C29
:1080D0009B00A1464A449844D30022AA9146049AA0
:1080E00099449446089BA59A634484466144944607
:1080F0009A468B00634400934346586802F040FD63
:108100004B4618605960029B002B24DB4D46039CB4
:108110000026002701E0286869680CCC01F024FFE4
:1081200002000B003000390000F0F8FF083D0600A7
:108130000F005C45EFD153469E60DF6004239C46F0
:108140000433E0449C46009BE144E2449845D3D18B
:10815000079B0093D1E600260027ECE794FDFFFF84
:10816000B0D8000018FEFFFFFFFFFF1F0000703EA9
:108170000000704100002040FFFFFF3F00218022EF
:108180005204141B0EAA5450009999420EDD0EA8F9
:1081900084469B000EAA8900D25861446344CF48AC
:1081A00000E01A68821A04C38B42FAD101243CE72A
:1081B000059B002B06D1009B0EAA013B9B00D558C6
:1081C000ED1517E70022C64B300000F0F7FD002840
:1081D00000D024E100253DE732003B000020C149EA
:1081E00002F034F906000F00002C00D132E7059AA6
:1081F0000020BC4900F0A6FB02000B003000390053
:1082000002F024F906000F0024E7012250E70026BF
:10821000002754E64B46059A079388468B000EA923
:10822000CB58183A08950592002B0DD18C46414643
:10823000AD4B43449B006344043B58680139183AF2
:108240000028F9D088460592059A0020A54900F03B
:1082500079FB434604000D00002B00DA05E29E0086
:108260000EAB9C464346DB0066449C46059370ABD0
:108270009946049F67440097306802F081FC220011
:108280002B0001F071FE002238607960974B2000CE
:10829000290001F069FE083F04000D00043EB945C5
:1082A000EAD14AAB03939B4600239A46069B42467B
:1082B000994643460132029204934B46002B00DA62
:1082C000AAE080208A4B009D9846C0058949002677
:1082D0000027002408E008239C460835E044544564
:1082E00011DC4346186859682A686B6801F03CFE47
:1082F00002000B003000390000F010FF01340600CE
:108300000F00A145E7DA5B46C0C39B4601239C46AC
:10831000009BE244083B0093029B9A45CDD1049B0D
:108320009846A49B022B00DD8EE0002B37DC1FD18A
:10833000059B00271D00039B00249C461E006544EE
:10834000083E2A686B683800210000F0E7FE083D0F
:1083500007000C00AE42F4D1089B002B03D0802311
:108360001B069C4664443A0023000D990A604B604A
:108370000720079B18409B239B009D443CBC9046D4
:108380009946A246AB46F0BD009B0EA95A1E92002C
:108390000EAB9B5807935B025B0A8B5057E6434634
:1083A000002B00DA70E100200021DB004AAAD61879
:1083B00048AF32687368083E00F0B0FEB742F8D1AB
:1083C000089B002B00D025E10B0002004A984B9936
:1083D0000D9C2260636002F039F8434607000C00F0
:1083E000002B13DD01254CAEB14638002E002100D4
:1083F0004C4601360CCC00F091FEA146B045F7DAB0
:10840000089B07000C00002B00D015E13A00230068
:108410000D998A60CB60ABE70026002773E7012344
:108420009C46009BE1440225002B00DDEBE5320079
:108430003B0000202B4902F009F806000F0009E676
:108440000024F2E54AAB0393A49B032B00D08FE7F3
:108450004346002B00DC14E1039ADB009B4613002B
:1084600091465B441E685F68234B43440293DB00E4
:10847000994448AB9A464B465C681B68180021003B
:1084800032003B000090019100F048FE04000D0016
:1084900002000B000098019901F0D8FF3B00320068
:1084A00000F03CFE4B469860D9601C605D6008237C
:1084B0005B429C46E14426002F00CA45DBD143467F
:1084C000012B00DCE3E0039A13005B441E685F6845
:1084D000029BDB0099464A44904610E0FFFFFF00F4
:1084E0000000E03F0000F03FFFFFFF3F0000703E54
:1084F00070D80000FB21F93FFFFFFF1F984643465D
:108500005C681B681800210032003B00009001915C
:1085100000F004FE04000D0002000B000098019919
:1085200001F094FF32003B0000F0F8FD4346039A4F
:108530009860D9601C605D60083B26002F009A425D
:10854000DCD14D4694460026002447460835654454
:108550002A686B683000210000F0E0FD083D06004D
:108560000C00AF42F4D1039B4A9F5D689968D868BC
:10857000089B002B65D08022120694460D9B654413
:10858000604464441F605D609960D8601E615C61F6
:10859000EEE69A464B460793059B30005A42390057
:1085A000089500F0CFF900223A4B06000F0000F0CA
:1085B00005FC002824D0384B00223000390001F09F
:1085C000D3FC02F0A7FA52460400950002F0D8FA54
:1085D0000022304B01F0C8FC02000B0030003900D3
:1085E00001F034FF02F096FA0EAA50510122059BC9
:1085F000524418339046059393000EAAD45023E6B4
:108600005346300039009C0002F084FA0EAB18513A
:10861000D04619E680230D9A1B06CB1810605360D4
:108620000B0002004A984B9901F010FF43460700E7
:108630000C00002B00DDD5E680231B069C4664441D
:10864000E4E62B003A000D9D2A606B600A000300EF
:10865000AA60EB60320023002A616B6188E6099B07
:10866000DB00009372AB049332E4A49B022B00DD89
:10867000E8E6002B00DD92E600D079E60027002432
:108680006AE6002600246EE70020002198E6002616
:10869000340068E7000070410000703EF0B5CE463F
:1086A000474680B587B000920193474A4B00814608
:1086B00088465B08934207DC4146484602F02AFAA6
:1086C0004146031E484666D04A4643464846414610
:1086D00001F04AFC04000D0002000B004846414630
:1086E00001F042FC394A3A4B06000F0020002900F5
:1086F00001F03AFC374A384B01F0A8FE22002B006B
:1087000001F032FC354A364B00F008FD22002B0008
:1087100001F02AFC334A344B01F098FE22002B0072
:1087200001F022FC314B324A00F0F8FC0E9B029023
:108730000391002B34D00098019900222D4B01F0B9
:1087400013FC029A039B049005913000390001F05C
:108750000BFC02000B000498059901F077FE220043
:108760002B0001F001FC009A019B01F06FFE224AF0
:1087700004000D00214B3000390001F0F5FB020030
:108780000B002000290000F0C9FC02000B00484645
:10879000414601F05BFE07B00CBC90469946F0BD27
:1087A00002000B002000290001F0DEFB124A134BEF
:1087B00001F04CFE32003B0001F0D6FB4A46434636
:1087C00000F0ACFCE7E7C046FFFF3F3E7CD5CF5A48
:1087D0003AD9E53DEB9C2B8AE6E55A3E7DFEB15742
:1087E000E31DC73ED561C119A0012A3F1111813F88
:1087F000A6F810110000E03F495555555555C53FA5
:1088000049004B0819007047474AF0B54F4691465A
:108810004B005B0D99444646D6464A46C0B5050016
:108820000C000E0088460700132A27DC002A4BDBC9
:108830003E4B13419A460B0052461340034318D057
:108840003B4A3C4B2800210000F068FC002200233A
:1088500000F0AAFA002847D0002C04DA80234A4608
:108860005B03134198444646534600279E43380015
:1088700031001CBC90469946A246F0BD332A08DD63
:108880008023DB009945F4D102000B0000F046FC88
:10889000EFE7294A9446012263445242DA40924665
:1088A0000242E6D0224A234B2800210000F036FC89
:1088B0000022002300F078FA002815D0002C1EDBDF
:1088C000534646469F430FE0194A1A4B28002100A1
:1088D00000F024FC0022002300F066FA002803D0F8
:1088E000002C04DB0027002638003100C1E76400BB
:1088F000640825430027002DF6D0104EF4E74B46C0
:10890000142B0BD03422D21A012393405D19BD429F
:1089100008D201239C462F00E044D1E7133B9C463C
:10892000E044CDE72F00CBE701FCFFFFFFFF0F0086
:108930009C7500883CE4377EEDFBFFFF0000F0BF34
:10894000002070474B0070B55B0D14000A00002B2F
:108950001AD14B005B08034315D0234B002201F0D2
:1089600003FB224B9C422DDB0A004B005B0D363B88
:108970001F4DE318AB422ADC002B0DDD1D4C1B05FF
:1089800022401A43110070BD1B4DAB42F0D10200D2
:108990000B0000F0C3FBF6E71D00353519DA174B65
:1089A00002009C4209DD0B001548164900F032F820
:1089B000134A144B01F0D8FAE5E70B0012481349AB
:1089C00000F028F8104A114B01F0CEFADBE7020064
:1089D000E9E7084C363322401B05134319000022F7
:1089E0000B4B01F0C1FACEE700005043B03CFFFF53
:1089F000FE070000FFFF0F80FF07000050C30000CC
:108A00009C7500883CE4377E59F3F8C21F6EA501BF
:108A10000000903C30B54A00DB0FDB0752081A43D8
:108A2000110030BD02B4714649084900095C490093
:108A30008E4402BC7047C04603B4714649084000EA
:108A40004900095A49008E4403BC7047002243087C
:108A50008B4274D303098B425FD3030A8B4244D306
:108A6000030B8B4228D3030C8B420DD3FF22090248
:108A700012BA030C8B4202D31212090265D0030B07
:108A80008B4219D300E0090AC30B8B4201D3CB03FD
:108A9000C01A5241830B8B4201D38B03C01A52413F
:108AA000430B8B4201D34B03C01A5241030B8B4241
:108AB00001D30B03C01A5241C30A8B4201D3CB022C
:108AC000C01A5241830A8B4201D38B02C01A524111
:108AD000430A8B4201D34B02C01A5241030A8B4214
:108AE00001D30B02C01A5241CDD2C3098B4201D32C
:108AF000CB01C01A524183098B4201D38B01C01AAA
:108B0000524143098B4201D34B01C01A5241030920
:108B10008B4201D30B01C01A5241C3088B4201D3CF
:108B2000CB00C01A524183088B4201D38B00C01A7C
:108B3000524143088B4201D34B00C01A5241411AA3
:108B400000D20146524110467047FFE701B50020B0
:108B500000F0F0F802BDC0460029F7D076E7704774
:108B600003460B437FD4002243088B4274D303098E
:108B70008B425FD3030A8B4244D3030B8B4228D32F
:108B8000030C8B420DD3FF22090212BA030C8B4255
:108B900002D31212090265D0030B8B4219D300E0F5
:108BA000090AC30B8B4201D3CB03C01A5241830B7A
:108BB0008B4201D38B03C01A5241430B8B4201D32A
:108BC0004B03C01A5241030B8B4201D30B03C01A53
:108BD0005241C30A8B4201D3CB02C01A5241830ACD
:108BE0008B4201D38B02C01A5241430A8B4201D3FC
:108BF0004B02C01A5241030A8B4201D30B02C01A26
:108C00005241CDD2C3098B4201D3CB01C01A52418C
:108C100083098B4201D38B01C01A524143098B4215
:108C200001D34B01C01A524103098B4201D30B01FE
:108C3000C01A5241C3088B4201D3CB00C01A524123
:108C400083088B4201D38B00C01A524143088B42E8
:108C500001D34B00C01A5241411A00D20146524181
:108C6000104670475DE0CA0F00D04942031000D3A0
:108C70004042534000229C4603098B422DD3030AF5
:108C80008B4212D3FC22890112BA030A8B420CD305
:108C9000890192118B4208D3890192118B4204D32E
:108CA00089013AD0921100E08909C3098B4201D3AE
:108CB000CB01C01A524183098B4201D38B01C01AE8
:108CC000524143098B4201D34B01C01A524103095F
:108CD0008B4201D30B01C01A5241C3088B4201D30E
:108CE000CB00C01A524183088B4201D38B00C01ABB
:108CF0005241D9D243088B4201D34B00C01A524192
:108D0000411A00D20146634652415B10104601D31E
:108D10004042002B00D54942704763465B1000D3A8
:108D2000404201B5002000F005F802BD0029F8D04E
:108D300016E770477047C046D0400B1C1141203ADF
:108D400003D49C4613411843634652429340184350
:108D50007047C0468446101C62468C46191C634608
:108D600000E0C0461FB501F097F8002801D40021AB
:108D7000C8421FBD10B500F0EFFF4042013010BDEA
:108D800010B501F089F8002801DB002010BD01209A
:108D900010BDC04610B501F07FF8002801DD0020AD
:108DA00010BD012010BDC04610B501F011F800281B
:108DB00001DC002010BD012010BDC04610B501F03F
:108DC00007F8002801DA002010BD012010BDC046C0
:108DD000F0B5CE46474615042D0C2E0080B507048D
:108DE000140C3F0C9946030C7E435D436743634379
:108DF0007F19340CE4199C46A54203D980235B02F9
:108E00009846C4444B4643435143250C36046544BD
:108E1000360C2404A4195B19591820000CBC904688
:108E20009946F0BDF0B54E4657464546DE46E0B59C
:108E300043025B0A450083B00F1C99462D0EC60FF6
:108E4000002D57D0FF2D24D08020DB00C004184314
:108E5000002381469A469B467F3D7C027A00FB0FA9
:108E6000640A120E984623D0FF2A4BD0E3008024D8
:108E70000020E4047F3A1C43AD186B1C4746019365
:108E8000534677403A000F2B48D87D499B00CB587A
:108E90009F46002B00D085E008339A46063B9B4650
:108EA0007C027A00FB0FFF25640A120E9846DBD184
:108EB000002C00D090E0524601231A439246012034
:108EC000DBE74C4658461700022824D0032800D17F
:108ED000CFE00022002301284DD15802D205400ADC
:108EE000FF071043384303B03CBC90469946A24666
:108EF000AB46F0BD002B5BD104239A46033B002513
:108F00009B46AAE7FF35002C60D1524602231A4344
:108F100092460220B1E7FF220023DEE74B461B0CFE
:108F20009C464B462604360C180461463300220C3E
:108F30006446000C43434E435043544380191A0C7B
:108F40001218964203D9802149028C4664441B04BE
:108F50001B0C1004C01883015E1EB341800E184321
:108F6000130C1B199B0103431C00230179D501231A
:108F700062081C401443019A7F32002A4DDD6307CA
:108F800004D00F232340042B00D00434230103D545
:108F90003C4B019A1C408032FE2ABCDCA3015B0AD8
:108FA000D2B29AE70C239A46093BFF259B4654E729
:108FB000180001F071FE4A46431F76259A400023AF
:108FC0006D4291462D1A9A469B4646E75246032328
:108FD0001A439246032050E7200001F05DFE431F34
:108FE0002D1A9C40763D002047E780230027DB03B5
:108FF000FF2272E7424666E74C463200584662E777
:1090000080234A46DB031A4222D01C4220D123434C
:109010005B025B0A4746FF225FE701239A1A1B2A7D
:1090200021DC23000199D3409E318C401A0023009B
:109030005C1EA34113435A0704D00F221A40042A8E
:1090400000D004335A0111D49B015B0A002244E78B
:1090500080234A46DB0313435B025B0A3700FF228F
:109060003BE7019587E70022002336E70122002332
:1090700033E78023DB0323435B025B0AFF222CE7F9
:10908000C0D80000FFFFFFF770B500283DD0C31720
:10909000C5185D40C40F280001F0FEFD9E22121A83
:1090A000962A07DCD2B2082833DD083885406802EA
:1090B000400A23E0992A0BDD052329001B1AD94019
:1090C00003001B339D402B005D1EAB4119430D0077
:1090D000052801DD431F9D402B000F490B406E0703
:1090E00009D00F263540042D05D004335D0102D58B
:1090F0009F220B40121A9B01580AD2B24002D2059D
:10910000400AE4071043204370BD002400220020E1
:10911000F4E76802400AF1E7FFFFFFFBF0B54F46B6
:109120004646D6460C000903C0B5490A470F5E0003
:1091300039431F03DB0F9C4665007B0A570F1F4313
:109140006D0DE40F760DA146C000B846D200AB1BF2
:1091500064457BD0002B5FDD002E00D0A4E03E00F4
:10916000164300D112E15E1E002E00D09EE1871A48
:109170004346B84280410125C91A4042091A0B02F0
:1091800000D431E149024E0A002E00D16EE13000D8
:1091900001F082FD0300083B1F2B00DD61E120226E
:1091A0003900D21A9E40D1409F400E439D4200DDBF
:1091B00051E15D1B6B1C1F2B00DD7CE12021C91AD6
:1091C0003D0030008F408840DD40791E8F413100E6
:1091D00007222843D940002507433A40002A09D0F6
:1091E0000F233B40042B05D03B1DBB42BF417F42B8
:1091F000C9191F000B0200D426E26A1CC64B550594
:109200006D0D9A4200D106E1C44AFF080A40530797
:1092100052023B43120B8EE0002B00D0B8E06B1CD7
:109220005B055B0D012B00DC30E1871A4346B84239
:10923000B641CB1A76429E1B330200D54CE13B006F
:109240003343A1D100220024002570E0002B00DC74
:10925000E5E0002E00D183E0AF4EB54260D080261D
:1092600036043743B846382B00DC3EE1434613430F
:109270001F007A1E97413F188742804140420918DB
:109280000B0200D4B0E0A44B01359D4200D1C3E0F5
:10929000A24A7B080A4001210F401F435108D3070F
:1092A00007221F433A4099E79B4EB54238D08026AB
:1092B00036043743B846382B00DDDCE01F2B00DCDA
:1092C00030E11E004746203EF740BC46202B04D02C
:1092D0004026F31A46469E403243170063467A1EE4
:1092E00097411F43CCE0002B00D104E243461343D7
:1092F00000D159E14B07C00818438023C9081B035C
:10930000194208D04546ED081D4204D14346D00815
:10931000590708432900420FC9007F4D1143C0007F
:109320004B07CA087C49C00803438D4268D012032A
:109330006D05120B6D0D002112031800130B0A0DA1
:1093400012051A43764B2D0513402B435B00E407AF
:109350005B08234319001CBC90469946A246F0BD09
:109360003E00164312D05E1E002E00D000E187188A
:109370008742804141444042091801250B0233D500
:10938000022585E764463300414610001D00C7E70B
:10939000002D00D0DAE00C000443F3D05C1C00D1B7
:1093A0009FE15D4CA64200D12FE1DB43382B00DD6D
:1093B00066E11F2B00DD83E120240500E41A0F0085
:1093C000DD40D940A0404346A7405B1A441EA0415F
:1093D00098462F433843171ABA42924143465242A5
:1093E000991A64463500CAE607223A40002A00D09E
:1093F000F6E64B07CA084849FF083B438D4296D121
:109400001900114300D19EE1802109030A43120390
:10941000120B414D8FE71500002200238BE7002B34
:1094200000D0C7E06B1C5F057F0D012F00DCF1E071
:10943000394DAB4200D1B9E085180A008542894117
:109440004244494251180722CF076D082F4349086B
:109450003A401D00C2E607223049ED1A31403A4039
:10946000BCE63E002838864000279FE6380001F021
:1094700013FC20308EE6434613431F007A1E9741AB
:10948000C71BB84280414042091A78E60E003B00F3
:1094900006431343002D61D1002E00D0F4E0002BD1
:1094A00000D11BE164463900100039E71A4FBB4276
:1094B0007AD03300FFE630001F3DE840202B03D078
:1094C0004021CB1A9E4037437B1E9F410722074312
:1094D0003A400021002589E7171A4346BA42B641AF
:1094E000591A76428E1B64464EE61F2B00DDADE016
:1094F00020264746F61AB740B9461700B246DF4065
:109500004E463E4337005646B240561EB2411743C0
:109510004246DA408918AEE6FF070000FFFF7FFFF2
:10952000FFFF0F8020264746F61AB740B9461700BE
:10953000B246DF404E463E4337005646B240561EC6
:10954000B24117434246DA40891A99E77F4CA64256
:109550005BD0802424045B42214327E7002E0CD1FA
:10956000002B00D1CBE0644639001000774DD7E6E0
:10957000764FBB4218D0330075E6002B14D04B0752
:10958000C00818438023C9081B03194207D0FC08F0
:109590001C4204D17907D0080843E14621004C461B
:1095A000420FC9001143C000684DB9E61D000022FA
:1095B0000023C0E6002D5BD10D00054300D1E2E69B
:1095C0005D1C00D1B0E0614DAE421FD0DB43382BB3
:1095D00071DC1F2B00DD96E020250F00ED1AAF4057
:1095E000B9460700AA46DF404D463D432F00554689
:1095F000A840D940451EA84188440743BF18974258
:1096000092415142414435003AE6644635004146B4
:10961000100085E60B000343002D00D063E6002B0D
:10962000F5D04346134300D17AE68718874280413C
:1096300007224144404209183A400B0200D4D5E6C3
:10964000434B01351940C9E5380069E61E0047461D
:10965000203EF740BC46202B04D04026F31A464655
:109660009E403243170063467A1E97411F4302E62D
:10967000364DAE42CAD080252D045B422943A6E771
:109680000843411E8841A6E6002B00D148E6871A10
:109690004346B842B641CB1A76429E1B33024BD5A5
:1096A000171A4346BA429241591A5242891A07225E
:1096B00064463A4092E501430F00791E8F419DE7D1
:1096C0001C000F00203CE740202B03D04024E31A6D
:1096D00099400843411E884138437CE6002200241B
:1096E00025E6171A4346BA429241591A5242891A3C
:1096F0006446350043E541461000144D10E68022D3
:109700000024120380E61D000F00203DEF40BC4600
:10971000202B03D04025EB1A9940084307006346ED
:10972000781E87411F4369E7871897429B41414450
:109730005B42C9183500A3E53B003343CED0072276
:1097400031003A4052E600231A00F4E5FF0700001A
:10975000FFFF7FFFF0B55746DE464E464546E0B573
:10976000834607000E03480085B092461C00360B66
:10977000400DCD0F002800D19DE0954B984239D087
:109780008023F6001B041E43924A7B0F3343994605
:10979000944603006344009300230026FF000293D5
:1097A00023031B0B98466300E40F52465B0D0194A4
:1097B00000D1B3E086498B4200D19EE04246D10001
:1097C000802212040A435146490F11438B468149B6
:1097D00052468C4600996344CB1A0021D200009374
:1097E0002B0063409A460F2E00D905E17A4BB60054
:1097F0009B599F465B463343994600D0B8E002230D
:109800000826002700900293CAE7CB463A00029947
:109810000195019B9A46022927D0032900D180E2B5
:10982000012944D06D49009B8C4663441C00002CE8
:1098300038DD530700D013E2D2085B46DB0109D5BF
:109840005946674B19408B468021C9008C46009BC6
:1098500063441C00634B9C4207DC5B4664055F0766
:109860005B0217431B0B620D02E000230027584ADE
:1098700000211B031C0B0B0D1B05234314055A4A27
:10988000380013401C4353466400DB0764081C4344
:10989000210005B03CBC90469946A246AB46F0BDBF
:1098A0000122524201231B1B382B00DCADE10022B8
:1098B00000230027DCE75B46334399465ED0002E49
:1098C00000D18AE1300001F0E7F903000B3B1C2BCB
:1098D00000DD7BE11D22D31A5A460100DA40083927
:1098E0008E4013005F46334399468F403F4B00261E
:1098F0001B1A00930023029352E7414653460B4341
:109900003B499B468C46009B634400935B46002B7F
:109910003BD1022300221E43022161E74346134349
:109920009B4637D04346002B00D162E1404601F010
:10993000B3F903000B3B1C2B00DD53E10200414651
:10994000083A914088461D21CB1A5146D9400B0058
:1099500041460B439B46534693401A00009B2549C2
:109960009C46604403008C4663440093002137E723
:109970000323B14600900C26029311E700230093C5
:1099800001330426002702930AE70323C3461E433C
:10999000032125E701331E430022012120E7002394
:1099A0009A46802300271B03094A61E78023494622
:1099B0001B03194200D1E2E05946194200D0DEE013
:1099C0000B431B0317001B0BA246014A50E7C0467E
:1099D000FF07000001FCFFFF00D90000FF030000AB
:1099E000FFFFFFFEFE070000FFFF0F800DFCFFFFE3
:1099F00001F8FFFFF3030000D94500D9CBE000D107
:109A0000C6E03C0048460027009B013B00935B46B4
:109A1000160E1B021E431302984633041B0C994674
:109A2000310C0191FFF798F84A4642430B04210C90
:109A3000050019438A4207D98919013D8E4203D88E
:109A40008A4201D9851E8919881A0199FFF784F87D
:109A500009048C464A46210464464243090C03002B
:109A600021438A4204D98919013B8E4200D8F1E092
:109A70002D041D43AB464346891A4246280C120466
:109A80001D0C5B46140C22001B041B0C5A43039450
:109A90006B434443029568431B19150CEB189C4219
:109AA00003D980246402A44660441C0C15041B04E2
:109AB0002D0C20185D19814277D373D00C1AA24A5D
:109AC0007D1BAF42BF419446009B7F426344E01B35
:109AD0001C00864200D1DBE00199FFF73DF84A46C1
:109AE00042430B04290C070019438A4207D98919FC
:109AF000013F8E4203D88A4201D9871E8919881AEC
:109B00000199FFF729F809044A46894629044D4678
:109B10004243090C030029438A4207D98919013BB2
:109B20008E4203D88A4201D9831E89193F04891ABB
:109B30003A00039F1A43380013041B0C5843814614
:109B40000298150C6F43434345434846000C844636
:109B5000DB1963449F4203D9802040028446654458
:109B600048461F0C00041B04000C7D191818A9425C
:109B700000D284E000D17FE001231A4357E680231E
:109B80004A461B0313431B031B0BAA466F4A6FE68F
:109B9000BA4200D935E74B46DC0758087B081C431E
:109BA000FF0734E70024AF4289D247444745A44128
:109BB0005B466442A4196418013BA6421ED2A0422F
:109BC0006DD800D1B6E0241A9B4678E703005A46C8
:109BD000283B9A400027914688E6584601F05CF8F9
:109BE000203072E603005246283B9A4093460022FA
:109BF000B4E6504601F050F820309AE6A642E2D191
:109C0000B845DCD9341A9B4659E71F2B65DC504C0C
:109C10000099A4465C46614408008C4011008240D3
:109C2000D940501E82410C4314435A46DA40130077
:109C3000620709D00F222240042A05D02200141DF9
:109C40009442894149425B181A0262D501220023DD
:109C500000270DE68A4200D80AE7831E891907E724
:109C60000F231340042B00D1E6E5171D97429241C4
:109C700053429B44FA08E0E5002800D1D7E571186B
:109C8000531EB14227D3A94215D358D01A0073E707
:109C9000002B00DC04E6012300229B44CDE50223D7
:109CA0004744474589415B429C46494289190C1902
:109CB000E344241A03E743465F0047459B41B84607
:109CC0005B429E19023A8919A94200D054E74045E7
:109CD00000D051E7ABE51A00F6E71F215F46494285
:109CE0000C1BE740202B07D01A49009B8C4663448D
:109CF00018005B4683401A43501E82413A430727AF
:109D00000023174009D00F2100231140140004291B
:109D100095D122005F075B021B0BD208174300227C
:109D2000A6E5802359461B030B431B0317001B0B9F
:109D3000064A9DE5BD42B2D89B460024BFE6804559
:109D4000B9D31A00C3E7C046FF030000FF070000B5
:109D50001E0400003E040000F0B54F464646D646BD
:109D60008446C0B58046194E18030F034D00000B02
:109D70005C0082463F0B6D0DC90F9146640DDB0FF1
:109D80000120B5420AD0B44203D0A54201D15745C3
:109D90000CD01CBC90469946A246F0BD66463E4398
:109DA000F7D1AC42F5D154461443F2D10120C84555
:109DB000EFD1994207D0002DEBD163461F43380005
:109DC000471EB841E5E70020E3E7C046FF07000073
:109DD000F0B54F464646D6464D00C0B50E03C90FF6
:109DE0008A462C491F035C008046360B6D0D914658
:109DF0003F0B640DDB0F8D421ED08C4216D0002D20
:109E00001ED130438446002C01D13A4323D0624610
:109E1000002A1AD09A4529D051460220013908401B
:109E200001381CBC90469946A246F0BD390011434A
:109E3000E5D002204042F4E73043FAD1AC420FD0E3
:109E4000002C0FD13A43E7D00CE00122013B9343B1
:109E500018000130E5E763460020002BE1D0DBE786
:109E60003A43E6D19A45D7D1A542D5DCA54205DBD8
:109E7000BE42D1D808D00020BE42D2D250460123E3
:109E8000013898430130CCE7C845C5D80020C84503
:109E9000F4D3C6E7FF070000F0B54F464646D64666
:109EA0004D00C0B50E03C90F8A462E491F035C0042
:109EB0008046360B6D0D91463F0B640DDB0F8D42D6
:109EC00018D08C4211D0002D18D130438446002C7C
:109ED0001ED13A431CD163460020002B30D051469E
:109EE00002200139084001382AE039001143EAD044
:109EF000022025E03043FBD1AC4226D0002C26D1F5
:109F00003A4324D15146022001390840013817E074
:109F10006246002A0FD09A45E1D1A54205DBBE4238
:109F2000DDD819D00020BE420AD2504601230138A4
:109F30009843013004E00122013B934318000130B3
:109F40001CBC90469946A246F0BD3A43D0D19A45F2
:109F5000C5D1A542C3DCE0E7C845C0D80020C8454C
:109F6000E3D3EDE7FF070000F0B55746DE464E4667
:109F70004546E0B5834606000F03480087B0924689
:109F80001D003F0B400DCC0F002800D16FE0DE4BD1
:109F9000984238D08023FF001B041F43730F3B43BC
:109FA0000193DA4B0027994600239B46F600814433
:109FB0002B0369001B0B52469846490DED0F0029F3
:109FC00000D185E0D04B994200D173E04346DA00DE
:109FD00080231B0413435246CC48520F844613433C
:109FE000524600206144D20089442100694000911A
:109FF0008C46012149448A460F2F00D990E0C4497C
:10A00000BF00CF59BF465B463B43019300D06AE196
:10A0100002230827002681469B46C9E7320058469E
:10A02000019B61460091022800D175E0032800D110
:10A03000FEE1012800D02CE10023002700260025A6
:10A040003F032A0D3F0BB34812053A4302401B055C
:10A050001343009A5B00D1075B080B4330001900E3
:10A0600007B03CBC90469946A246AB46F0BD5B4665
:10A070003B43019300D12FE1002F00D1A5E138002F
:10A0800000F00AFE03000B3B1C2B00DD96E11D22B5
:10A09000D31A5A460100DA405E4608398F40130051
:10A0A0008E403B4301939C4B00271B1A994600238B
:10A0B0009B467DE7414653460B4393498C46E1441A
:10A0C000002B00D01AE102220220174300228CE765
:10A0D000134300D10DE14346002B00D181E14046FE
:10A0E00000F0DAFD02000B3A1C2A00DD72E10100EB
:10A0F000434608398B4098461D239A1A5346D3404D
:10A100001A004346134352468A404946081A824978
:10A1100089468144002068E77B4B002700268EE7B4
:10A12000140C1204120C1100370C3604350C794350
:10A1300028008C462E00604360448346564321002D
:10A14000300C80465846794340440291844506D9F4
:10A150008846802149028C46E044414602913604FB
:10A16000010C360C00048B4681191E0C1B041B0CC1
:10A170000391190079438C46280075436544A8462D
:10A180005843050C45447743A94203D9802149022D
:10A190008C466744290C8C4639000004000C2D04C1
:10A1A0002D186144AB4405915946049101990F045F
:10A1B0003F0C080C390051434243904602008C4644
:10A1C000090C8B4662437C4344445C44A04503D95C
:10A1D0008021490288464244210C88466146090490
:10A1E000090C8C4639005943434370437E430F0C9E
:10A1F000F6182404BE19644442448C46B34203D981
:10A2000080235B0298464044029B61469846049B2B
:10A21000370443449B46AB45AD416B420D04059961
:10A220002D0C8C467F196744FD18A8465D462D19F4
:10A23000A542A44193466442A446C344DC448F42F1
:10A24000BF4198459B4193459241A445A4415B423F
:10A250007F421F43360C52426442BF192243BF184B
:10A26000624638184302D20D039913436A020A4327
:10A27000501E82416146ED0D2A434E023243D90100
:10A2800000D4B3E00126500832400243DE073243D7
:10A290005B08224C5444002C62DD510709D00F208A
:10A2A0001040042805D0101D9042924152429B1844
:10A2B0000200D90104D580241948E4000340544425
:10A2C0001848844200DD27E75E075B02D2081F0BB7
:10A2D000630516435B0DB2E600239946013304275C
:10A2E00000269B4664E60323019781460C279B4684
:10A2F0005EE6012201201743002276E603230320B5
:10A300001F43434671E6C046FF07000001FCFFFF04
:10A3100040D90000FFFF0F800DFCFFFFFF0300008E
:10A32000FFFFFFFEFE0700000023802700933F038E
:10A330000026434B83E6019B3200A446584670E654
:10A34000AC466EE6802701993F0339422DD03B424F
:10A350002BD11F433F033F0B00951600384B6EE691
:10A3600001252D1B382D00DD66E61F2D40DC35480C
:10A370001C005044160082408440EE40501E824132
:10A3800034431443EB40620709D00F222240042AD1
:10A3900005D02200141D9442804140421B181A022D
:10A3A0003ED501230027002649E68027019B3F0375
:10A3B0001F433F033F0B0094214B40E603005A46E6
:10A3C000283B9A40002601926DE6584600F064FC56
:10A3D000203057E603005246283B9A4013000022E3
:10A3E00093E6504600F058FC20307BE6CA4650E722
:10A3F0001F201E004042041BE640202D03D0124CBB
:10A400005444A3401A43501E82413243072600277A
:10A41000164009D00F200023104014000428B9D1A1
:10A4200022005E075B021F0BD2081643002306E6DC
:10A4300080273F031F433F033F0B1600004BFEE501
:10A44000FF0700001E0400003E040000F8B5574658
:10A450004E464546DE460C000903E0B5490A460F64
:10A460005F0031431E03DB0F760A9B46530F3343D5
:10A47000C84E6500C000E40FD2006D0DA2468146B3
:10A480007F0D9C469046B74200D1B9E05B4601265D
:10A4900073409B46EE1BA34500D183E0002E63DD95
:10A4A000002F00D0B1E06346134300D123E1731EB7
:10A4B000002B00D0BAE1861A6346B04280410125E4
:10A4C000C91A4042091A0B0200D447E149024B0A5B
:10A4D00098464346002B00D189E1404600F0DCFB62
:10A4E0000300083B1F2B00DD7CE120223000D21A44
:10A4F0004146D040994002009E400A439D4200DD03
:10A500006AE15D1B6B1C1F2B00DD94E12021100014
:10A510003500C91A8E40DA408840DD40711E8E41F8
:10A52000110007222843002506433240002A09D0A3
:10A530000F233340042B05D0331DB342B64176427E
:10A5400089191E000B0200D43DE26A1C914B55058F
:10A550006D0D9A4200D119E18F4AF6080A4057075B
:10A5600052023743120B9BE0002E00D0C5E06E1C58
:10A570007605760D012E00DC48E16746861ACB1B76
:10A58000B042BF417F42B8461F004346FF1A3B001E
:10A59000B8461B0200D55FE137439AD10022002460
:10A5A000002579E0002E00DCFAE0002F00D18DE0DC
:10A5B000784B9D4267D0802367461B041F43BC46EF
:10A5C000382E00DC52E1634613435A1E93411E1895
:10A5D00086428041404209180B0200D4BEE06D4B18
:10A5E00001359D4200D1D2E06B4A73080A40012137
:10A5F0000E401E435108D30707221E43324095E701
:10A600001E00164300D045E740E7624B9D423AD01A
:10A61000802367461B041F43BC46382E00DDEBE059
:10A620001F2E00DC3AE133006746203BDF403B0051
:10A63000202E05D04027BF1B6646BE4032439046C1
:10A640004646721E96413343DAE0002B00D114E2F5
:10A650006346134300D168E180234E07C008C90850
:10A660001B030643194208D06046C008184204D1B3
:10A6700063460100D2085E071643F3009946C900FD
:10A68000720F444D11434B46DE08424B4F07374390
:10A69000CA089D4200D16EE012036D05120B6D0DCC
:10A6A00000211203130B0A0D12051A433B4B2D0513
:10A6B00013402B435B00E4075B0823433800190079
:10A6C0003CBC90469946A246AB46F8BD6346134350
:10A6D00011D0731E002B00D007E1861886428041FE
:10A6E00061444042091801250B0237D502257BE75A
:10A6F0003E00614691463500C5E75C46002D00D01E
:10A70000E1E00B000343F3D0731C00D1ACE1214B1B
:10A710009F4200D13AE1F343382B00DD6FE11F2B5C
:10A7200000DD8CE120250E00ED1AAE40B04606009B
:10A73000AA46DE40454635432E005546D940A8403E
:10A740006346451EA8415B1A9C463043161AB24226
:10A75000924163465242991A3D00B4E607223240C4
:10A76000002A00D0E4E60B4BF6084F073743CA082F
:10A770009D4200D090E73B00134300D1A6E1802327
:10A780001B031A431203120B024D89E71500002226
:10A79000002785E7FF070000FFFF7FFFFFFF0F8017
:10A7A000002E00D0C7E06B1C5E05760D012E00DC8C
:10A7B000F0E0C84DAB4200D1B9E085180A008542EF
:10A7C00089416244494251180722CE076D082E4341
:10A7D000490832401D00A9E6BF49ED1A1140072281
:10A7E0003240A3E6320028388240002686E6300058
:10A7F00000F052FA203073E6634613435A1E934129
:10A80000C61AB04280414042091A5CE60E00674613
:10A8100006431743002D5ED1002E00D0F3E0002F39
:10A8200000D11EE15C46614691462CE7A94FBE422D
:10A830007BD01E00F1E610001F3DE840202B03D026
:10A840004021CB1A9A401643731E9E4107220643AD
:10A8500032400021002583E7161A6346B242804148
:10A86000591A40420B1A98465C4632E61F2E00DD0C
:10A87000ABE02027BB1B9A4663465746BB40994630
:10A8800013004F46F3401F433B005746BA40571E44
:10A89000BA4113436246F240891898E62027BB1B51
:10A8A0009A4663465746BB40994613004F46F340CD
:10A8B0001F433B005746BA40571EBA4113436246F6
:10A8C000F240891A9CE7834B9F425FD080252D047C
:10A8D0007342294320E7002E0CD1002F00D1D0E095
:10A8E0005C46614691467B4DCDE67A4FBE421CD018
:10A8F0001E0065E6002F18D0C0084E0706438020D2
:10A90000C9080003014208D06346DC08044204D1B0
:10A910002100DA46D2085E071643F3009946012467
:10A920005346C900720F11431C406A4DABE61D002F
:10A9300000220027B4E6002D59D10B00034300D1BB
:10A94000D6E6731C00D1B2E0624B9F421ED0F343A7
:10A95000382B6FDC1F2B00DD97E020250E00ED1A51
:10A96000AE40B0460600AA46DE40454635432E00BE
:10A970005546A840D940451EA8418C440643B61808
:10A9800096429241514261443D0025E63D006146B8
:10A99000914678E60B000343002D00D055E6002BCE
:10A9A000F5D06346134300D16DE686188642804198
:10A9B00061444042091800220B0200D4D0E6464B05
:10A9C00001351940B2E5B1465DE633006746203BEC
:10A9D000DF403B00202E05D04027BF1B6646BE400F
:10A9E000324390464646721E96413343EFE5394B5B
:10A9F0009F42CBD080252D0473422943A8E708430A
:10AA0000411E8841A2E6002F00D13CE66346861A2B
:10AA1000CF1AB0429B415B42FB1A98461B024ED5AF
:10AA2000161A6346B2429241591A5242891A5C463A
:10AA300000227BE501430E00711E8E419FE71D0041
:10AA40000E00203DEE40B046202B04D04025EB1AEE
:10AA500099400843814648464346411E8841184371
:10AA600074E60022002417E6161A6346B2429241A9
:10AA7000591A5242891A3D0025E561469146154D05
:10AA800001E680220024120379E61D000E00203D1D
:10AA9000EE40B046202B04D04025EB1A99400843E5
:10AAA00081464E464346711E8E411E4367E7861817
:10AAB00096429B4161445B42C9183D008CE5474684
:10AAC0003743CED007224146324049E600273A00BC
:10AAD000E6E5C046FF070000FFFF7FFF70B50C4EA4
:10AAE0000D031C0349005B002D0B490D240B5B0D6E
:10AAF000B14208D0064900208B4203D11443200004
:10AB0000441EA04170BD05430120002DFAD1F1E79C
:10AB1000FF07000030B5144D0A034B00120B5B0D0C
:10AB2000C90F0024AB4211DD104CA34210DC80247D
:10AB3000640322430E4CE41A1F2C0CDD0D48C31A8B
:10AB4000DA4013005C42002900D11C00200030BD17
:10AB5000094BCC18FAE7094DE040AC4663449A40F3
:10AB600013000343EEE7C046FE0300001D0400008F
:10AB70003304000013040000FFFFFF7FEDFBFFFF25
:10AB800070B500282DD0C317C5185D40C40F28002C
:10AB900000F082F8154B1B1A5B055B0D0A2815DDCA
:10ABA0000B38854000222D032D0B002110002D03B2
:10ABB0000A0D2D0B12052A430D4D1B052A40134388
:10ABC0005B00E4075B082343190070BD0200290005
:10ABD000153291400A000B21081AC5402D032D0B98
:10ABE000E3E70024002300250022DEE71E04000026
:10ABF000FFFF0F804100090E4B1C70B5DBB246020F
:10AC0000750AC40F012B14DDE0239B006D07360B82
:10AC1000CB1800210A0D280012051C4D32435B059C
:10AC20002A405B0813435B00E4075B0823431900D9
:10AC300070BD002914D1002D1ED0280000F02CF882
:10AC40000A281CDC0B232A001B1ADA4003001533E8
:10AC50009D400F4B12031B1A5B05160B5B0DD8E7CB
:10AC6000002D06D0320B802636036D071643094BA4
:10AC7000CFE7084B0026CCE700230026C9E70300F6
:10AC80002A000B3B9A400025E3E7C046FFFF0F80F8
:10AC900089030000FF0700001C2101231B049842C8
:10ACA00001D3000C10391B0A984201D3000A08395D
:10ACB0001B09984201D30009043902A2105C401814
:10ACC0007047C046040302020101010100000000B8
:10ACD0000000000030B51C00094B05001B6885B062
:10ACE000D868084B002A01D1074B1A000292019341
:10ACF00000912B002200054900F026F800F0A6FD87
:10AD00007C00002080D90000D6C700008DD900004B
:10AD1000014B18687047C0467C000020084B10B5F6
:10AD20000400002B02D0002100E000BF054B186892
:10AD3000836A002B00D09847200001F05DFBC046DD
:10AD400000000000BCD900000EB403B5010003AB45
:10AD5000044804CB0068019300F076F802B008BC08
:10AD600003B018477C00002070B500260C4D0D4C38
:10AD7000641BA410A64209D1002601F03FFB0A4D36
:10AD80000A4C641BA410A64205D170BDB300EB5859
:10AD900098470136EEE7B300EB5898470136F2E7E3
:10ADA0004C0200204C0200204C0200205C020020DB
:10ADB000002310B59A4200D110BDCC5CC4540133BD
:10ADC000F8E710B5884202D98B18984203D30023C4
:10ADD00007E08B5C8354013AFBD210BDCC5CC454B9
:10ADE00001339A42FAD1F8E703001218934200D1D6
:10ADF000704719700133F9E7936810B5013B936010
:10AE0000002B04DA9469A34207DB0A2905D01368F2
:10AE1000581C10601970080010BD00F04BFC0100B8
:10AE2000F9E7F8B506000F001400D518AC4201D1BF
:10AE3000002007E021783A003000FFF7DDFF013401
:10AE4000431CF3D1F8BD0000F0B59FB002900F0095
:10AE500016000593002805D083690493002B01D1C7
:10AE600000F0F4FD7B4B9F425BD1029B5F68BB8986
:10AE70001B0762D53B69002B5FD0002306AC6361E2
:10AE8000203363761033A37635002B78002B01D066
:10AE9000252B5CD1AB1B04930CD0320039000298F7
:10AEA000FFF7BFFF431C00D1C4E06269049B9446D6
:10AEB000634463612B78002B00D1BBE001220023A7
:10AEC0005242626002A9543252186E1C2360E36041
:10AED000A3601370A365317805225F4800F0D4FEAB
:10AEE000751C002835D12268D30604D5532302A946
:10AEF0005B1820211970130704D5532302A95B188E
:10AF00002B21197033782A2B2CD0350000210A20F0
:10AF1000E3682A786E1C303A092A64D900292ED0B9
:10AF200026E04E4B9F4202D1029B9F689FE74C4B0D
:10AF30009F429CD1029BDF6899E73900029800F09C
:10AF40000FFC002899D0012040421FB0F0BD013510
:10AF50009BE7414B2268C01A0123834013432360BF
:10AF60002E00B8E7059B191D1B680591002B01DB1E
:10AF7000099304E05B42E3600223134323602B78D0
:10AF80002E2B0AD16B782A2B35D1059B02351A1D41
:10AF90001B680592002B2BDB0793324E2978032286
:10AFA000300000F071FE002806D04023801B834053
:10AFB0002268013513432360297806222A486E1C33
:10AFC000217600F061FE00283AD0284B002B25D1D5
:10AFD0000722059B07339343083305936369039A5C
:10AFE0009B18636150E7434301219B18350090E7AC
:10AFF00001235B42D0E700230A201A000135636079
:10B0000029786E1C3039092903D9002BC5D0079245
:10B01000C3E74243012352183500F1E705AB009323
:10B020003A00134B2100029800E000BF0390039BFD
:10B030000133D3D1BB895B0600D584E70B9884E745
:10B0400005AB00933A000A4B2100029800F080F80B
:10B05000ECE7C04614DA0000C0D9000034DA000082
:10B06000F4D90000C6D90000CAD9000000000000D1
:10B0700023AE0000F7B5150001938A680B690090B4
:10B080000C00934200DA130022002B604332127846
:10B09000002A01D001332B6023689B0602D52B6860
:10B0A00002332B60062723681F4027D02300433339
:10B0B0001B785A1E93412268920630D422000199CF
:10B0C00043320098089EB047431C25D006232068D1
:10B0D0002A68E16803400025042B03D18D1AEB4355
:10B0E000DB171D40A3682269934201DD9B1AED180E
:10B0F0000027BD4220D1002010E00137E3682A6814
:10B100009B1ABB42D2DD220001231932019900981B
:10B11000089EB047431CF0D101204042FEBD3020C4
:10B12000E1184331087021005A1C45310978A218F2
:10B13000433202331170C1E7220001231A32019910
:10B140000098089EB047431CE6D00137D1E70000C5
:10B15000F0B589B004920A0043320593039002923D
:10B160000A7E0C000E9B6E2A00D186E01FD8632A4F
:10B1700033D008D8002A00D18CE0582A4DD02500C1
:10B1800042352A7030E0642A01D0692AF7D1196863
:10B1900025680A1D280629D508681A60002803DAE0
:10B1A0002D23029A404213706B4E0A274FE0732AF8
:10B1B00074D008D86F2A1FD0702AE0D120220968E5
:10B1C0000A43226003E0752A16D0782AD7D12200DC
:10B1D000782145321170614E22E025001A6842350F
:10B1E000111D196013682B70012365E008681A604F
:10B1F0006906D3D500B2D1E719682568081D186023
:10B2000008682E0605D5544E08276F2A1BD00A273A
:10B2100019E06D06F7D580B2F5E745314E4E0A705C
:10B2200018682268011D00681960150621D5D3072A
:10B2300002D520231A4322601027002803D120239F
:10B2400022689A4322602300002243331A70636805
:10B25000A360002B58DB0422216891432160002861
:10B2600054D1029D002B5AD02500337842352B70E3
:10B2700055E05506DBD580B2D9E71A680D68101D78
:10B280004969186013682E0601D5196002E06D0641
:10B29000FBD519800023029D23614FE01A68111D20
:10B2A0001960156800216268280000F0EDFC002894
:10B2B00001D0401B6060636823610023029A137011
:10B2C0003CE023692A0004990398059DA847431C84
:10B2D0003ED023689B0715D4079BE068984239DA73
:10B2E000180037E022000123193204990398059EC3
:10B2F000B047431C2CD00135E368079A9B1AAB4238
:10B30000F0DCE9E70025F7E70028ADD0029D390021
:10B31000FDF722FC735C013D2B700028F7D1082F4C
:10B3200009D12368DB0706D563682269934202DCF2
:10B330003023013D2B70029B5B1B2361059B07AAF9
:10B3400000932100049B0398FFF794FE431CB8D19F
:10B350000120404209B0F0BDD1D90000E2D900007F
:10B360000D4B70B51C680500A36B002B0FD1182086
:10B3700000F06EFC094BA0630360094B012243609F
:10B38000084B83600B238381002302614361002209
:10B39000A36B1D615A6170BD7C0000200E33CDABE4
:10B3A00034126DE6ECDE0500124B10B51C68A36B81
:10B3B000002B0FD1182000F04BFC0F4BA063036053
:10B3C0000E4B012243600E4B83600B2383810023CD
:10B3D00002614361A46B0B4A206961690A4BFDF766
:10B3E000F7FC012200238018594120616161480067
:10B3F000400810BD7C0000200E33CDAB34126DE64A
:10B40000ECDE05002D7F954C2DF451580CB430B571
:10B41000164B9DB00C1E1D6808DA8B2301202B6093
:10B4200040421DB030BC08BC02B01847822302A9BC
:10B430009B008B810023029008619C4200D0631E18
:10B440008B604B6101235B42CB81209A21AB2800AA
:10B45000019300F055FD431C01DA8B232B60002C77
:10B46000DFD00023029A1370DBE7C0467C00002087
:10B470000EB400B50B499CB01DAB0290069007912D
:10B4800004910948094904CB0591006802A9019378
:10B4900000F036FD0023029A13701CB008BC03B004
:10B4A0001847C046FFFFFF7F7C0000200802FFFF17
:10B4B000020010B51378541C002B05D1CC5CD45479
:10B4C0000133002CFAD110BD2200F3E7C9B2037892
:10B4D000002B04D08B4200D170470130F7E74B427C
:10B4E000594149420840F7E702780B78002A03D017
:10B4F000013001319A42F7D0D01A70470023C25C64
:10B500000133002AFBD1581E7047002330B59A4200
:10B510000AD0013AC45CCD5CAC4204D1934202D063
:10B520000133002CF6D1631B180030BD30B5050087
:10B53000002A00D130BD0C78013A6B1C2C7001310F
:10B54000002C05D19A189A42F4D01C700133FAE706
:10B550001D00EDE710B50378002B0FD10B785A4290
:10B5600053415B42184010BD0023CA5C002AFAD048
:10B57000C45C944201D10133F7E701300378002B1A
:10B58000F2D11800EFE70000F0B51F000E0087B001
:10B590000590019102920C98347800F0EAFA0822A2
:10B5A00000194378751C134036D12D2C36D1B51CAB
:10B5B00074780126002F62D0102F09D1302C07D1CA
:10B5C00020222B789343582B54D110276C780235C6
:10B5D0002D4B3900F31818000393FDF7BDFA0491C1
:10B5E00001210023494202008C4618002100303915
:10B5F00009291AD80C00A74223DD591C09D063463B
:10B60000824206D302D10499A14202DB012378438E
:10B6100020182C780135E9E72E00BCE72B2C01D04F
:10B620001E00C7E7B51C7478FAE7210041391929D3
:10B6300001D8373CDFE721006139192901D8573C8F
:10B64000D9E75A1C08D1059A23331360029B03984B
:10B65000002B09D107B0F0BD002E00D04042029A65
:10B66000002AF7D0002B01D06B1E0193029B019A98
:10B670001A60EFE73024002FAAD10827A8E7302C62
:10B680009ED00A27A4E7C046FFFFFF7F37B513000F
:10B69000064A05001068046A002C00D1044C0A0018
:10B6A00000942900FFF770FF3EBDC0467C000020DB
:10B6B000E0000020F8B505000E001400002804D0BA
:10B6C0008369002B01D100F0C1F9224B9C422DD19E
:10B6D0006C68A369A360A3891B0731D52369002B7C
:10B6E0002ED023682269F7B2981A6369F6B28342B2
:10B6F00005DC2100280000F03BF9002826D1A368D2
:10B700000130013BA36023685A1C22601F706369EB
:10B71000834204D0A389DB071AD50A2E18D1210051
:10B72000280000F025F9002812D00FE00A4B9C42B7
:10B7300001D1AC68CDE7094B9C42CAD1EC68C8E79F
:10B740002100280000F00CF80028CAD0012676421B
:10B750003000F8BD14DA000034DA0000F4D900003B
:10B76000364B70B51D6806000C00002D05D0AB6986
:10B77000002B02D1280000F069F9314B9C420FD117
:10B780006C680C23E25E93B219072DD4D90611D44C
:10B7900009230120336037331343A381404270BD36
:10B7A000284B9C4201D1AC68EBE7274B9C42E8D187
:10B7B000EC68E6E75B0713D5616B002908D023002E
:10B7C0004433994202D0300000F06AFA00236363E8
:10B7D0002422A3899343A381002363602369236008
:10B7E0000823A2891343A3812369002B0BD1A02135
:10B7F0008022A389890092000B40934203D021004C
:10B80000300000F0E1F90123A289134011D0002398
:10B81000A36063695B42A361002023698342BED1B8
:10B820000C23E25E1306BAD540231343A3810138EB
:10B83000B5E7920700D46369A360EDE77C000020C0
:10B8400014DA000034DA0000F4D9000010B5062044
:10B8500000F090FC012000F0CFFD0000F7B58A89D0
:10B8600005000C00130760D44B68002B04DC0B6C44
:10B87000002B01DC0020FEBDE76A002FFAD0002378
:10B880002E682B6080235B01216A1A4034D0606DE2
:10B89000A3895B0706D56368C01A636B002B01D0D0
:10B8A000236CC01A0200216A00232800E76AB84707
:10B8B000A189431C06D12B681D2B30D82B4ADA40B6
:10B8C000D3072CD50023636023692360CB0405D5FF
:10B8D000431C02D12B68002B00D16065616B2E6088
:10B8E0000029C7D023004433994202D0280000F039
:10B8F000D7F900206063BEE701232800B847431C46
:10B90000C6D12B68002BC3D01D2B01D0162B01D123
:10B910002E60AFE74023A2891343A381ABE7402306
:10B920000B430120A3814042A5E70F69002FA1D05E
:10B930000B680F60DB1B01930023920700D14B695A
:10B94000A360019B002B00DC94E7019B3A00216A75
:10B950002800A66AB047002803DC4023A2891343CD
:10B96000DFE7019B3F181B1A0193EAE70100402023
:10B970000B6970B505000C00002B01D1002070BDD3
:10B98000002804D08369002B01D100F05FF80B4B35
:10B990009C4209D16C680C22A35E002BEED02100E2
:10B9A0002800FFF75BFFEAE7054B9C4201D1AC683A
:10B9B000F1E7044B9C42EED1EC68ECE714DA0000AE
:10B9C00034DA0000F4D90000002310B5040003604D
:10B9D0004360836081814366C28103614361836107
:10B9E000190008225C30FFF7FFF9054B24626362FF
:10B9F000044BA362044BE362044B236310BDC046B7
:10BA0000B5C10000DDC1000015C2000041C2000048
:10BA100010B5024900F08CF810BDC04671B90000A5
:10BA200070B568254A1E55430E002900743100F098
:10BA300081F9041E08D000212A00016046600C3004
:10BA4000A0606832FFF7D0F9200070BD836913B59C
:10BA50000400002B28D18364C3640365134B144A8C
:10BA60001B6882620193984201D101238361200007
:10BA700000F020F86060200000F01CF8A0602000BA
:10BA800000F018F80022E06004216068FFF79CFFD6
:10BA900001220921A068FFF797FF02221221E06826
:10BAA000FFF792FF0123A36113BDC046BCD900007C
:10BAB00011BA0000F8B51C4B07001E68B369002BD3
:10BAC00002D13000FFF7C2FF4836B4687368013B0B
:10BAD00004D53368002B07D03668F6E70C22A55E44
:10BAE000002D0DD06834F2E704213800FFF798FFED
:10BAF00030600028F0D10C2304003B602000F8BD2A
:10BB000020000A4B656625606560A560E3602561DD
:10BB10006561A561082229005C30FFF765F965635E
:10BB2000A563A564E564E9E7BCD900000100FFFF57
:10BB3000F7B504000700002601914834002C01D11C
:10BB40003000FEBD6368A5680093009B013B009335
:10BB500001D52468F2E7AB89012B08D90E22AB5E30
:10BB6000013304D029003800019B9847064368350B
:10BB7000EBE7EC300068704770B50E001D000E2337
:10BB8000C95E96B01400002907DA00232B60B38940
:10BB90001B0611D48023DB000FE06A4600F088FB0F
:10BBA0000028F2DBF022019B12021340054A9B1889
:10BBB0005A4253412B60EDE740230020236016B02A
:10BBC00070BDC04600E0FFFFF7B502268B89050077
:10BBD0000C00334206D02300473323602361012346
:10BBE0006361F7BD01AB6A46FFF7C6FF0099070026
:10BBF000280000F09FF8002808D10C22A35E9A05C7
:10BC0000EFD4032293431E43A681E4E70F4BAB62BC
:10BC10008023A28920601343A381009B206163617C
:10BC2000019B002B0DD00E23E15E280000F052FB9B
:10BC3000002806D00322A38993431A00012313434B
:10BC4000A381A0893843A081CBE7C04611BA000088
:10BC500010B5034B0100186800F06CF810BDC04629
:10BC60007C00002082B0002900D101A9101E06D05E
:10BC7000002B06D013780B601078431E984102B059
:10BC8000704702204042FAE7C9B28218904201D1BF
:10BC90000020704703788B42FBD00130F6E70000AC
:10BCA00070B50500002910D00C1F2368002B00DAA6
:10BCB000E418280000F034FB1D4A1368002B05D15E
:10BCC00063601460280000F02CFB70BDA34209D90A
:10BCD000216860188342F3D118685B6841182160BD
:10BCE000EEE713005A68002A01D0A242F9D9196878
:10BCF0005818A0420BD120680918581819608242C0
:10BD0000E0D110685268411819605A60DAE7A04221
:10BD100002D90C232B60D5E721686018824203D139
:10BD2000106852684118216062605C60CAE7C046D2
:10BD3000181C0020032370B5CD1C9D430835060058
:10BD40000C2D1ED20C25A9421DD8300000F0E8FAB7
:10BD5000254A14682100002919D1244C2368002B9E
:10BD600003D1300000F0CAF920602900300000F053
:10BD7000C5F9431C2BD10C233000336000F0D1FAFD
:10BD800003E0002DDFDA0C233360002070BD0B6868
:10BD90005B1B19D40B2B03D90B60CC18256003E077
:10BDA0004B688C420DD11360300000F0BAFA2000CD
:10BDB00007220B30231D9043C31AE7D05A42E250AA
:10BDC000E4E763600C00EFE70C004968C3E7032376
:10BDD000C41C9C43A042E1D0211A300000F08EF92F
:10BDE000431CDBD1C7E7C046181C00201C1C0020E8
:10BDF000F8B507000D001600002905D11100FFF766
:10BE000099FF04002000F8BD002A03D1FFF748FF86
:10BE10003400F7E700F086FA2C00B042F2D231008D
:10BE20003800FFF787FF041EECD029003200FEF730
:10BE3000BFFF29003800FFF733FFE3E7F0B58E6856
:10BE400085B007000C00039201939E423CD89023DA
:10BE50008A89DB001A4234D00325096923685B1AFA
:10BE60000293636902985D43EB0F5D19019B6D10AE
:10BE700001331B18AB4200D91D00530532D52900F0
:10BE80003800FFF757FF061E09D10C233B60402303
:10BE90000120A28940421343A38105B0F0BD029A5C
:10BEA0002169FEF785FFA389144A1A4080231343B2
:10BEB000A381029B2661F61826606561019EED1A3A
:10BEC000A560019B9E4200D9019E32000399206823
:10BED000FEF777FFA36800209B1BA36023689E19D1
:10BEE0002660DAE72A003800FFF782FF061EE0D15D
:10BEF00021693800FFF7D4FEC7E7C0467FFBFFFF8C
:10BF0000F0B59FB0029005938B890F0016001B06B9
:10BF100011D50B69002B0ED14021FFF70BFF3860C4
:10BF20003861002805D10C23029A013813601FB034
:10BF3000F0BD40237B61002306AC63612033637650
:10BF40001033A37635002B78002B01D0252B46D15A
:10BF5000AB1B04930CD0320039000298FFF76EFF40
:10BF6000431C00D1AEE06269049B94466344636164
:10BF70002B78002B00D1A5E0012200235242626001
:10BF800002A9543252186E1C2360E360A360137040
:10BF9000A365317805225448FFF776FE751C00280A
:10BFA0001FD12268D30604D5532302A95B18202190
:10BFB0001970130704D5532302A95B182B2119709C
:10BFC00033782A2B16D0350000210A20E3682A781E
:10BFD0006E1C303A092A4ED9002918D010E00135DC
:10BFE000B1E7414B2268C01A012383401343236009
:10BFF0002E00CEE7059B191D1B680591002B01DB68
:10C00000099304E05B42E3600223134323602B782F
:10C010002E2B0AD16B782A2B35D1059B02351A1DA0
:10C020001B680592002B2BDB0793304E29780322E7
:10C030003000FFF729FE002806D04023801B8340F4
:10C0400022680135134323602978062228486E1C94
:10C050002176FFF719FE00283CD0264B002B25D176
:10C060000722059B07339343083305936369039ABB
:10C070009B18636166E7434301219B183500A6E7DF
:10C0800001235B42D0E700230A201A0001356360D8
:10C0900029786E1C3039092903D9002BC5D00792A5
:10C0A000C3E74243012352183500F1E705AB009383
:10C0B0003A00114B2100029800E000BF0390039B5F
:10C0C0000133D3D1BB890B985B0600D42FE7012045
:10C0D00040422CE705AB00933A00074B2100029841
:10C0E000FFF736F8EAE7C046C0D90000C6D900001D
:10C0F000CAD90000000000003DBE0000002370B55A
:10C10000064C05000800236000F060F9431C03D1D1
:10C110002368002B00D02B6070BDC046942F0020F8
:10C1200070B504000D001F2904D9162303600120F7
:10C13000404270BD436C002B04D08A009B181A68E3
:10C14000002A08D1200000F031F82A000100200068
:10C1500000F01AF8EDE70020012AEAD0511C03D1C3
:10C16000162301302360E4E7002428001C60904778
:10C170002000DEE710B5034B01001868FFF7D0FF81
:10C1800010BDC0467C000020002370B5064C0500A1
:10C1900008001100236000F001F9431C03D123685B
:10C1A000002B00D02B6070BD942F002010B500F044
:10C1B000E5F810BD70B50C000E25495F00F0BAF827
:10C1C000002803DB636D1B18636570BDA389024AF9
:10C1D0001340A381F9E7C046FFEFFFFFF8B51F004A
:10C1E0008B8905000C001600DB0505D50E23C95E02
:10C1F0000022022300F080F8A389054A280013409A
:10C20000A38132000E23E15E3B0000F02BF8F8BD65
:10C21000FFEFFFFF70B50C000E25495F00F06CF8D2
:10C22000A389421C03D1054A1340A38170BD80221B
:10C2300052011343A3816065F8E7C046FFEFFFFF9B
:10C2400010B50E23C95E00F021F810BD0B1E04D0FE
:10C25000FF2A04D98A2303608B3B180070470A70B9
:10C260000123FAE770B50500080011000022064C12
:10C2700022601A0000F0B8F8431C03D12368002B99
:10C2800000D02B6070BDC046942F0020002370B5F5
:10C29000064C05000800236000F060F8431C03D141
:10C2A0002368002B00D02B6070BDC046942F002067
:10C2B000002370B5064C050008001100236000F053
:10C2C00055F8431C03D12368002B00D02B6070BDB0
:10C2D000942F0020002370B5064C05000800236051
:10C2E00000F054F8431C03D12368002B00D02B60CE
:10C2F00070BDC046942F002070B5050008001100E5
:10C300000022064C22601A0000F050F8431C03D1B2
:10C310002368002B00D02B6070BDC046942F0020F6
:10C32000704770470B1F1B68181F002B01DA0B5852
:10C33000C018704770B50500080011000022064CB7
:10C3400022601A0000F03AF8431C03D12368002B46
:10C3500000D02B6070BDC046942F002058220120D1
:10C36000014B40421A607047942F00205822012050
:10C37000014B40421A607047942F00205822012040
:10C38000014B40421A607047942F00205822024B04
:10C3900000201A607047C046942F002058220120C8
:10C3A000014B40421A607047942F00205822012010
:10C3B000014B40421A607047942F00205822012000
:10C3C000014B40421A607047942F0020044A1368C2
:10C3D000002B00D1034B1818106018007047C0469E
:10C3E000201C0020982F002058220120014B4042A1
:10C3F0001A607047942F0020FEE7C046F8B5C0468B
:10C40000F8BC08BC9E467047F8B5C046F8BC08BCEE
:10C410009E467047646174610000000090C4000093
:10C42000EB01000099C4000017040000A1C4000043
:10C4300029070000A8C4000039080000ADC40000AE
:10C44000DF020000B8C4000083040000BDC4000087
:10C45000B1090000C9C400001B020000D3C40000E1
:10C4600031060000E1C400009F05000072616E64A7
:10C470006F6D00616C6C006C6173740066616C734D
:10C4800065007472756500252E3135732E2E2E00D1
:10C490006D616B654C697374006164644C617374A5
:10C4A0000064656C657465006A6F696E00636F7027
:10C4B0007946726F6D546F0066696E64006A6F69C9
:10C4C0006E537472696E677300756E69636F64652D
:10C4D000417400756E69636F6465537472696E6749
:10C4E00000667265654D656D6F727900E80F00003A
:10C4F000F80F00001210000090100000C81000009B
:10C50000FE100000361100005C11000098110000C0
:10C51000DA1100003012000074120000E012000076
:10C52000281300004E13000086130000CC130000F7
:10C53000F213000020140000521400008A140000BE
:10C540000E150000D61500004C160000B8160000AD
:10C550000C1700002C1700004E17000000180000F8
:10C5600046180000BE180000E80F0000E80F0000A9
:10C57000EC18000054190000D81900001E1A000021
:10C58000661A0000D81A00004A1B0000921B000027
:10C59000D81B00000E1C0000541C00009A1C000058
:10C5A000E21C0000361D0000941D0000D21D00009A
:10C5B0003C1E0000721E0000BA1E0000021F000098
:10C5C0004A1F0000841F0000CC1F00001420000040
:10C5D000E80F0000E80F0000E80F00007C200000DA
:10C5E000E80F0000B2200000DE200000142100004F
:10C5F00040210000E80F0000E80F0000E80F0000F5
:10C60000E80F000076210000C2210000E80F0000C2
:10C61000E80F000008220000582200007E220000DF
:10C62000E80F0000E80F0000E80F0000AC22000057
:10C63000DC2200000C230000422300006C230000D9
:10C64000A2230000CC230000F42300001C240000DF
:10C650004C2400007C240000A6240000D02400000C
:10C66000002500002A250000E80F0000E80F000068
:10C67000E80F0000E80F0000E80F00005A25000056
:10C68000A0250000CC250000F8250000242600008D
:10C690005A26000090260000C6260000FC26000056
:10C6A00028270000542700008A270000E80F000018
:10C6B000E80F0000E80F0000E80F0000E80F00009E
:10C6C000E80F0000E80F0000E80F0000E80F00008E
:10C6D000E80F0000E80F0000E80F0000E80F00007E
:10C6E000E80F0000B6270000EC2700002825642092
:10C6F0006974656D206C6973742900286F626A65BE
:10C70000637420747970653A20256429005374613C
:10C71000636B20756E646572666C6F770000000055
:10C72000070000000300000069C700000D29000099
:10C7300071C70000BD2900007AC70000552A00001B
:10C7400083C700001129000015000000010000004F
:10C7500002000000040000000500000006000000C8
:10C7600043616C6C696F706500686173546F6E65CE
:10C7700000706C6179546F6E650068617353657207
:10C78000766F00736574536572766F00474320744B
:10C790006F6F6B2025642075736563733B20667231
:10C7A000656520256420776F726473003C496E7460
:10C7B000656765723E003C4F626A6563743E003C8B
:10C7C0004C6973743E000D0A564D2050616E6963CA
:10C7D0003A2025730D0A006D6973630011C80000CB
:10C7E000D93600001AC80000713600001EC80000CB
:10C7F000C535000026C800006B35000030C80000B9
:10C80000013500003CC80000033400006E756C6CFC
:10C8100000686578546F496E740073696E006A73BE
:10C820006F6E476574006A736F6E436F756E740048
:10C830006A736F6E56616C75654174006A736F6ED2
:10C840004B65794174000000BCC80000453700000A
:10C85000C4C8000049370000CEC800006737000098
:10C86000D7C8000071370000E2C800007B37000025
:10C87000EEC8000085370000FEC800008F370000BA
:10C880000EC900009937000023C90000A33700003B
:10C8900038C90000AD37000044C90000B7370000B8
:10C8A00054C90000C137000060C9000053370000C0
:10C8B0006DC900005D3700006E65740068617357D4
:10C8C00069466900737461727457694669007374CC
:10C8D0006F7057694669007769666953746174754A
:10C8E00073006D79495041646472657373007374A9
:10C8F00061727448747470536572766572007374F3
:10C900006F707448747470536572766572006874E1
:10C91000747053657276657247657452657175659A
:10C92000737400726573706F6E64546F48747470C2
:10C93000526571756573740068747470436F6E6EC0
:10C9400065637400687474704973436F6E6E6563D9
:10C9500074656400687474705265717565737400F1
:10C9600068747470526573706F6E73650068747468
:10C9700070436C6F7365000D0E0F04050C0B0A06F7
:10C98000070809000000000008080800080A4A40DB
:10C9900000000A5FEA5FEA0ED92ED36E193244898D
:10C9A000330C924C924D08080000000488080804DB
:10C9B0000804848488000A448A4000048EC48000ED
:10C9C0000000048800000EC00000000008000122E2
:10C9D0004488100C9252524C048C84848E1C824CDD
:10C9E000901E1EC244924C06CA525FE21FF01EC146
:10C9F0003E02448ED12E1FE24488100ED12ED12E3D
:10CA00000ED12EC4880008000800000480048802AB
:10CA100044880482000EC00EC008048244880ED1EF
:10CA200026C0040ED135B36C0C925ED2521C925CBF
:10CA3000925C0ED010100E1C9252525C1ED01C90B4
:10CA40001E1ED01C90100ED013712E12525ED252A8
:10CA50001C8808081C1FE242524C12549814921071
:10CA60001010101E113B75B131113935B3710C9294
:10CA700052524C1C925C90100C92524C861C925C50
:10CA800092510ED00C825C1FE48484841252525264
:10CA90004C1131312A44113135BB7112524C925232
:10CAA000112A4484841EC488101E0EC808080E1063
:10CAB000080482410EC242424E048A400000000037
:10CAC00000001F0804800000000ED2524F10101CFE
:10CAD000925C000ED0100E02424ED24E0C925C9030
:10CAE0000E06C81C88080ED24EC24C10101C925262
:10CAF0000800080808024002424C101498149208DA
:10CB000008080806001B75B131001C925252000C37
:10CB100092524C001C925C90000ED24EC2000ED07D
:10CB200010100006C8049808080EC80700125252D8
:10CB30004F0011312A4400113135BB00124C8C9248
:10CB400000112A4498001EC4881E06C48C848608DE
:10CB50000808080818080C881800000C83600000FA
:10CB600000000000010000000200000003000000BF
:10CB7000040000000500000006000000070000009F
:10CB800008000000090000000A0000000B0000007F
:10CB90000C0000000D0000000E0000000F0000005F
:10CBA0001000000012000000140000001600000039
:10CBB000180000001A0000001C0000001E00000009
:10CBC00020000000230000002600000029000000D3
:10CBD0002C0000002F000000320000003600000092
:10CBE0003A0000003E000000420000004600000045
:10CBF0004B00000050000000550000005A000000EB
:10CC000061000000680000006F0000007600000076
:10CC10007D000000840000008B00000092000000F6
:10CC200099000000A0000000A7000000AE00000076
:10CC3000B5000000BC000000C3000000CA000000F6
:10CC4000D1000000D8000000DF000000E600000076
:10CC5000ED000000F4000000FB000000FF000000F9
:10CC6000B0CC0000E5370000BBCC0000293D00003F
:10CC7000C5CC0000A1390000D2CC0000993B0000D7
:10CC8000D9CC0000E93B0000E2CC0000393C0000B8
:10CC9000EECC0000353B0000FFCC0000113A000054
:10CCA0000CCD0000CD3A0000646973706C617900AE
:10CCB0006C696768744C6576656C006D6244697375
:10CCC000706C6179006D62446973706C61794F6654
:10CCD00066006D62506C6F74006D62556E706C6FA3
:10CCE00074006D62447261775368617065006D62B3
:10CCF0005368617065466F724C6574746572006E3E
:10CD0000656F506978656C53656E64006E656F5031
:10CD10006978656C53657450696E004E6F74206558
:10CD20006E6F75676820726F6F6D206576656E2017
:10CD3000616674657220636F6D70616374696F6E94
:10CD400000436F6D70616374656420466C61736845
:10CD500020636F64652073746F72650A25642062B6
:10CD600079746573207573656420282564252529E9
:10CD7000206F6620256400426164207265636F72D3
:10CD80006420666F756E6420647572696E672069D1
:10CD90006E697469616C697A6174696F6E0025648B
:10CDA0002025642025642028256420776F72647311
:10CDB00029002564207265636F7264732C202564DA
:10CDC00020776F7264732C206D617849442025644C
:10CDD0002C20636F6D70616374696F6E206379637B
:10CDE0006C657320256400526573746F72656420EE
:10CDF0002564207363726970747300537461727474
:10CE0000656400726164696F00000000AACE0000D2
:10CE1000F9460000B7CE000095490000C7CE0000DB
:10CE200015490000D5CE0000294B0000E0CE0000DF
:10CE300021470000F0CE0000A947000004CF000009
:10CE40009147000013CF00000B4D00001FCF0000E2
:10CE5000894C000028CF00002D4C000033CF00008B
:10CE6000754B00003ECF0000B14B000047CF0000E3
:10CE7000E54B000050CF0000314700005FCF0000BD
:10CE80001147000068CF0000414700006E756D62D9
:10CE90006572006E6F6E65006F7468657200706118
:10CEA000697200737472696E670064697361626CA1
:10CEB00065526164696F006D657373616765526582
:10CEC000636569766564007061636B657452656360
:10CED00065697665007061636B657453656E6400A7
:10CEE0007265636569766564496E7465676572002D
:10CEF00072656365697665644D65737361676554D2
:10CF000079706500726563656976656453747269EA
:10CF10006E670073656E64496E7465676572007351
:10CF2000656E64506169720073656E6453747269F2
:10CF30006E67007365744368616E6E656C0073653F
:10CF40007447726F757000736574506F7765720007
:10CF50007369676E616C537472656E6774680064A0
:10CF600065766963654944006C6173744D657373DC
:10CF700061676549440000000000000096300777B3
:10CF80002C610EEEBA51099919C46D078FF46A70BD
:10CF900035A563E9A395649E3288DB0EA4B8DC79DD
:10CFA0001EE9D5E088D9D2972B4CB609BD7CB17E5D
:10CFB000072DB8E7911DBF906410B71DF220B06A2D
:10CFC0004871B9F3DE41BE847DD4DA1AEBE4DD6D3D
:10CFD00051B5D4F4C785D38356986C13C0A86B643D
:10CFE0007AF962FDECC9658A4F5C0114D96C06635D
:10CFF000633D0FFAF50D088DC8206E3B5E10694C3D
:10D00000E44160D5727167A2D1E4033C47D4044B7C
:10D01000FD850DD26BB50AA5FAA8B5356C98B2425C
:10D02000D6C9BBDB40F9BCACE36CD832755CDF45DC
:10D03000CF0DD6DC593DD1ABAC30D9263A00DE510C
:10D040008051D7C81661D0BFB5F4B42123C4B356FC
:10D050009995BACF0FA5BDB89EB802280888055F7C
:10D06000B2D90CC624E90BB1877C6F2F114C6858DC
:10D07000AB1D61C13D2D66B69041DC760671DB01CA
:10D08000BC20D2982A10D5EF8985B1711FB5B6069C
:10D09000A5E4BF9F33D4B8E8A2C9077834F9000FDC
:10D0A0008EA8099618980EE1BB0D6A7F2D3D6D087C
:10D0B000976C6491015C63E6F4516B6B62616C1C6C
:10D0C000D83065854E0062F2ED95066C7BA5011B9C
:10D0D000C1F4088257C40FF5C6D9B06550E9B7123C
:10D0E000EAB8BE8B7C88B9FCDF1DDD62492DDA15FC
:10D0F000F37CD38C654CD4FB5861B24DCE51B53A1C
:10D100007400BCA3E230BBD441A5DF4AD795D83D1B
:10D110006DC4D1A4FBF4D6D36AE96943FCD96E345B
:10D12000468867ADD0B860DA732D0444E51D03333B
:10D130005F4C0AAAC97C0DDD3C710550AA4102274B
:10D1400010100BBE86200CC925B56857B3856F201B
:10D1500009D466B99FE461CE0EF9DE5E98C9D9297B
:10D160002298D0B0B4A8D7C7173DB359810DB42EBB
:10D170003B5CBDB7AD6CBAC02083B8EDB6B3BF9A07
:10D180000CE2B6039AD2B1743947D5EAAF77D29D93
:10D190001526DB048316DC73120B63E3843B649473
:10D1A0003E6A6D0DA85A6A7A0BCF0EE49DFF099373
:10D1B00027AE000AB19E077D44930FF0D2A30887E3
:10D1C00068F2011EFEC206695D5762F7CB67658093
:10D1D00071366C19E7066B6E761BD4FEE02BD38993
:10D1E0005A7ADA10CC4ADD676FDFB9F9F9EFBE8EF3
:10D1F00043BEB717D58EB060E8A3D6D67E93D1A133
:10D20000C4C2D83852F2DF4FF167BBD16757BCA612
:10D21000DD06B53F4B36B248DA2B0DD84C1B0AAFB2
:10D22000F64A0336607A0441C3EF60DF55DF67A832
:10D23000EF8E6E3179BE69468CB361CB1A8366BCC2
:10D24000A0D26F2536E2685295770CCC03470BBB12
:10D25000B91602222F260555BE3BBAC5280BBDB212
:10D26000925AB42B046AB35CA7FFD7C231CFD0B5B2
:10D270008B9ED92C1DAEDE5BB0C2649B26F263ECA4
:10D280009CA36A750A936D02A906099C3F360EEBB2
:10D290008567077213570005824ABF95147AB8E272
:10D2A000AE2BB17B381BB60C9B8ED2920DBED5E552
:10D2B000B7EFDC7C21DFDB0BD4D2D38642E2D4F1A2
:10D2C000F8B3DD686E83DA1FCD16BE815B26B9F632
:10D2D000E177B06F7747B718E65A0888706A0FFF92
:10D2E000CA3B06665C0B0111FF9E658F69AE62F852
:10D2F000D3FF6B6145CF6C1678E20AA0EED20DD752
:10D300005483044EC2B30339612667A7F71660D071
:10D310004D476949DB776E3E4A6AD1AEDC5AD6D9B1
:10D32000660BDF40F03BD83753AEBCA9C59EBBDED1
:10D330007FCFB247E9FFB5301CF2BDBD8AC2BACA81
:10D340003093B353A6A3B4240536D0BA9306D7CDF1
:10D350002957DE54BF67D9232E7A66B3B84A61C411
:10D36000021B685D942B6F2A37BE0BB4A18E0CC3D1
:10D370001BDF055A8DEF022D416C6C207461736BBD
:10D38000732073746F7070656400763037370020D7
:10D390002573202573004D656D6F727920636C6570
:10D3A00061726564004E6F206672656520746173FA
:10D3B0006B20656E747269657300000004D4000010
:10D3C0004D5F000011D40000B35F00001DD40000C9
:10D3D000835F000023D40000935F000029D4000085
:10D3E000A35F00002FD40000755C000039D400005A
:10D3F000D15F000041D40000A15D000073656E7331
:10D400006F727300616363656C65726174696F6EDE
:10D410000074656D70657261747572650074696C15
:10D4200074580074696C74590074696C745A00748F
:10D430006F75636852656164006932635265616447
:10D44000006932635772697465000000C0D400003F
:10D4500059600000CED400005D600000D7D4000009
:10D4600069600000E1D400006D600000EAD40000B3
:10D4700071600000EFD4000075600000F4D400007B
:10D480007960000000D500007D60000007D5000035
:10D490008160000010D500008560000015D50000F7
:10D4A0008960000020D500008D6000002AD50000B2
:10D4B0006160000034D5000065600000746674008F
:10D4C000656E61626C65446973706C617900676553
:10D4D000745769647468006765744865696768743F
:10D4E00000736574506978656C006C696E650072D4
:10D4F00065637400726F756E646564526563740071
:10D50000636972636C6500747269616E676C650053
:10D510007465787400746674546F7563686564002C
:10D52000746674546F7563685800746674546F75CC
:10D5300063685900746674546F75636850726573DC
:10D54000737572650057656C636F6D6520746F202D
:10D550004D6963726F426C6F636B73210000000052
:10D560000000000000000000D5640000916400008D
:10D57000B7640000C1640000CB640000B564000023
:10D58000705F73706920213D204E554C4C002F6810
:10D590006F6D652F62726F6D61676F73612F2E7093
:10D5A0006C6174666F726D696F2F7061636B616718
:10D5B00065732F6672616D65776F726B2D61726432
:10D5C00075696E6F6E6F726469636E7266352F6C0B
:10D5D00069627261726965732F5350492F535049C4
:10D5E0002E63707000535049436C6173733A3A5321
:10D5F0005049436C617373284E52465F5350495FE4
:10D60000547970652A2C2075696E74385F742C20EB
:10D6100075696E74385F742C2075696E74385F7428
:10D6200029000000000000000100000002000000CE
:10D6300016000000040000000500000006000000C5
:10D640000700000008000000090000000A000000B8
:10D650000B0000000C0000000D0000000E00000098
:10D660000F0000001A0000001B0000001400000062
:10D670001300000011000000030000001000000073
:10D680001C0000001D0000001E0000001200000031
:10D69000150000001700000018000000190000002D
:10D6A0000000000000000000F56A00002572000084
:10D6B000756B0000896B00007F6B0000F16A000051
:10D6C000E56A0000956B0000116B0000E16A000044
:10D6D000000000000000304300000000000030C3E4
:10D6E0007371727400000000FB21F93FFB210940B7
:10D6F0007CD91240FB2119407A6A1F407CD9224014
:10D70000BBFD2540FB2129403A462C407A6A2F4038
:10D710005C4731407CD932409C6B3440BBFD354086
:10D72000DB8F3740FB2139401BB43A403A463C403E
:10D730005AD83D407A6A3F404C7E40405C47414069
:10D740006C1042407CD942408CA243409C6B4440C8
:10D75000AC344540BBFD4540CBC64640DB8F47401F
:10D76000EB584840FB21494083F9A200444E6E002B
:10D77000FC291500D1572700DD34F50062DBC0001D
:10D780003C999500419043006351FE00BBDEAB0025
:10D79000B761C5003A6E2400D24D42004906E00050
:10D7A00009EA2E001C92D100EB1DFE0029B11C00DD
:10D7B000E83EA700F535820044BB2E009CE98400BA
:10D7C000B4267000417E5F00D69139005383390042
:10D7D0009CF439008B5F840028F9BD00F81F3B00E2
:10D7E000DEFF97000F980500112FEF000A5A8B00FB
:10D7F0006D1F6D00CF7E360009CB2700464FB70066
:10D800009E663F002DEA5F00BA277500E5EBC70072
:10D810003D7BF100F739070092528A00FB6BEA006A
:10D820001FB15F00085D8D00300356007BFC460091
:10D83000F0AB6B0020BCCF0036F49A00E3A91D00CA
:10D840005E619100081BE60085996500A0145F00E9
:10D850008D40680080D8FF0027734D000606310018
:10D86000CA561500C9A873007BE260006B8CC0002B
:10D8700000000040FB21F93F000000002D44743EF1
:10D88000000000809846F83C0000006051CC783BD6
:10D8900000000080831BF0390000004020257A380A
:10D8A000000000802282E336000000001DF369358D
:10D8B0000200000003000000040000000600000059
:10D8C0001C8F0000C68E0000C68E0000F48F000082
:10D8D000C28E0000C28E0000EA8F0000F48F0000AC
:10D8E000C28E0000EA8F0000C28E0000F48F00009C
:10D8F000F88F0000F88F0000F88F00000090000003
:10D90000F89900006A980000AE9800001298000094
:10D91000AE9800009E990000AE980000129800009A
:10D920006A9800006A9800009E9900001298000012
:10D930000A9800000A9800000A980000AC990000BC
:10D9400020A1000022A0000022A0000040A30000AF
:10D950001CA000001CA0000028A3000040A30000A1
:10D960001CA0000028A300001CA0000040A3000091
:10D9700036A3000036A3000036A3000044A3000035
:10D980002C2066756E6374696F6E3A200061737344
:10D99000657274696F6E2022257322206661696C3E
:10D9A00065643A2066696C6520222573222C206C00
:10D9B000696E65202564257325730A0080000020A8
:10D9C000232D302B2000686C4C0065666745464768
:10D9D00000303132333435363738394142434445EB
:10D9E000460030313233343536373839616263645A
:10D9F000656600000000000000000000000000005C
:10DA00000000000000000000000000000000000016
:10DA10000000000000000000000000000000000006
:10DA200000000000000000000000000000000000F6
:10DA300000000000000000000000000000000000E6
:10DA400000000000000000000000000000000000D6
:10DA5000000000004300504F534958000020202090
:10DA6000202020202020282828282820202020208E
:10DA7000202020202020202020202020208810105E
:10DA800010101010101010101010101010040404BA
:10DA90000404040404040410101010101010414178
:10DAA0004141414101010101010101010101010166
:10DAB000010101010101010110101010101042427A
:10DAC0004242424202020202020202020202020236
:10DAD00002020202020202021010101020000000D6
:10DAE0000000000000000000000000000000000036
:10DAF0000000000000000000000000000000000026
:10DB00000000000000000000000000000000000015
:10DB10000000000000000000000000000000000005
:10DB200000000000000000000000000000000000F5
:10DB300000000000000000000000000000000000E5
:10DB400000000000000000000000000000000000D5
:10DB500000000000000000000000000000000000C5
:04DB600000000000C1
:08DB6400A425FF7F0100000071
:10DB6C00FFFFFFFF4006000001000000E803DC059A
:10DB7C00DC05DC05DC050000FFFFFFFFFFFFFFFFFE
:10DB8C001800000019FCFFFFFFFFFFFF0200000060
:10DB9C0003000000FFFFFFFF000000000100000079
:10DBAC000000020001000000FFFFFFFF000000006A
:10DBBC00020000000000040002000000FFFFFFFF55
:10DBCC00000000000300000000000800030000003B
:10DBDC000A00000008000000010000008000002086
:10DBEC000000000014DA000034DA0000F4D9000060
:10DBFC000000000000000000000000000000000019
:10DC0C000000000000000000000000000000000008
:10DC1C0000000000000000000000000000000000F8
:10DC2C0000000000000000000000000000000000E8
:10DC3C0000000000000000000000000000000000D8
:10DC4C004300000000000000000000000000000085
:10DC5C0000000000000000000000000000000000B8
:10DC6C004300000000000000000000000000000065
:10DC7C000000000000000000000000000000000098
:10DC8C004300000000000000000000000000000045
:10DC9C000000000000000000000000000000000078
:10DCAC004300000000000000000000000000000025
:10DCBC000000000000000000000000000000000058
:10DCCC004300000000000000000000000000000005
:10DCDC000000000000000000000000000000000038
:10DCEC0043000000000000000000000000000000E5
:10DCFC000000000000000000000000000000000018
:10DD0C0043000000000000000000000000000000C4
:10DD1C0000000000000000000000000000000000F7
:10DD2C004DC2000065BC0000000000005CDA000081
:10DD3C008EC40000D6C70000D6C70000D6C70000AE
:10DD4C00D6C70000D6C70000D6C70000D6C7000053
:10DD5C00D6C70000D6C70000FFFFFFFFFFFFFFFF85
:10DD6C00FFFFFFFFFFFF0000010041534349490043
:10DD7C000000000000000000000000000000000097
:10DD8C00000000000000000000004153434949001E
:10DD9C000000000000000000000000000000000077
:10DDAC00000000000000000000000000E90000007E
:10DDBC00A967000001690000416E0000C10000006D
:04000003000069B5DB
:00000001FF
